:020000040800F2
:10800000508C002069810008DDEC0008E5DD0008E7
:10801000D9EC0008499B0008015501080000000048
:10802000000000000000000000000000690B0108D3
:1080300085BF0008000000005DF9000879170108FD
:108040006556010883810008838100088381000848
:1080500083810008838100088381000883810008F0
:1080600083810008838100088381000883810008E0
:1080700083810008838100088381000883810008D0
:10808000838100088381000883810008D19B000858
:108090004D9B0008838100086D9B000883810008C8
:1080A00083810008838100088381000883810008A0
:1080B0008381000819190108838100088381000861
:1080C0008381000883810008838100088381000880
:1080D0008381000819420108C1420108994301083F
:1080E000838100088381000883810008000000006C
:1080F0000000000000000000000000000000000080
:108100000000000000000000838100088381000857
:10811000C5310108BD320108838100088381000850
:10812000838100088381000883810008838100081F
:10813000838100088381000883810008DD9E000898
:1081400083810008E99D0008499E0008838100089A
:10815000DFF810D000F0AEFC00480047658E010843
:10816000AFF30080508C0020064880470648004747
:10817000FEE7FEE7FEE7FEE7FEE7FEE7FEE7FEE7D7
:10818000FEE7FEE74D18010851810008202A04DBB4
:10819000203A00FA02F1002070479140C2F120031A
:1081A00020FA03F3194390407047202A04DB203A59
:1081B00021FA02F00021704721FA02F3D040C2F107
:1081C0002002914008431946704740EA01039B078B
:1081D00003D009E008C9121F08C0042AFAD203E03C
:1081E00011F8013B00F8013B521EF9D27047D2B2A0
:1081F00001E000F8012B491EFBD270470022F6E790
:1082000010B513460A4604461946FFF7F0FF20460C
:1082100010BD30B505462A460B4612F8010B13F87F
:10822000014B08B1A042F8D01CB1002802D06D1C4F
:10823000F1E7284630BD421C10F8011B0029FBD194
:10824000801A704730B504460020034600E05B1CEE
:10825000934203D2E05CCD5C401BF8D030BDF0B45B
:1082600080EA0102D40F4200B2EB410F02D2024673
:10827000084611464A0042D0C30DDDB2C1F3C752D1
:10828000AD1A202D35DAC1F3160141F4000204B114
:108290005242C5F1200602FA06F12A411044B3EB1E
:1082A000D05F23D0C4B1012DA0EBC35009DCF0BCDA
:1082B0004FF0004202EAC352DBB200F5000000F0CA
:1082C00055BB400000F1807000EBC350A0F18070FE
:1082D00040EAD170490009E0490841EAC071A0EBC9
:1082E000C35000F50000400800EBC350F0BC00F0A4
:1082F00034BB6142012202EB4101001BF6E7F0BCF6
:10830000704781F00041AAE780F00040A7E780EACB
:10831000010210B502F00043400022D04A001FD0F5
:10832000010E01EB1261C0F35600C2F3560240F495
:10833000000042F40002A0FB022000047F39140474
:1083400000D0401C50EA124001D44000491EC2B285
:108350000C0604EBD010401C4008802A02D003E039
:10836000002010BD20F00100002900DA0020184391
:1083700010BD30B480EA010202F0004530F0004246
:1083800021F0004013D090B1C30DD40DC2F31601FB
:10839000C0F31600E41A41F4000140F400027D34F9
:1083A000914201D3641C00E04900002C02DA30BC89
:1083B000002070474FF400000023914201D3891A36
:1083C000034340084FEA4101F7D151B1914202D134
:1083D0004FF0004105E002D24FF0010101E06FF0E3
:1083E000010103EBC450284430BC00F0B6BA2DE9BB
:1083F000FE4F804681EA0300C00F0C46009021F03A
:10840000004123F00045B8EB0200A94105D24046E7
:10841000214690461C460B46024623F0004010437E
:1084200047D0270DC7F30A00C3F30A510290401A40
:10843000019040286BDAC3F3130040F4801B0098CE
:10844000924620B10023D2EB030A63EB0B0B019899
:108450005946C0F140025046FFF798FE06460D46C9
:1084600050465946019A00F066FA10EB0800614147
:10847000002487EA115284EAE7731A4340D0009A35
:1084800062B3019A012A4FEA075215DC001B61EB27
:1084900002014FF0004202EA0752CDE90042001CFF
:1084A00041F5801132462B4600F09DFA03B0BDE83D
:1084B000F08F40462146F9E7001B61EB0201001CEA
:1084C00041F5801300185B412018A2F5001747EB17
:1084D000030140EAD570B6196D4111E06D084FEA0D
:1084E000360645EAC0754FEA0752001B61EB0201F0
:1084F000001C41F5801149084FEA30000019514134
:1085000032462B4603B0BDE8F04F00F05DBA00984C
:10851000012240000023D0EB020263EBE0730098DD
:1085200021464FEAE074B8EB000061EB0401E9E793
:1085300083F000435BE781F0004158E72DE9FE4FEF
:1085400081EA030404F0004421F0004100944FF05C
:10855000000B23F0004350EA01045ED052EA03040A
:108560005BD0C3F30A54C1F30A552C44A4F2F3348C
:108570000194A0FB0254C1F3130141F48011C3F331
:10858000130343F4801301FB024400FB034E840AEF
:10859000970A44EA815447EA8357A4FB0768029587
:1085A0008D0A05FB07854FEA932C04FB0C54270525
:1085B000029D4FEA065847EA1637B5EB08056EEB01
:1085C000070C870E920E47EA811742EA8312A7FB37
:1085D0000201B6EB0B0164EB00042B0D43EA0C33F4
:1085E0005E1844EB1C50DA465146E7FB0201C5F326
:1085F00013044FEA0B3343EA14534FEA0432019C4D
:1086000043EA0603A4F10C040294009CCDE900B4F3
:1086100000F0E9F903B0BDE8F08F00200146F9E76A
:108620002DE9F04D81EA030404F0004B21F00045F0
:1086300014464FF0000A23F0004150EA050220D012
:1086400054EA01021DD0C5F30A570246C5F31303CD
:10865000C1F31300C1F30A5640F4801543F48013AC
:10866000A7EB0608101BD64608F2FD3873EB050091
:1086700002D308F1010801E092185B41B8F1000F44
:1086800003DA00200146BDE8F08D00204FF4801190
:10869000064684460EE0171B73EB050705D3121B35
:1086A00063EB050306434CEA010C49084FEA30002E
:1086B00092185B4150EA0107EDD152EA030012D053
:1086C00082EA040083EA0501084305D0101BAB4190
:1086D00006D20122002306E000224FF0004302E010
:1086E0006FF0010253101AEB06004CEB085110EB2F
:1086F0000A0041EB0B01BDE8F04D00F065B9C10F78
:1087000080EAE0700844CA079623002100F02EB9E1
:1087100096230022114600F029B90EB540F23341EC
:1087200002910021CDE900110A460B4600F05BF9E9
:1087300003B000BD00F0004220F00040C10DC0F3C6
:10874000160040F400007F2901DA002070479629C6
:1087500003DCC1F19601C84001E096398840002A47
:10876000F4D04042704720F00040C10DC0F3160025
:1087700040F400007F2901DA00207047962903DCCD
:10878000C1F19601C8407047963988407047C1F3DF
:108790000A5210B5C1F3130140F2FF3341F48011C6
:1087A0009A4201DA002010BD40F233439A42A2F20D
:1087B000334203DC5242FFF7F8FC10BD904010BD7D
:1087C00000F0004230F000400AD0C10D01F56071A8
:1087D000C0F3160042EA0151C20840071143704736
:1087E000002001467047000030B5041E71F10004FE
:1087F00004DB4FF00044404264EB0101141E73F1AE
:10880000000405DB1C464FF00043524263EB0403B7
:108810008B4208BF824230BD30B5041E71F10004A6
:1088200004DB4FF00044404264EB0101141E73F17D
:10883000000405DB1C464FF00043524263EB040387
:10884000994208BF904230BD01F0004330B421F09E
:10885000004150EA010206D00A0DA2F56072C1F390
:108860001301002A02DC30BC00207047440F44EAA8
:10887000C104C100E01830BC00EBC25000F06DB87C
:10888000002801DBC0F10040002901DBC1F10041FB
:1088900081427047002801DBC0F10040002901DB64
:1088A000C1F100418842704730B50B4601460020B7
:1088B0002022012409E021FA02F59D4205D303FAA2
:1088C00002F5491B04FA02F52844151EA2F1010223
:1088D000F1DC30BD2DE9F05F0546002092469B4655
:1088E00088460646814640241BE0284641464746C6
:1088F0002246FFF75AFC53465A46C01A914110D3FC
:10890000114618462246FFF741FC2D1A67EB010875
:108910004F46224601200021FFF738FC17EB0009E3
:108920004E41201EA4F10104DFDC484631462A46B0
:108930004346BDE8F09F202A06DBCB17203A41FAD8
:1089400002F043EAE07306E041FA02F3D040C2F1DC
:10895000200291400843194670470029A8BF70477C
:10896000401C490008BF20F00100704710B4B0FA65
:1089700080FC00FA0CF050EA010404BF10BC704700
:1089800049B1CCF1200421FA04F411FA0CF118BF1A
:10899000012121430843A3EB0C01CB1D4FEA0061E9
:1089A0004FEA102042BF002010BC704700EBC350BC
:1089B00010440029A4BF10BC7047401C490008BFE8
:1089C00020F0010010BC704710B5141E73F10004B4
:1089D00008DA401C41F1000192185B411A4301D1B1
:1089E00020F0010010BD2DE9F04D92469B4611B1DB
:1089F000B1FA81F202E0B0FA80F220329046FFF73D
:108A0000C5FB04460F4640EA0A0041EA0B01534603
:108A10005A46084313D0114653EA010019D0C8F151
:108A200040025046FFF7C1FB05460E4650465946E8
:108A30004246FFF7ABFB084305D0012004E0204687
:108A40003946BDE8F08D0020054346EAE0762C4328
:108A500037430A986305E40AA0EB08000022FD0AE8
:108A600044EA47540A3002D500200146E9E70105EF
:108A700010196941DDE9084500196941BDE8F04D6B
:108A8000A2E7C1F30A52C1F3130140F2FF3341F4EC
:108A900080119A4202DA00200146704740F23343C7
:108AA0009A42A2F2334202DC5242FFF77EBBFFF74A
:108AB0006DBB0000064C074D06E0E06840F0010386
:108AC00094E8070098471034AC42F6D3FFF744FB14
:108AD00060CE010880CE010870B58C1810F8015BDB
:108AE00015F0070301D110F8013B2A1106D110F847
:108AF000012B03E010F8016B01F8016B5B1EF9D14B
:108B00002B0705D40023521E0DD401F8013BFAE7D0
:108B100010F8013BCB1A921C03E013F8015B01F83B
:108B2000015B521EF9D5A142D8D3002070BD014689
:108B30000878704710B5214840792049C9788842A3
:108B40000DD01F48007850B9042003F0F5FD30B96E
:108B500001201B49087004200DF036FB0CE017487B
:108B600040791649C978884206D11548007801280D
:108B700002D1002012490870104880790F49097904
:108B800088420DD00F48007850B9032003F0D4FD7F
:108B900030B901200B49087005200DF015FB0CE0E1
:108BA0000648807905490979884206D10548007848
:108BB000012802D100200349087010BDEC250020D7
:108BC000DC080020DD08002010B51B48007830B11B
:108BD000012814D0022820D003282AD123E0032022
:108BE00003F0AAFD18B103201349087006E0042021
:108BF00003F0A2FD10B102200F4908701AE0032013
:108C000003F09AFD18B9042003F096FD08B1012085
:108C100000E00020084908700CE002F077FB01201A
:108C20000549087006E002F027FB012002490870A0
:108C300000E000BF00BF10BD4C09002021B18268D8
:108C400042F00102826003E0826822F00102826049
:108C5000704721B1826842F48072826003E08268CA
:108C600022F4807282607047014600208A6802F018
:108C700004020AB1012000E00020704701460020F4
:108C80008A6802F008020AB1012000E00020704763
:108C900030B502460020002350680F4C20400D796B
:108CA0000C6844EA05242043506090680B4C204037
:108CB000D1E902542C434D7944EA450420439060A5
:108CC000D06A20F470000C7C641EE4B2234340EAB6
:108CD0000350D06230BD0000FFFEF0FFFDF7F1FF52
:108CE000F0B504460D4600200021092D11DDE06895
:108CF000A5F10A0606EB4607072606FA07F18843A0
:108D0000A5F10A0606EB460603FA06F10843E06001
:108D10000CE0206905EB4507072606FA07F18843B2
:108D200005EB450603FA06F108432061072A0FDA2E
:108D3000606B561E06EB86071F2606FA07F188436E
:108D4000561E06EB860605FA06F10843606322E02C
:108D50000D2A0FDA206BD61F06EB86071F2606FAB0
:108D600007F18843D61F06EB860605FA06F108438D
:108D7000206310E0E06AA2F10D0606EB86071F26CD
:108D800006FA07F18843A2F10D0606EB860605FAFE
:108D900006F10843E062F0BD816841F0080181609E
:108DA000704721B1826842F4A002826003E08268C9
:108DB00022F4A00282607047816841F00401816062
:108DC00070470000F8B505460E46002490208DF847
:108DD000000001208DF801008DF802608DF803502D
:108DE0000949086005F014F900BF08E01DF8040007
:108DF00005F048F90A2000F029F8601CC4B2042CE0
:108E0000F4DB05F025F9F8BD9881214208B5012170
:108E1000082007F02DFAC020ADF8000003208DF8DF
:108E2000020010208DF803006946054803F064FF36
:108E30000120044908600449C1F8980108BD0000F8
:108E4000000C01409C8121420080214200BF411E54
:108E500089B2081EFBD1704710B51048007B10B9CD
:108E60000BF072FC20B100200C49C874012010BD29
:108E70000B480078022805DD09480078062801DA49
:108E80000120F4E70548C07C30B901200349C874CB
:108E900007F064FB014988600020E8E760090020D2
:108EA0003026002000B591B00121084607F0B0F946
:108EB000012140F2112007F0DBF94FF4004007F0E8
:108EC0009BF93920ADF8400000208DF8430010A92F
:108ED000374803F011FF00200B900E904FF46020F4
:108EE0000D9001208DF8310004208DF83C00012008
:108EF0008DF830000BA92F48FFF7CAFE0523012289
:108F00000A212C48FFF7ECFE052302220D212948F7
:108F1000FFF7E6FE052303220E212648FFF7E0FEB9
:108F2000052304220F212348FFF7DAFE21484C30A5
:108F3000009080150690002004901F4801904FF487
:108F4000806007908020059000200290042003900C
:108F50002020089000200A904FF480500990694624
:108F6000164802F0F3FE0121144802F0E3FE01214D
:108F70001048FFF76EFE01210E48FFF75FFE0D4817
:108F8000FFF70AFF00BF0B48FFF778FE0028FAD171
:108F90000848FFF711FF00BF0648FFF765FE0028ED
:108FA000FAD101210348FFF7FCFE11B000BD00001B
:108FB0000010014000240140600000200800024031
:108FC0002DE9F04104460F460C2010F07FFA0546CB
:108FD0003888288078686860206830B9012020725D
:108FE0006560AD602560BDE8F081266800E0B66888
:108FF000B06861688842FAD1B5602068A86000BF97
:10900000F1E7000070B502F0A1FB0E4909780E4AA5
:1090100052F8210080470B4909780C4A52F8210088
:10902000804704460748007800EB4000084901EB00
:10903000C00050F824501DB12046A84701490870CF
:1090400070BD00003026002070070020900700202F
:10905000B006002000200649097819B90121044A08
:10906000117003E00021024A1170052070470000D2
:10907000AF060020014601F00F000A0902EB820250
:1090800000EB4200C0B2704710B5012007F000F9B4
:10909000002007F0FDF810BD10B5A2B0002441F289
:1090A00004000C49A1F80500202048800A48007CF3
:1090B000401C0949087409A00CF09EFB01AA02A9F2
:1090C000044802F061FE0021094809F01FFF22B0A8
:1090D00010BD0000F61F00207C21002073656E6427
:1090E0002043686172676520646174610A0D000045
:1090F000A005002010B5114890F86C00642804D138
:10910000062003F033FB002010BD0C4A106F126FD5
:10911000D169884720B91C2003F028FB0020F3E721
:10912000064A106F126F516A884720B9212003F058
:109130001DFB0020E8E70120E6E70000F007002023
:1091400010B5A2B0002441F209000A49A1F80500B7
:10915000122048800848007C401C0749087407A07A
:109160000CF04AFB01AA02A9024802F00DFE22B04F
:1091700010BD0000F61F00207C21002053656E64A6
:10918000204368617267696E6744617461200A0DEB
:109190000000000000B5A1B00020009041F20300E3
:1091A0000E49A1F805000E4801780C488172042090
:1091B0000A4948800B48007C401C0A4908740AA0F0
:1091C0000CF01AFB6A4601A9044802F0DDFD0021FB
:1091D0000A4809F09BFE21B000BD0000F61F0020E8
:1091E0000C0200207C21002073656E642073746182
:1091F00074652064617461200A0D000098050020E8
:1092000010B5242003F07AFA0021034809F07EFE0D
:10921000002002F095FA10BD4826002010B5A2B03B
:10922000002441F221001549A1F805001448007DF1
:10923000C8711348808A010A1048017210484069B9
:10924000010C0E4841720E484069000E0B498872AD
:10925000042048800B48007C401C0A4908740AA07E
:109260000CF0CAFA01AA02A9044802F08DFD0421FB
:109270000248C01D0EF0F7FE22B010BDF61F002000
:10928000B01B00207C2100200A0D7368656E676AA0
:109290006979696E676461200A0D000010B5A2B09B
:1092A00000244FF481500F49A1F805005520C871E2
:1092B000AA210C48017202200A4948800A48007C11
:1092C000401C0949087409A00CF096FA01AA02A9E9
:1092D000044802F059FD02210248C01D0EF0C3FEF1
:1092E00022B010BDF61F00207C2100204F544120E9
:1092F00041434B200A0D000010B5A2B0002441F2FA
:1093000008001E49A1F805001D481EA1096801605A
:109310001EA109684160194819490968C0F8071079
:1093200017494968C0F80B101548017A1348C173F2
:1093300013480089010A1148017411488068010C22
:109340000E4841740E488068000E0C4988740C4821
:10935000017B0A48C1740D20084948800D48007CF3
:10936000401C0C4908740CA00CF046FA01AA02A992
:10937000024802F009FD22B010BD0000F61F0020D7
:10938000AE2300205332303100000000574C494ECC
:10939000470000007C21002073656E6420626D73BD
:1093A0002076657273696F6E0A0D00000648008AA8
:1093B000401C054908820846008AC82801DBAA200B
:1093C00070470020FCE700003026002010B5012186
:1093D0004FF0C05006F02CFF012005F089FD10BDB4
:1093E000F0B503460C46FF25FF261512D6B209E05C
:1093F00013F8010B80EA05010648405C80EA060587
:109400000548465C201EA4F10107BCB2F0D146EA33
:109410000520F0BD44C2010844C3010870B50246EE
:109420000C46FF25FF2309E012F8010B80EA050135
:109430000648405C80EA03050548435C201EA4F111
:109440000106B4B2F0D143EA052070BD44C2010860
:1094500044C3010810B5022101A007F042F810BD75
:109460004154000010B50A2101A007F03AF810BDE0
:1094700041542B53544154453D3F000070B50446C0
:109480000E462546288845F6A521884202D1284661
:1094900010F09CF870BD000030B589B00446202162
:1094A00001A8FEF7ABFE202101A8FEF7A7FE224689
:1094B00006A101A80CF0B0F901A8FEF7BCFE054614
:1094C000294601A807F00DF809B030BD41542B4ED4
:1094D000414D453D2573000010B5092101A007F05D
:1094E00000F810BD41542B4E414D453D3F0000005A
:1094F00010B50D2101A006F0F4FF10BD41542B550D
:109500004152545F4346473D3F00000010B50B21D8
:1095100001A006F0E6FF10BD41542B564552494FBD
:109520004E3D3F0010B525480078012845D124481C
:109530000078062837D2DFE800F003170D36202A1E
:10954000072220A12148FEF77DFE10B902201C4908
:10955000087028E00A221EA11C48FEF773FE10B90D
:109560000120174908701EE01C491848FEF751FEFB
:1095700010B104201249087015E00B2218A11348FD
:10958000FEF760FE10B905200D4908700BE00F488A
:109590000B494860154800880881144801880B4829
:1095A000FFF76CFF00BF00BF0020044908700F499F
:1095B000088080210548FEF721FE10BD1202002020
:1095C0007C21002041542B4F4B0D0A00A01C002091
:1095D00041542B4F4B0D0A303330330020170020FD
:1095E00041542B4F4B0D0A30310D0A001002002060
:1095F00010B516480078072824D2DFE800F0040AE6
:1096000007230D1F220000F077FA1CE000F078FA23
:1096100019E000F031FA16E000F05CFA0C4890F81E
:10962000760018B900200949887006E0084890F8CB
:109630007600012801D10549887004E000F00AF89D
:1096400001E000E000BF00BF10BD00007C21002051
:109650001017002010B5594890F8A800012808D12B
:109660005748007C0A2803DB0020544981F8A800F1
:1096700010BD4FF47A70534908805148007C14287B
:109680000EDD4E4890F8760018B900204C498870DD
:1096900006E04A4890F87600012801D148498870D0
:1096A0004748807807287AD2DFE800F004070E6682
:1096B0006782830000F0B0F97DE000F06DF90020D2
:1096C0003E4981F8A80076E03E4801883E4809F00E
:1096D0001DFC01284FD13D480088401C3B490880B3
:1096E00008460088092801DD00200880002136484E
:1096F00009F00CFC3548008810B900F021F93AE077
:1097000032480088012802D1FFF7C6FC33E02F4819
:109710000088022802D1FFF73DFD2CE02B4800888D
:10972000032828D029480088042802D100F050F8E6
:1097300021E026480088052802D1FFF7DDFD1AE068
:1097400022480088062802D1FFF7FAFC13E01F48E0
:109750000088072802D10CF083FE0CE01B4800882B
:10976000082802D10CF016FE05E0184800880928E8
:1097700001D10CF03DFE1EE01DE01148417C407C13
:10978000401C0F4A5074142911DD00201146087046
:109790000A4890F8760018B90020887007E009E0C0
:1097A000064890F87600012801D10549887002E04A
:1097B00001E000E000BF00BF00BF59E71017002024
:1097C0007C21002084050020800500207C050020ED
:1097D00010B5A2B000200190002441F207004B49CF
:1097E000A1F805004A48808B4949C98B484342F299
:1097F000107190FBF1F084B24548007F4349C87175
:109800004348808B0112414801724148817F3F48A3
:1098100041723F48C08B01123C488172C4723C487F
:1098200090F8291039480173394890F828103748C2
:109830004173202181735F21C1733548C17E334854
:109840000174334890F82610304841743048C08C79
:1098500001122E4881742E48C17E2C48C1742C48B8
:10986000417A2A4801752A48B0F8090001122748B0
:1098700041752748C17A254881752548B0F80B0005
:1098800001122248C17522484178204801762048BB
:10989000B0F8010001121D4841761D4841791B486E
:1098A00081761B48B0F8050001121848C1761848A7
:1098B000C179164801771648817C144841771448CD
:1098C000408A010A11488177114890F82A100F4800
:1098D000C1770F4890F82B100C4880F820100DA08D
:1098E0000BF08AFF1A200949488001AA02A90748FB
:1098F00002F04AFA0C48007C401C0B490874002115
:109900000A4809F003FB22B010BD0000F61F00203A
:10991000F00D002073656E6420444344432064616D
:1099200074610A0D000000007C210020B8050020B1
:1099300070B504460D462946204606F0C5FD70BDAB
:1099400000B5A1B0002000900AA00BF055FF3A200E
:109950000E4948806A4601A90C4802F015FA0C48E5
:10996000007C401C0A49087400210A4809F0CEFA1C
:1099700021B000BD73656E642068656172746265B4
:1099800061742064617461200A0D0000F61F0020DC
:109990007C2100209005002000B591B000200090AF
:1099A00040F6B831134809F0B1FA01281FD141F24D
:1099B00001001149A1F8050010A00BF01DFF0E4891
:1099C000C01D1349CA6E0260096F416011490A68DF
:1099D00082604968C1601020074948806A4601A931
:1099E000054802F0D1F90021024809F08FFA11B0C0
:1099F00000BD00008C050020F61F002073656E641A
:109A0000204C6F67696E20646174610D0A0000006C
:109A1000101700203CC1010800B591B00020009053
:109A200041F288310C4809F071FA012811D1000384
:109A30000A49A1F805000020488009A00BF0DCFECF
:109A40006A4601A9054802F09FF90021024809F081
:109A50005DFA11B000BD000088050020F61F00204F
:109A600053656E642052656769737465726564201E
:109A7000646174610A0D000010B54FF47A711248E8
:109A800009F044FA01281ED11048007818B90120C5
:109A90000E49087013E00D480078012806D10C48E3
:109AA000FFF7FAFC02200949087008E0074800782F
:109AB000022804D1FFF710FD00200449087000219E
:109AC000014809F023FA10BD74050020700500203C
:109AD0002017002010B540F6B831064809F016FAF4
:109AE000012805D1FFF7BEFC0021024809F00EFA5B
:109AF00010BD00007805002010B5FFF7ABFC10BDCD
:109B000010B54FF47A710E4809F000FA012815D10A
:109B10000C48007828B9FFF7F9FC012009490870C2
:109B200008E008480078012804D1FFF7E1FC002094
:109B3000044908700021024809F0E8F910BD00004E
:109B40006C0500206B05002000BFFEE700B585B066
:109B50006A460021044800F0D2FE694600200DF05C
:109B6000DDFC05B000BD00000064004010B54FF4FE
:109B70000071154800F06EFC01280DD11349124800
:109B800000F02CFC012802D100200DF0A5FD4FF4BF
:109B900000710D4800F0F6F94FF480610A4800F0BA
:109BA00059FC01280ED10949891C074800F016FC10
:109BB000012802D100200DF0B5FD4FF4806102486C
:109BC00000F0E0F910BD0000006400400200F01059
:109BD00010B50021194800F0CBFF0446022C08D034
:109BE000012C00D100E000200246002108460DF0C3
:109BF000D1FC0121114800F0BBFF0446022C08D023
:109C0000012C00D100E000200246012100200DF0CF
:109C1000C1FC0221094800F0ABFF0446022C08D029
:109C2000012C00D100E000200246022100200DF0AE
:109C3000B1FC0121014800F0A5F910BD006400400D
:109C400000B589B006F091FF0121092006F010FB54
:109C50000121480606F0ECFA0121880606F0E8FA30
:109C60000021594800F0FAFD4FF40050ADF82000F3
:109C700003208DF8220018208DF8230008A95348EE
:109C800003F03AF84FF48050ADF8200048208DF8EA
:109C9000230008A94D4803F02FF800208DF81A0082
:109CA00001208DF81B0000208DF81C008DF81D0090
:109CB0008DF81E0001208DF81F0000208DF8160081
:109CC00001208DF8170008208DF8180001208DF86C
:109CD00019000620ADF8140005A93B4800F053FC1C
:109CE0003B48407BD0B10E208DF80E0000208DF84F
:109CF0000F0001208DF810000020ADF80400ADF831
:109D00000600ADF80800ADF80A000120ADF80C001F
:109D10008DF8110001A800F0F3F903E02D490020AF
:109D200000F047FB01221021274800F023FC4120CE
:109D30008DF8000001208DF8010000208DF8020050
:109D400001208DF80300684604F0DCFF0122114673
:109D50001D4800F00FFC012251021B4800F00AFCD4
:109D600001229102184800F005FC0122D103164897
:109D700000F000FC0121144800F070FD3F208DF838
:109D8000000001208DF8010000208DF80200012064
:109D90008DF80300684604F0B5FF42208DF80000FE
:109DA00001208DF8010000208DF8020001208DF8BF
:109DB0000300684604F0A6FF06F0D9FE06A00BF0EB
:109DC0001BFD002009B000BD00680040000C0140F0
:109DD000600900200C06002063616E2032206F7045
:109DE000656E210A0000000010B586B001201349FD
:109DF0008873134806F04BFF00241AE00121114834
:109E000000F060FC90B101AA01210E4800F077FD3E
:109E10009DF80D0058B901A901200DF07FFB0598B0
:109E2000009001A80FC80AF0A1FC00E003E0601C4C
:109E3000C4B2032CE2DB00BF06B010BD60090020F5
:109E4000843700200068004010B54FF400711F48AF
:109E500000F000FB012810D11D491C4800F0BEFA9B
:109E6000012805D10DF038FC1949184800F06EF8AA
:109E70004FF40071154800F085F84FF480611348E5
:109E800000F0E8FA012820D11149891C0F4800F0A0
:109E9000A5FA012811D10F4948740846007C401CDE
:109EA00008740D4806F0F3FE01200DF03BFC084954
:109EB000891C064800F04AF802E0002005490874B1
:109EC0004FF48061014800F05DF810BD006800406B
:109ED0000200F010600900208C37002010B500212E
:109EE000194800F045FE0446022C08D0012C00D190
:109EF00000E000200246002101200DF04BFB012173
:109F0000114800F035FE0446022C08D0012C00D187
:109F100000E000200246012108460DF03BFB022133
:109F2000094800F025FE0446022C08D0012C00D17F
:109F300000E000200246022101200DF02BFB012150
:109F4000014800F01FF810BD0068004000220C4BD3
:109F5000994202D10023836111E0C1F3130201F0A1
:109F600000730BB1C2600AE001F080630BB10261C3
:109F700005E001F000630BB1826000E042607047D1
:109F80007000F030B1F5007F3AD00FDC202928D0E6
:109F900006DC01291CD004291DD0082940D11DE070
:109FA000402921D0B1F5807F3AD126E0B1F5004FAC
:109FB00031D006DCB1F5806F25D0B1F5006F2FD11F
:109FC00024E0B1F5803F12D0B1F5003F28D111E077
:109FD000154A826025E00822C26022E01022C26099
:109FE0001FE0082202611CE01022026119E0082231
:109FF000426016E01022426013E00422426010E04A
:10A00000042242600DE0042242600AE000228261E4
:10A010000422426005E0002282610422426000E0E6
:10A0200000BF00BF704700000101010010B50446E9
:10A030000B48844209D10121480606F009F90021A4
:10A040004FF0007006F004F908E00121880606F0E0
:10A05000FFF800214FF0806006F0FAF810BD000014
:10A06000006400402DE9F04104460D4617461E46A7
:10A07000ECB10020207220606060B5F5006F03D362
:10A0800004202072656002E000202072256006B185
:10A0900027B90020A0720220607208E000206072E0
:10A0A000A6723246394604F10B00FEF78EF8BDE881
:10A0B000F0812DE9F04104460D4617461E46ECB1ED
:10A0C0000020207220606060B5F5006F03D304208B
:10A0D0002072656002E000202072256006B127B979
:10A0E0000020A0720220607208E000206072A67258
:10A0F0003246394604F10B00FEF767F8BDE8F081FF
:10A1000010B50021837A012202FA03F13D4A126858
:10A1100042F001023B4B1A603A4A1C3212688A43F1
:10A12000384B1C331A60027BCAB9364A0C321268AB
:10A130008A43344B0C331A604288C38842EA034393
:10A14000304A4032847A42F834300288838842EAC6
:10A1500003432C4A4032847A02EBC4025360027BF0
:10A16000012A19D1274A0C3212680A43254B0C33B5
:10A170001A604288038842EA0343224A4032847AC2
:10A1800042F83430C288838842EA03431D4A403291
:10A19000847A02EBC4025360C27A3AB9194A121D9A
:10A1A00012688A43174B1B1D1A6006E0154A121DE0
:10A1B00012680A43134B1B1D1A60028932B9114AF7
:10A1C000143212688A430F4B14331A600289012A31
:10A1D00006D10C4A143212680A430A4B14331A602F
:10A1E000427B012A06D1074A1C3212680A43054BFA
:10A1F0001C331A60034A126822F00102014B1A60F4
:10A2000010BD0000006600402DE9FF4706460F46DE
:10A21000B94600244FF00108404600F0E9FB8DF8F4
:10A220000A8001208DF80B008DF80C00ADF80800B5
:10A230008DF80D0000253EE0204604EBD07149105A
:10A24000A4EB4101491C012902D0022920D10FE0D1
:10A2500056F83500042101EBC000000CADF80000F9
:10A2600036F8350001EBC00080B2ADF802000FE017
:10A2700056F83500042101EBC000000CADF80400D5
:10A2800036F8350001EBC00080B2ADF8060000BF23
:10A2900000BF641C204604EBD0714910A4EB4101BF
:10A2A00041B96846FFF72CFF9DF80A00401CC0B278
:10A2B0008DF80A006D1C4D45BEDB204604EBD071C5
:10A2C0004910A4EB410111B16846FFF719FFBDE841
:10A2D000FF872DE9FF4706460F46B94600244FF099
:10A2E0000108404600F084FB8DF80A8001208DF8BB
:10A2F0000B0000208DF80C000120ADF808008DF84F
:10A300000D00002547E02046E11704EB917189100C
:10A31000A4EB8101491C012906D002290DD0032993
:10A3200014D0042924D11AE056F835004FF6FF71F5
:10A3300001EA4010ADF800001AE056F835004FF67B
:10A34000FF7101EA4010ADF8020011E056F8350047
:10A350004FF6FF7101EA4010ADF8040008E056F82E
:10A3600035004FF6FF7101EA4010ADF8060000BF5E
:10A3700000BF641CE11704EB91718910A4EB81010B
:10A3800041B96846FFF7BCFE9DF80A00401CC0B208
:10A390008DF80A006D1C4D45B5DBE11704EB91719A
:10A3A0008910A4EB810111B16846FFF7A9FEBDE851
:10A3B000FF8770B504460D46132624B9314628465A
:10A3C000FFF787FF08E0012C04D131462846FFF74C
:10A3D0001BFF01E0002070BD0120FCE710B5024624
:10A3E000002001F4700343B19369C1F313042340C7
:10A3F0000BB101202DE000202BE001F0807343B170
:10A400005368C1F3130423400BB1012021E0002065
:10A410001FE001F0006343B19368C1F313042340CC
:10A420000BB1012015E0002013E001F0007343B1EF
:10A43000D368C1F3130423400BB1012009E00020CD
:10A4400007E01369C1F3130423400BB1012000E0BE
:10A45000002010BD70B504460D46002660692840F6
:10A46000002871D0B5F5807F5CD010DC082D35D088
:10A4700006DC012D20D0022D24D0042D72D127E03E
:10A48000102D31D0202D35D0402D6BD138E0B5F5D1
:10A49000004F60D009DCB5F5007F49D0B5F5806F7D
:10A4A0004CD0B5F5006F5DD14FE0B5F5803F2DD0B4
:10A4B000B5F5003F56D12FE0A0682D4901F09EF878
:10A4C000064651E0E068032101F098F806464BE0AB
:10A4D000E068082101F092F8064645E0E0681021A6
:10A4E00001F08CF806463FE02069032101F086F870
:10A4F000064639E02069082101F080F8064633E07D
:10A500002069102101F07AF806462DE060680821E4
:10A5100001F074F8064627E06068102101F06EF83B
:10A52000064621E0A069012101F068F806461BE01B
:10A53000A069022101F062F8064615E0A069042135
:10A5400001F05CF806460FE00FE0A069702101F011
:10A5500055F8064608E06068042101F04FF8064609
:10A5600002E0FFE7002600BF00E00026304670BD95
:10A57000010101001AB143690B43436102E04369E1
:10A580008B434361704730B50246002000231468B6
:10A5900024F002041460146844F00104146000E024
:10A5A0005B1C546804F001041CB94FF6FF74A3420D
:10A5B000F6D1546804F001040CB900206CE08C79E9
:10A5C000012C04D1146844F08004146003E0146882
:10A5D00024F080041460CC79012C04D1146844F078
:10A5E0004004146003E0146824F0400414600C7A02
:10A5F000012C04D1146844F02004146003E01468B2
:10A6000024F0200414604C7A012C04D1146844F026
:10A610001004146003E0146824F0100414608C7AB1
:10A62000012C04D1146844F00804146003E0146899
:10A6300024F008041460CC7A012C04D1146844F08E
:10A640000404146003E0146824F0040414608C789B
:10A65000A407CD7844EA05640D7944EA05444D79B0
:10A6600044EA05540D886D1E2C43D461146824F00F
:10A6700001041460002300E05B1C546804F0010432
:10A680001CB14FF6FF74A342F6D1546804F00104E4
:10A690000CB1002000E0012030BD2DE9F04107465B
:10A6A0000C461546264616B100212846B047BDE89F
:10A6B000F08170B506460C461546E9B2E0B20EF0E0
:10A6C00047F970BD0246002019B9D36803F00300B2
:10A6D00006E0012903D1136903F0030000E0002024
:10A6E0007047000000B589B00121052005F0C0FDCC
:10A6F0000121480605F09CFD0021524800F0AEF80B
:10A700004FF48050ADF8200003208DF8220018206F
:10A710008DF8230008A94C4802F0EEFA4FF40060CF
:10A72000ADF8200048208DF8230008A9464802F023
:10A73000E3FA00208DF81A0001208DF81B0000209C
:10A740008DF81C008DF81D008DF81E008DF81F007F
:10A750008DF816008DF817000C208DF818000120D8
:10A760008DF819000920ADF8140005A93548FFF748
:10A770000AFF00208DF80E008DF80F0001208DF8E3
:10A7800010000020ADF80400ADF80600ADF8080098
:10A79000ADF80A00ADF80C0001208DF8110001A8F9
:10A7A000FFF7AEFC012202212648FFF7E3FE14204A
:10A7B0008DF8000001208DF8010000208DF80200C6
:10A7C00001208DF80300684604F09CFA012211462E
:10A7D0001C48FFF7CFFE012251021A48FFF7CAFEBC
:10A7E000012291021748FFF7C5FE0122D103154847
:10A7F000FFF7C0FE0121134800F030F813208DF858
:10A80000000001208DF8010000208DF802000120D9
:10A810008DF80300684604F075FA16208DF80000E4
:10A8200001208DF8010000208DF8020001208DF834
:10A830000300684604F066FA04A00AF0DDFF002079
:10A8400009B000BD006400400008014063616E2053
:10A8500031206F70656E210A0000000010B50246BD
:10A860000B4600204FF6FF71BBB9146824F00204B8
:10A8700044F00104146000E0491E546804F003042D
:10A88000012C01D00029F7D1546804F00304012CF5
:10A8900001D0002032E0012030E0012B13D11468F8
:10A8A00024F00304146000E0491E546804F003041B
:10A8B0000CB10029F8D1546804F003040CB1002055
:10A8C0001CE001201AE0022B17D1146824F00104C7
:10A8D00044F00204146000E0491E546804F00304CC
:10A8E000022C01D00029F7D1546804F00304022C93
:10A8F00001D0002002E0012000E0002010BD10B5D2
:10A9000000F5D87303EB01131B6803F00403137203
:10A91000137A53B900F5D87303EB01131B6840F2A7
:10A92000FF7404EA5353136009E000F5D87303EB96
:10A9300001131B686FF0604404EAD303536000F511
:10A94000D87303EB01131B6803F00203537200F585
:10A95000D87303EB01135B6803F00F03937200F5E8
:10A96000D87303EB01135B681B0AD37400F5D8732B
:10A9700003EB01139B68D37200F5D87303EB01134B
:10A980009B681C0A147300F5D87303EB01139B68D2
:10A990001C0C547300F5D87303EB01139B681B0E5A
:10A9A000937300F5D87303EB0113DB68D37300F5E1
:10A9B000D87303EB0113DB681C0A147400F5D87319
:10A9C00003EB0113DB681C0C547400F5D87303EB24
:10A9D0000113DB681B0E937421B9C36843F0200395
:10A9E000C36003E0036943F02003036110BD00006E
:10A9F0000B49096841F00101094A116011460968D3
:10AA000043F60E729143064A11601146096841EA05
:10AA1000002111601146096821F0010111607047A1
:10AA20000066004010B502460020504B9A420CD1FF
:10AA30000B68B3F5457F00D120E00B68B3F57A7F52
:10AA400001D101201AE0022018E0936803F080632E
:10AA5000B3F1806F01D1002010E0936803F0006330
:10AA6000B3F1006F01D1012008E0936803F0805337
:10AA7000B3F1805F01D1022000E00420042874D0EB
:10AA800002F5C07303EB00131B6803F0010402F529
:10AA9000C07303EB00131C600B7A7BB94B7A0C88F4
:10AAA00043EA445302F5C07404EB001424682343C2
:10AAB00002F5C07404EB0014236010E00B7A4C68BC
:10AAC00043EAC4034C7A234302F5C07404EB001438
:10AAD0002468234302F5C07404EB001423608B7ACE
:10AAE00003F00F038B7202F5C07303EB00135B6876
:10AAF00023F00F0402F5C07303EB00135C6002F552
:10AB0000C07303EB00135B688C7A234302F5C074B7
:10AB100004EB001463608B7B1C064B7B44EA03440C
:10AB20000B7B44EA0323CC7A234302F5C07404EB85
:10AB30000014A3608B7C1C064B7C44EA03440B7C12
:10AB400044EA0323CC7B234302F5C07404EB0014D6
:10AB5000E36002F5C07303EB00131B6843F00104CC
:10AB600002F5C07303EB00131C6010BD00680040C9
:10AB700010B50246002321B1012907D002290FD1C7
:10AB800009E090681D4C00EA04030BE090681C4C3F
:10AB900000EA040306E090681A4C00EA040301E0AE
:10ABA000002300BF00BF184C181BA34216D007DCBF
:10ABB00083B16FF08060184470B1022818D111E0A1
:10ABC000B0F5007F10D0114C204448B1B0F5003FE3
:10ABD0000ED10BE002230DE000230BE0002309E07F
:10ABE000002307E0012305E0012303E0012301E046
:10ABF000002300BF00BFD8B210BD00000300000456
:10AC00000003000800000310000100080001FFF726
:10AC100070B51D48858884881C480068E8B11C48C8
:10AC200000683C21B0FBF1F0194908600846006853
:10AC3000C0001849086008460068FDF769FD06462F
:10AC40001549FDF796FB1549086000200F4908607B
:10AC50000F4908600F49086014E0114800683C285B
:10AC60000AD20B4800682044094908600C48006873
:10AC7000401C0B49086005E00020094908600120DC
:10AC80000249086070BD00006000002098000020AC
:10AC9000900000209400002000401C46A00D0020E1
:10ACA0009C00002010B5054890F8210020B929200B
:10ACB00001F05CFD002010BD0120FCE7380E0020F3
:10ACC00030B503460C46002118785D7800EB05206E
:10ACD000184DA5F81B009878DD7800EB052001B22F
:10ACE000B1F57A6F02DDA1F57A6001E0C1F57A6015
:10ACF00001B2104DA5F81D100A2906DB2846B0F850
:10AD00001D000D4DA5F8070003E000200A4DA5F831
:10AD1000070018795D7900EB0520064DA5F81F00A6
:10AD20002846B0F81F00A5F81F00987985F8210083
:10AD3000012030BD380E0020B30E002010B50346B0
:10AD40001C78074880F827405C7880F828409C7879
:10AD500080F82940DC7880F82A40012010BD0000EE
:10AD6000380E002070B505460C461646032C00DD53
:10AD70000324224629460248FDF727FA012070BD28
:10AD8000380E002030B503460C46002118785D7857
:10AD900040EA0520144D68829878DD7840EA052065
:10ADA000114DA88218795D7940EA052001B2B1F50C
:10ADB0007A6F02DDA1F57A6001E0C1F57A6001B237
:10ADC000094DE9829879DD7940EA052001B2B1F5B3
:10ADD0007A6F02DDA1F57A6001E0C1F57A6001B217
:10ADE000014D2983012030BD380E002010B50346E7
:10ADF000082900DD082118780A4CE0705878207185
:10AE00009C7808484471DC7884711C79C471587945
:10AE1000044C20729C7903484472DC7984720120CE
:10AE200010BD0000380E002010B503461878024C03
:10AE3000A076012010BD0000380E002010B503469A
:10AE40001879074C84F834005C79054880F835405F
:10AE50009C7980F83640DC7980F83740012010BDBD
:10AE6000380E002010B503461C78074880F82340B0
:10AE70005C7880F824409C7880F82540DC7880F865
:10AE80002640012010BD0000380E002030B50346DA
:10AE90000C461546082C00DD08241878FEF7EAF861
:10AEA0001449C8725878FEF7E5F812490873987883
:10AEB000FEF7E0F80F494873D878FEF7DBF80D4944
:10AEC00088731879FEF7D6F80A49C8735879FEF7DF
:10AED000D1F8084908749879FEF7CCF80549487408
:10AEE00005480B310A6802608A88828089798171FD
:10AEF000012030BD380E00202D0E002010B5044674
:10AF00000BA00AF079FC00F0B7F900F0DBF900BF04
:10AF100001200949C871094803F00FFE00BF012054
:10AF200005494872064803F008FE012010BD0000E4
:10AF300054310D0A00000000EC250020C40A002056
:10AF4000000B002010B5044602A00AF055FC0220B8
:10AF500010BD00005431300D0A00000010B5044649
:10AF600002A00AF049FC062010BD00005431310D4A
:10AF70000A00000010B5044602A00AF03DFC0620BD
:10AF800010BD00005431320D0A00000010B5044617
:10AF900004A00AF031FC03F045FF00F09FF9002007
:10AFA00010BD00005431330D0A00000010B50446F6
:10AFB00003A00AF021FC00F091F9012010BD00006F
:10AFC0005431340D0A00000010B504460AA00AF0FE
:10AFD00013FC00BF01200A4908720A4803F0ADFDC6
:10AFE00000F064F900BF002005494872064803F0EC
:10AFF00079FD072010BD00005431350D0A00000016
:10B00000EC250020EC0A0020000B002010B50446BF
:10B0100006A00AF0F1FB00F055F900200549087080
:10B02000054908700549087010BD00005431360DFF
:10B030000A000000AD000020AC000020600C0020E1
:10B0400010B5044600F03EF900F030F9002010BDC4
:10B0500010B5044602A00AF0CFFB022010BD00008C
:10B0600054320D0A0000000010B5044602A00AF098
:10B07000C3FB032010BD000054330D0A0000000084
:10B0800010B5044600200449C874088203A00AF0E1
:10B09000B3FB042010BD00003026002054340D0AFC
:10B0A0000000000010B5044602A00AF0A5FB052030
:10B0B00010BD000054350D0A0000000010B5044614
:10B0C00002A00AF099FB062010BD000054360D0ABC
:10B0D0000000000010B5044606A00AF08DFB002019
:10B0E000064948710649087500F0F8F803F09AFE21
:10B0F000002010BD54370D0A00000000D4250020A8
:10B100003026002010B5044602A00AF075FB02208C
:10B1100010BD000054380D0A0000000010B50446B0
:10B1200002A00AF069FB022010BD000054390D0A8C
:10B130000000000010B5252001F0E0FA00210348CE
:10B1400007F0E4FE012000F0FBFA10BD4C260020C1
:10B1500010B52248406A00F0004018B120A00AF063
:10B160004BFB34E01D48406A00F0804018B120A03D
:10B170000AF042FB2BE01948406A00F0005018B179
:10B1800020A00AF039FB22E01448406A00F0805009
:10B1900018B121A00AF030FB19E01048406A00F015
:10B1A000006018B11FA00AF027FB10E00B48406AAE
:10B1B00000F0806018B11FA00AF01EFB07E00748EE
:10B1C000406A00F0007010B11DA00AF015FB0348A2
:10B1D000406A40F080700149486210BD0010024092
:10B1E000B5CDB9A6BAC4B8B4CEBB0D0A00000000F4
:10B1F000B4B0BFDABFB4C3C5B9B7B8B4CEBB0D0ADB
:10B2000000000000B6C0C1A2BFB4C3C5B9B7B8B48E
:10B21000CEBB0D0A00000000C8EDBCFEB8B4CEBB2A
:10B220000D0A0000C9CFB5E72FB5F4B5E7B8B4CE25
:10B23000BB0D0A00D2FDBDC5B8B4CEBB0D0A0000DF
:10B24000424F52B8B4CEBB0D0A00000010B50848FA
:10B2500003F048FC012000F096FE064803F06DFC68
:10B260004FF4FA7000F08FFE024803F03BFC10BD73
:10B27000A00B0020B40B002010B503F061FB64208C
:10B2800000F081FE03F074FB01200349487103A024
:10B290000AF0B2FA10BD0000EC250020434C4F53D9
:10B2A000455F41435265616C790D0A0010B500207D
:10B2B0000249C871024803F015FC10BDEC250020BE
:10B2C000C40A002010B5002002490872024803F0A9
:10B2D00009FC10BDEC250020EC0A002010B5002070
:10B2E0000449887104A00AF087FA074803F0FAFBC2
:10B2F00010BD0000EC250020434C4F53455F4443F4
:10B300005265616C790D0A009C0A002010B500207E
:10B310000449887104A00AF06FFA074803F0E2FBC1
:10B3200010BD0000EC250020434C4F53455F4443C3
:10B330005265616C790D0A009C0A002010B500204E
:10B340000449887104A00AF057FA074803F0CAFBC1
:10B3500010BD0000EC250020434C4F53455F444393
:10B360005265616C790D0A009C0A0020F0B5044614
:10B370000D462946204600F009F80746615D681C25
:10B38000205C41EA002686EA0700F0BD70B502465F
:10B390004FF6FF7048F2050517E0491E12F8014B01
:10B3A00080EA042000230EE000F400462EB14FF6A0
:10B3B000FF7606EA4000684003E04FF6FF7606EAB3
:10B3C00040005E1CF3B2082BEEDB0029E5D170BD16
:10B3D00000BF00BF0C4A126F128802EB82025200BB
:10B3E000094BB3F8463092FBF3F0074AB2F8482015
:10B3F000A2F57A6200EB8003A2EB430211B2024A8B
:10B40000126F518070470000F007002000200120DB
:10B410007047000010B50E48007D18B101200D499D
:10B42000087002E000200B490870062001F084F942
:10B4300040B907480078062807D100BF064803F046
:10B4400066FB10B90220034908700248007810BD5D
:10B4500030260020AA060020500B002001460A8852
:10B46000322A01DC012070470020FCE710B500BF44
:10B470000648C08F0649898A884204DA282001F0EC
:10B4800075F9002010BD0120FCE70000F007002046
:10B49000380E002010B52048007920B1012807D0CF
:10B4A00002280DD108E011211C4801F087FB07E0BC
:10B4B0001A4801F0B5FB03E0112001F0C1FB00BF09
:10B4C00000BF3221164807F021FD012805D10BF0FD
:10B4D0004FF90021124807F019FD124890F8380082
:10B4E00000F01000B0B101200F4908750D48806BC5
:10B4F00020F010000B498863FA210948083007F052
:10B5000005FD012806D10BF083FC0021044808301A
:10B5100007F0FCFC10BD0000D42500207D69010867
:10B5200014260020380E00203026002010B52C48AC
:10B530000088401C80B22A4908800A2803DB0020CA
:10B54000088001F06DFF274880880012264981F8A5
:10B55000E80024480179244880F8E91021488079DE
:10B56000214981F8F8001F48C1791F4880F8F91077
:10B570001E480088401C80B21C49088064281DDBDE
:10B58000002008801A4800781A4991F8281088424B
:10B5900014D0184890F8280015490870082114485C
:10B5A000FFF7F4FE84B212490C7221121048417266
:10B5B00000230A220146104800F010FD0D48407893
:10B5C00001280CD10B488078012808D100200949B6
:10B5D0004870887002F0FCFB01200649487110BDDC
:10B5E000A40C0020CC380020D0370020A20C002072
:10B5F00052490020FC4800205C49002002460020FF
:10B6000002EA01030BB1012000E0002070470000B6
:10B61000002003490978C1F3800101B1012070477E
:10B62000CC380020002003490978C1F3400101B162
:10B6300001207047CC38002010B5034600202AB105
:10B640008B4201D0012006E0002004E08B4201D1B2
:10B65000012000E0002010BD00200249097A01B15C
:10B6600001207047CC38002001460020012901D07C
:10B67000032900D10120704701460020012905D08F
:10B68000022903D0042901D00A2900D101207047E2
:10B690000146002001F0800202B9012070470246F5
:10B6A00000208A4200D1012070470020012070470D
:10B6B00070B500201649086016490870002513E08F
:10B6C00005EBC50000EB400113480C18192120467A
:10B6D000FCF794FD19212046FFF758FE86B26676E6
:10B6E0003112A176681CC5B2122DE9DB4FF4F3725A
:10B6F00009490A48FCF769FD00234FF4F372064933
:10B70000074800F06BFC00F00DF800F00FF870BD7A
:10B710008C0C0020940C0020F8380020E03A002027
:10B72000E549002010B508F0F9FF10BD00200249DE
:10B730000880024908807047960C0020980C002071
:10B74000012201490A547047502600200120704709
:10B7500010B5044908698047022801D1012010BDB5
:10B760000020FCE76C00002070B50521AB4805F017
:10B770007BFA28B10020AA490873A84805F087FA87
:10B780000521A648083005F06FFA30B10020A44921
:10B790008873A248083005F07AFA05219F481030D6
:10B7A00005F062FA30B100209D4908749B481030C2
:10B7B00005F06DFA9B49C86880470646FDF700F81A
:10B7C00004460022984BFDF70FF807D22A2000F01C
:10B7D000B3FF18B92A2000F0C9FF0EE09149C868EC
:10B7E000804704469149FDF755F806D22A2000F01B
:10B7F000A3FF10B12A2000F081FF8A49C868804762
:10B800000646FCF7DDFF04460022894BFDF704F8ED
:10B8100007D2322000F090FF18B9322000F0A6FFC6
:10B820000FE08049C868804704464FF08341FDF728
:10B8300027F806D2322000F07FFF10B1322000F04E
:10B840005DFF7C4890F84C00C0F30100032802D152
:10B850002E2000F08BFF7748406CC0F381600328F6
:10B8600002D10B2000F082FF7248406CC0F30170DF
:10B87000032802D12B2000F079FF6E48406C800F26
:10B88000032802D12C2000F071FF6A48406CC0F3FD
:10B890000140032802D12D2000F068FF6548406C6C
:10B8A000C0F38150032802D10C2000F05FFF6148F3
:10B8B00090F84400C0F30000012802D10D2000F0F0
:10B8C00055FF5C48B0F84400C0F38130032802D132
:10B8D0000E2000F04BFF574890F84400C0F3800062
:10B8E000012802D10F2000F041FF524890F8440097
:10B8F000C0F3C000012802D1102000F037FF4D48EE
:10B9000090F84400C0F30010012802D1112000F08B
:10B910002DFF484890F84400C0F34010012802D1A0
:10B92000122000F023FF434890F84400C0F3811038
:10B93000032802D1132000F019FF3E48006CC0F329
:10B940008060012802D1142000F010FF3948006CFB
:10B95000C0F30060012802D1152000F007FF354830
:10B96000006CC0F34060012802D1162000F0FEFEFA
:10B970003048006CC0F30070012802D1172000F09D
:10B98000F5FE2C48006CC00F012802D1182000F0F1
:10B99000EDFE2848006CC0F34040012802D1192078
:10B9A00000F0E4FE2348006CC0F30150032802D1EC
:10B9B0001A2000F0DBFE1F48B0F84000C0F3C020A2
:10B9C000012802D11B2000F0D1FE1A4890F86C002B
:10B9D000C0F38000012802D11D2000F0C7FE1548E9
:10B9E00090F86C00C0F3C000012802D11E2000F0C6
:10B9F000BDFE104890F86C00C0F34010012802D141
:10BA00001F2000F0B3FE0B4890F86C00C0F3C0108C
:10BA1000012802D1202000F0A9FE70BD7C37002053
:10BA2000600900206C00002000002140000010414F
:10BA3000008030404825002070B51F491F4800F0A5
:10BA4000DBFF04461E491D480C3000F0D5FF0546BB
:10BA50001B481D38B0F81D00002806DD012C04D15C
:10BA6000012000F083FE002070BD15481D38B0F89D
:10BA70001D00B0F5A07F0EDD032D0CD10321114870
:10BA800005F0F2F838B1052000F070FE0D4805F021
:10BA9000FEF80020E8E70B4805F0F9F8032000F075
:10BAA0004BFE08B10020DFE7312000F045FE08B171
:10BAB0000020D9E70120D7E7AC0D00206C2600203C
:10BAC000550E00206C37002010B52A2000F034FEFF
:10BAD00000B110BD33494868804755280BDB34203E
:10BAE00000F044FE2F4948688047642813DB30206B
:10BAF00000F03CFE0FE02B49486880475A280ADCDA
:10BB0000302000F0FBFD274948688047502802DCC0
:10BB1000342000F0F3FD244890F9000055280BDB99
:10BB2000332000F023FE204890F90000692813DB41
:10BB3000312000F01BFE0FE01B4890F900005F2849
:10BB40000ADC312000F0DAFD174890F90000502897
:10BB500002DC332000F0D2FD1348007A88B111498D
:10BB600008681249FCF78CFE0BD20221104805F040
:10BB70007BF830B1352000F0F9FD0D4805F087F86D
:10BB80000EE00948007A58B1064908680749FCF7F1
:10BB900081FE05D2352000F0B1FD054805F077F8AB
:10BBA00000BF96E76C000020EC250020000020413B
:10BBB0009437002010B5002415480078002805DBD4
:10BBC00013480078042801DC012408E010480078BC
:10BBD000052803D00E480078072800D1022403204E
:10BBE00000F0AAFD88B9042000F0A6FD68B9302055
:10BBF00000F0A2FD48B9312000F09EFD28B90548AB
:10BC0000407810B90348807800B10324204610BD65
:10BC100030260020EC25002010B541F288310F4875
:10BC200007F074F9012807D1252000F09FFD0120BD
:10BC300005F082FB002010BD41F288310748001F4B
:10BC400007F064F9012807D1242000F08FFD0020BF
:10BC500005F072FB0020EEE70120ECE74C26002007
:10BC600001460878704700002DE9FC4701A92948E2
:10BC700000F09CF9DFF8A090002420E0274931F87B
:10BC8000140001F023FB0546FF2D16D0244830F8A0
:10BC9000150000EB0908234830F81460224830F8FA
:10BCA00014000199471831463846FFF75FFB20B969
:10BCB000324639464046FCF788FA601CC4B2092C6B
:10BCC000DCDB08F0C9FF694612480A3800F06EF95B
:10BCD00008210098FFF74AFB98B9009800781349AB
:10BCE000087008460078124981F82800084690F844
:10BCF000280003280CDB0A2081F829000120C870E5
:10BD000006E000200A4981F82900C87081F828005F
:10BD1000BDE8FC8766490020D037002018C701081D
:10BD200080C6010806C70108F4C601085249002070
:10BD3000FC48002021B1026842F00102026004E0E8
:10BD400002684FF6FE731A400260704710B5002279
:10BD5000026847F6F0739A430C6A8B6823430C69B8
:10BD600023434C6923438C692343CC6923434C6AA6
:10BD700023438C6A23431A430260CB6843600B68F9
:10BD800083604B68C36010BD2DE9F04706460C4642
:10BD900092460025A946A84606B114B90020BDE880
:10BDA000F087708819301FFA80F8A5222846691C90
:10BDB000CDB222545A222846691CCDB222542846BC
:10BDC000691CCDB204F800804FEA18222846691C8D
:10BDD000CDB2225420222846691CCDB222546019CB
:10BDE00010221849FCF7F1F905F11000C5B272797B
:10BDF0002846691CCDB22254B6F80500020A28462E
:10BE0000691CCDB222547088022807DB7288601941
:10BE1000F11DFCF7DAF9B0782844C5B2294620466E
:10BE2000FDF7FCFA07462846691CCDB227543A0AAA
:10BE30002846691CCDB2225429462046FDF778FDDC
:10BE40000120ACE71017002010B51B48007820B186
:10BE500001280BD002282CD117E01848407B08B1EC
:10BE6000012000E000201449087023E0002013495D
:10BE700088740846407B08B1012000E002200E498A
:10BE800008700F4804F003FF14E000200D4908700B
:10BE90000D49087003210A4804F0E6FE40B1002075
:10BEA00005490870012005498874054804F0EFFE33
:10BEB00000E000BF00BF10BDA906002060090020FF
:10BEC0009C370020A7060020A806002038B5694648
:10BED000254800F06BF81B25002438E0A91E04EB70
:10BEE000C40202EB4202009BD018FFF73FFAE8B908
:10BEF00004EBC40202EB4202009BD11804EBC40223
:10BF000002EB4203194A98182A46FCF75EF904EB43
:10BF1000C40202EB4202009BD11804EBC40202EB04
:10BF20004202134BD0182A46FCF74FF904EBC40029
:10BF300000EB40010D48405C092806D10D4800681F
:10BF40000121A14008430B490860601CC4B2122CB7
:10BF5000C4DB4FF0FF3008490860084A084903482D
:10BF600005F05EFB38BD0000E5490020F8380020F0
:10BF7000E03A00208C0C0020900C0020940C002053
:10BF8000C63C0020704710B5044606E0142009F0B6
:10BF90007FFB02F0C5F9601E84B2002CF6DC10BDF8
:10BFA00070B50646DDE90445012070BD02460A4829
:10BFB000904201D108600DE007487F38904201D1DE
:10BFC000086007E004488938904201D1086001E028
:10BFD000002070470120FCE7E54900202DE9F041F1
:10BFE00004460D4616461F463B4632462946204625
:10BFF0000FF0F4FC0120BDE8F0814161704770470B
:10C00000533530385F4443553234303110B512491E
:10C010000869804704461148807F80B9104800793C
:10C0200068B900BF01200E4988710EA009F0E4FB39
:10C03000104802F082FD10A009F0DEFB0BE007487B
:10C04000807F012807D10648007920B1FFF75EF90B
:10C050000DA009F0D1FB10BD6C000020680C002081
:10C06000EC2500204F50454E5F44435265616C798A
:10C070000D0A00009C0A0020BDF8C8EBD6B1C1F73C
:10C08000B3E4B5E70D0A0000D6B1C1F7B0CEC7B929
:10C090000D0A00002DE9F84F83464FF0000A0020FA
:10C0A0000090584601F026F98046B8F1FF0F29D0DC
:10C0B000584601F00BF90546FF2D23D01248445D88
:10C0C000DFF84890124830F8150000EB09062146C9
:10C0D0003046FFF75BF987B23755641C381230558C
:10C0E000641C0C4830F818100B4801EB000ABAF138
:10C0F000000F05D00023224631465046FFF76EFF61
:10C1000008F0AAFDBDE8F88FA6C60108D0370020C8
:10C1100080C60108F4C60108664900202DE9FC4FDD
:10C1200082460F4615461C464FF00008012001903C
:10C1300000200090DFF87CB059212278501C20703C
:10C14000A9542178481C207005F801A06A46594678
:10C15000384605F065FA00BF24E03BF818004FEAC6
:10C160002029154850F82960C6F307412278501C51
:10C170002070A954C6F307212278501C2070A954BE
:10C180002278501C2070AE5409EBC90000EB40002F
:10C19000384441782278501C2070A95408F10100DD
:10C1A00000F0FF089DF800008045D6DB0020BDE8C8
:10C1B000FC8F0000C63C002010C601082DE9FF4797
:10C1C000814690461F46DDE90C5400264FF0010AD7
:10C1D00059212278501C2070A9542178481C2070C5
:10C1E00005F8019000BF4DE0019820F07F402949FB
:10C1F00051F82610884243D19DF806102278501C31
:10C200002070A9549DF805102278501C2070A95464
:10C210009DF804102278501C2070A95406EBC6002B
:10C2200000EB4000395C2278501C2070A954B8F112
:10C23000010F03D0B8F1FF0F00D025E04FF0000A46
:10C2400006EBC60000EB40003844807D00B91BE0DF
:10C2500001212278501C2070A95408212278501CFA
:10C260002070A95406EBC60202EB42023A44911C2C
:10C270002278501905F002F921780844207003E073
:10C28000701CC6B2122EAFDB00BF504604B0BDE832
:10C29000F087000010C6010800B5A6480078C0F37A
:10C2A000001038B1A448006820F020002030A249D6
:10C2B000086005E0A048006820F020009E49086062
:10C2C0009C480078C0F3401038B19B48006820F0CB
:10C2D000400040309849086005E09748006820F029
:10C2E00040009549086093480078C0F3801038B149
:10C2F0009148006820F0800080308F49086005E098
:10C300008D48006820F080008B49086089480078DB
:10C31000C00940B18848006820F4807000F5807042
:10C320008549086005E08448006820F480708249EF
:10C3300008608048407800F0010040B17E48006805
:10C3400020F4007000F500707B49086005E07A4831
:10C35000006820F400707849086076484078C0F39F
:10C36000400040B17448006820F4806000F58060AF
:10C370007149086005E07048006820F480606E49EB
:10C3800008606C484078C0F3800040B16A4800689B
:10C3900020F4006000F500606749086005E0664829
:10C3A000006820F400606449086062484078C0F387
:10C3B000C00040B16048006820F4805000F5805013
:10C3C0005D49086005E05C48006820F480505A49E7
:10C3D000086058484078C0F3001040B156480068E3
:10C3E00020F4005000F500505349086005E0524821
:10C3F000006820F40050504908604E484078C0F36F
:10C40000401040B14C48006820F4804000F5804066
:10C410004949086005E04848006820F480404649E2
:10C42000086044484078C0F3801040B1424800683A
:10C4300020F4004000F500403F49086005E03E4818
:10C44000006820F400403C4908603A484078C00940
:10C4500040B13948006820F4803000F5803036491A
:10C46000086005E03448006820F4803032490860F4
:10C470003048807800F0010040B12F48006820F477
:10C48000003000F500302C49086005E02A480068BB
:10C4900020F4003028490860FFF7DEF858B125483D
:10C4A000007A08280DDB2448006820F010001030C6
:10C4B0002149086005E02048006820F010001E496E
:10C4C0000860FFF7C9F840B9FFF7A2F828B9FFF7ED
:10C4D000A9F810B91948407B28B1002018490880F4
:10C4E0001849088000BD16480088401C80B21449D5
:10C4F0000880C82809DD1048006820F00100401CB1
:10C500000D49086000200E4908800E480088401C34
:10C5100080B20C490880B0F5967F09DD06480068B6
:10C5200020F00200801C04490860002005490880B2
:10C5300000BFD7E7CC3800208C0C00206009002019
:10C54000960C0020980C00202DE9F04106460D467F
:10C55000114F06EBC60000EB400110480C18122EDC
:10C5600001DBBDE8F0812078A84211D0092D0FD160
:10C57000204605F04BF8607820B93878401C3870B8
:10C5800038786070A07DFF2802D0A07D401CA07587
:10C59000257000BFE5E70000940C0020F83800206B
:10C5A00010B502A009F028F910BD00004556454E0F
:10C5B000545F410D0A00000010B516A009F01CF9E7
:10C5C000002420E01648407910B9FEF755FE01E03E
:10C5D00002F028FC6420FFF7D6FC1148407910B91E
:10C5E000FEF74AFE01E002F01DFC6420FFF7CBFCE1
:10C5F00000BF0C4802F08BFA09494979884200D102
:10C6000010BD601CC4B2052CDCDB042000F0AEF8C9
:10C6100000BFF5E74556454E545F41430D0A000003
:10C62000EC2500203C0B002010B502A009F0E4F836
:10C6300010BD00004556454E545F420D0A000000F3
:10C6400010B502A009F0D8F810BD00004556454EBF
:10C65000545F430D0A00000010B517A009F0CCF894
:10C66000002422E017488079012802D1FEF766FEF7
:10C6700001E002F0F1FB6420FFF785FC11488079AE
:10C68000012802D1FEF75AFE01E002F0E5FB64202A
:10C69000FFF779FC00BF0C4802F039FA09498979A3
:10C6A000884200D110BD601CC4B2052CDADB032027
:10C6B00000F05CF800BFF5E74556454E545F444333
:10C6C0000D0A0000EC250020500B002010B51021B1
:10C6D0000648FBF793FD0648002101604160018197
:10C6E0000020044908600449086010BDF0260020BD
:10C6F00000270020540900205809002070B5054685
:10C70000284600F0E1F9284600F016F878B12846EE
:10C7100000F0AEFD0446284600F0A0FD06460548A0
:10C72000005D0021B14008400249085500BF0120CA
:10C7300070BD0000F02600202DE9F041044620469F
:10C7400000F096FD0546204600F088FD06460648A6
:10C75000405D0121B14000EA010717B10120BDE8A9
:10C76000F0810020FBE70000F026002070B50546B0
:10C770002846FFF7E1FF90B9284609F011FD284649
:10C7800000F076FD0446284600F068FD06460548A0
:10C79000005D0121B14008430249085500BF012056
:10C7A00070BD0000F02600200149C86070470000FD
:10C7B0000020024030B5044604250F4800F0AAF8D6
:10C7C0000546042D16D10D48006940F002000B49C2
:10C7D000086108464461006940F04000086106486D
:10C7E00000F098F805460548006941F6FD710840DB
:10C7F00002490861284630BDFFFF0F0000200240BB
:10C8000004200B49C96801F0010109B101200EE0C3
:10C810000749C96801F0040109B1022007E0044991
:10C82000C96801F0100109B1032000E0042070473D
:10C83000002002400348006940F08000014908617F
:10C84000704700000020024070B504460D460426E3
:10C850004FF6FF7000F05EF80646042E12D10A482B
:10C86000006940F001000849086125804FF6FF701B
:10C8700000F050F806460448006941F6FE71084091
:10C8800001490861304670BD0020024078B5064677
:10C890000C460425002000904FF6FF7000F03AF897
:10C8A0000546042D26D11448006940F001001249C4
:10C8B000086134804FF6FF7000F02CF80546042D17
:10C8C00011D1B01C0090200C009908804FF6FF7029
:10C8D00000F020F805460848006941F6FE7108405E
:10C8E0000549086106E00448006941F6FE71084008
:10C8F00001490861284678BD0020024002480349EA
:10C9000048600348486070472301674500200240A3
:10C91000AB89EFCD00B502460423FFF771FF034654
:10C9200003E0FFF76DFF0346521E012B01D1002AE1
:10C93000F7D102B90523184600BD000010B50A2939
:10C9400000DD10BD028801EB41030E4C24F82320CA
:10C95000827801EB410304EB83039A70C27801EB08
:10C96000410304EB8303DA70027901EB410304EB2A
:10C9700083031A7101EB410304EB830382689A601D
:10C9800000BFDEE75426002000B501211148FFF763
:10C99000D5FF02211048FFF7D1FF03210F48FFF711
:10C9A000CDFF04210E48FFF7C9FF05210D48FFF711
:10C9B000C5FF06210C48FFF7C1FF07210B48FFF711
:10C9C000BDFF08210A48FFF7B9FF09210948FFF711
:10C9D000B5FF00BDE0080020EC080020F8080020AA
:10C9E00004090020100900201C090020280900204B
:10C9F000340900204009002070B504460E46304638
:10CA0000A168884705462079A84203D00020A0707D
:10CA100025710EE0E078A84202D10020A07008E065
:10CA2000A078401CA070A0782188884201DB207982
:10CA3000E070E07870BD00002DE9F0410746204825
:10CA40000088401E86B2002500241E4800EBC60068
:10CA500041683846FBF714FF07D31A4800EBC500BE
:10CA600041683846FBF716FF03D240F6FF70BDE879
:10CA7000F0811EE0A81900EBD071C1F34F041148FA
:10CA800000EBC40041683846FBF704FF02D2601E89
:10CA900086B20EE00B4800EBC40041683846FBF755
:10CAA000EFFE02D2601C85B203E0064830F9340084
:10CAB000DDE7B542DEDD034830F93500D7E7000099
:10CAC0006A000020C0BB010810B50246002018E033
:10CAD0000E49095C914212D1014605E00B4C4B1CFA
:10CAE000E35C63544B1CD9B2C0F10A0303448B428C
:10CAF000F4DC07490968491E054B196010BD411C4B
:10CB0000C8B20A28E4DB00BFF8E7000000270020D5
:10CB10005809002010B524211948FBF76FFB122299
:10CB2000174918480AF06AFC1022154912311648B4
:10CB30000AF064FC12480078FF2802D01048007800
:10CB400050B90A20FFF71FFA10A008F055FE122274
:10CB50000B490C480AF052FC0948807CFF2802D09F
:10CB60000748807C58B90A20FFF70DFA0DA008F09D
:10CB700043FE10220249123103480AF03FFC10BD67
:10CB8000CC26002000F0010800F801086273705FF5
:10CB900052656164437075466C61736820310D0A9B
:10CBA000000000006273705F5265616443707546F7
:10CBB0006C61736820320D0A0000000070B50446F5
:10CBC0000D466421124806F0A1F9012808D1A047BA
:10CBD00000201049C872486000210D4806F096F9FF
:10CBE0000C48C07A112811D10A48407CA8420DD1C6
:10CBF000084840686FF30F000749884206D10020BB
:10CC00000449C872486001200449087170BD0000E1
:10CC100004260020C80E00200000EC1CD4250020B3
:10CC200010B504460220A0470220034908710021E4
:10CC3000024806F06BF910BDD4250020082600201C
:10CC400010B504461148C07A132812D10F48407C11
:10CC5000A0420ED10D4840686FF30F000C49884286
:10CC600007D100200949C87248600A4908710A4979
:10CC700088633221094806F049F9012804D10020CF
:10CC8000044908710449886310BD0000C80E0020E3
:10CC90000000EC1CD4250020380E002008260020BF
:10CCA00010B50F4948680FA1FBF7B3FA38B10C4A29
:10CCB000127E921ED1B20A4A906803F05BFF0849C7
:10CCC00048680BA1FBF7A5FA48B1054A127E032379
:10CCD00003EB8202D1B2024A906803F05FFF10BDFD
:10CCE000602100204F726465725F436F64650000CD
:10CCF0005365745F534E00002DE9F0410246002554
:10CD00000026002000230024002791F803C00CF027
:10CD10000F0591F803C00CF0100CBCF1000F03D00C
:10CD200091F802C04CEA050591F800C0BCF1000F73
:10CD300031D0146800202BE04FF0010C0CFA00F306
:10CD4000B1F800C00CEA03069E4220D183004FF0E8
:10CD50000F0C0CFA03F7BC4305FA03FC4CEA04047D
:10CD600091F803C0BCF1280F06D14FF0010C0CFA6A
:10CD700000FCC2F814C00AE091F803C0BCF1480FEF
:10CD800005D14FF0010C0CFA00FCC2F810C0401C99
:10CD90000828D1D31460B1F800C0BCF1FF0F34DD16
:10CDA000546800202EE000F1080C4FF0010808FA4A
:10CDB0000CF3B1F800C00CEA03069E4221D18300B7
:10CDC0004FF00F0C0CFA03F7BC4305FA03FC4CEAD6
:10CDD000040491F803C0BCF1280F05D100F1080C40
:10CDE00008FA0CF8C2F8148091F803C0BCF1480F9F
:10CDF00007D100F1080C4FF0010808FA0CF8C2F84E
:10CE00001080401C0828CED35460BDE8F08100009B
:10CE1000F0B50A46002300240021002500F000465A
:10CE2000B6F1004F02D11D4EF16901E01B4E716851
:10CE3000C0F3034583B200F44016B6F5401F08D195
:10CE400021F07061154E766826F07066134F7E6093
:10CE500012E000F48016B6F5801F06D1032606FA0C
:10CE600005F4A14341F0706106E0460D360103FA76
:10CE700006F6B14341F0706122B1460D360103FA66
:10CE800006F6314300F00046B6F1004F02D1034EE2
:10CE9000F16101E0014E7160F0BD00000000014051
:10CEA0000246002093680B400BB1012000E00020F7
:10CEB00070470161704701460878704710B50E4908
:10CEC0000869804702280ED103210C4803F0CCFEEC
:10CED00048B10A4803F0DBFE07498868804740B242
:10CEE0000749087007E0044908698047022802D012
:10CEF00000200349087010BD6C000020743700202A
:10CF0000EC2500202DE9F05F1048B0F802A0104A8F
:10CF10000121504608F02CFB0D480068FBF750FC3F
:10CF2000804642460B460B480B49FBF779FB064609
:10CF300000220A4BFBF7FCFA0446FBF785FC83460C
:10CF4000FFF77AFD06494881BDE8F09F60000020A8
:10CF5000B80000209A999999999913400000F03FE0
:10CF6000A00D00203CB504460B4600210020019096
:10CF700035A000680090012C32D100BF07E0585C5A
:10CF80001DF80150684001AD6854481CC1B2042925
:10CF9000F5DB9DF8050000F0F0009DF8045005F069
:10CFA0000F0540EA051010709DF805000007000EFF
:10CFB0009DF8065040EA151050709DF8060000F0EC
:10CFC000F0009DF8075040EA151090709DF807009A
:10CFD00000F00F059DF8040065F31F10D07030E0DD
:10CFE000002107E0585C1DF80150684001AD68540D
:10CFF000481CC1B20429F5DB9DF8040000F00F05C0
:10D000009DF8050065F31F1010709DF805000009DC
:10D010009DF8065005F00F0540EA051050709DF888
:10D02000070000F0F0009DF8065040EA15109070DF
:10D030009DF8070000F00F009DF8045040EA15101D
:10D04000D07000203CBD00009023B02170B5054693
:10D0500007F03CFB4443601C10B9AA20444303E0A2
:10D0600014B907F033FB04442C70200C6870200ABC
:10D07000A870EC70002070BD2DE9FF4304460F46F8
:10D080001546002003903E4695F801900B2E77D26E
:10D09000DFE806F0900607555D90779090900800C5
:10D0A00000BF00BF4B46324603A9204600F036F9C8
:10D0B000A8B90020039059219DF80C20501CC0B243
:10D0C0000390A1549DF80C10481CC0B20390665404
:10D0D00009219DF80C20501CC0B20390A154012ED0
:10D0E0002CD10020039059219DF80C20501CC0B277
:10D0F0000390A1549DF80C10481CC0B203906654D4
:10D1000009219DF80C20501CC0B20390A1540021AD
:10D110009DF80C20501CC0B20390A1542948C17A3C
:10D120009DF80C20501CC0B20390A1542548817A70
:10D130009DF80C20501CC0B20390A1543BE003ABFF
:10D14000224620490C313046FEF7E8FF33E068788C
:10D150008DF80A00A8788DF80900E8788DF80800A5
:10D1600095F8048003A8174B0C334246CDE90040E4
:10D1700030460299FFF722F808B1002003901AE028
:10D1800018E068788DF80A00A8788DF80900E8782A
:10D190008DF8080095F8048003A80A4B0C3342462A
:10D1A000CDE9004030460299FEF7FAFE08B10020B2
:10D1B000039000E000BF00BF9DF80C0004B0BDE884
:10D1C000F0830000EC3800202DE9F04706460024EB
:10D1D00000271D4890F82C001B4991F82B1000EBFC
:10D1E000012087B262222146641C72543A0A214609
:10D1F000641C72542146641C7754DFF8509000255B
:10D2000007E0134830F81500B84200D103E0681C6D
:10D21000C5B2132DF5DB00BF132D00D10224022C63
:10D220000ED00C4810F805800B4A32F8152002EB9E
:10D23000090130194246FAF7C8FF04EB080084B22E
:10D240002046BDE8F0870000FC480020D0370020D1
:10D25000BAC60108A6C6010880C6010801460A46EA
:10D26000C81701EB5070C010A1EBC000C0B27047EE
:10D2700001460A46C81701EB5070C0F3C70070475B
:10D2800000B5FEF7C5F938B10F48006820F0080076
:10D2900008300D49086005E00B48006820F00800E0
:10D2A00009490860FEF7BEF938B10748006820F068
:10D2B0000400001D0449086005E00348006820F0F0
:10D2C00004000149086000BD8C0C00200246FF20CC
:10D2D000002108E0064B33F81130934201D1084693
:10D2E00003E04B1CD9B21329F4D300BF70470000F0
:10D2F000BAC601080246FF20002108E0064B33F8B9
:10D300001130934201D1084603E04B1CD9B20929E0
:10D31000F4D300BF7047000018C701082DE9F041A1
:10D3200004460E4615460020002100220027DFF8A3
:10D33000E4C0ACF80A704FF059089446521C04F847
:10D340000C809446521C04F80C504FF00908944687
:10D35000521C04F80C8000BF56E001EBC10707EB3C
:10D36000470C2C4F0C3717F80C701F405FB901EBBE
:10D37000C10707EB470C274F0C3717F80C709F427B
:10D3800001D00A2D3ED1244F3F68CF4007F001075E
:10D39000C7B301201F4F7F897F1CDFF878C0ACF82E
:10D3A0000A701E4F57F82170C7F30748174602F15D
:10D3B000010C0CF0FF0204F80780184F37F82170B9
:10D3C000C7F30728174602F1010C0CF0FF0204F81E
:10D3D0000780124F17F82180174602F1010C0CF05C
:10D3E000FF0204F8078001EBC10707EB470C094F68
:10D3F0000C3717F80C80174602F1010C0CF0FF02F5
:10D4000004F807804F1CF9B21229A6DB3270BDE880
:10D41000F0810000EC380020900C002010C60108BC
:10D420002DE9F8433C480088002806DD3A4800888A
:10D43000401E39490880BDE8F883FFF721FFFEF759
:10D440002BFF364890F8270000B1F4E73448006815
:10D450000090002515E00098E84000F0010010B1B0
:10D460004FF0090807E005EBC50000EB40012D482F
:10D47000405C20F0010841462846FFF765F8681C2B
:10D48000C5B2122DE7DB1B262748007800EBC00051
:10D4900000EB400123480C1820782349097801EB60
:10D4A000C10101EB4101214A515C88421AD0B11EF1
:10D4B0002046FDF76BFF87B267763912A176207898
:10D4C0001949097801EBC10101EB4101174A505498
:10D4D0001749154A127806FB0210002332462146EE
:10D4E000FEF77CFD10480078401C0F490870084684
:10D4F0000078122801DB002008700E480078401CDC
:10D50000C0B20C4908700A2803DB0020087007F03D
:10D51000C5FB00BF8FE70000880C0020FC480020FE
:10D520008C0C0020F8380020A00C0020E03A0020ED
:10D53000E5490020A10C00200246002112E001EB89
:10D54000410000EBC1000E4B03EB0010007890424D
:10D5500006D101EB410000EBC10003EB0010704766
:10D56000481CC1B2022909D201EB410000EBC10005
:10D57000034B03EB00100078FF28E0D10020EEE71A
:10D580002C1500202DE9F0478246BAF1010F34D165
:10D59000EB2182200BF028FC6449088008460088B3
:10D5A000B0F5004F0CDB08460088B0F5803F07DA85
:10D5B000084600884FF6FF71081A5C49088008E0A9
:10D5C0005A4800884FF6FF71884202DB0020574915
:10D5D000088056480088FBF7A0F88046544A554B0F
:10D5E000FAF7ACFF06460022534BFBF719F8044646
:10D5F000FBF72AF95149086094E0BAF1020F59D1BA
:10D60000E321B2200BF0F0FB48490880084600886F
:10D61000B0F5004F0ADB01204949088043480088E3
:10D620004FF6FF71081A4149088002E00020444982
:10D6300008803E480088FBF770F880463C4A3D4B26
:10D64000FAF77CFF064600223B4BFAF7E9FF044657
:10D65000FBF7FAF83949086008460068FBF7B0F8AC
:10D6600006464FF03332374BFAF768FF0446364A26
:10D67000364BFAF7D5FF8046FBF7E6F82F490860EE
:10D680002F48008801284DD14FF4FA61304805F049
:10D690003DFC012806D12FA008F0AEF800212C484F
:10D6A00005F034FC254801680020FAF72AFE2349DA
:10D6B000086037E0BAF1030F34D1E321B4200BF056
:10D6C00093FB1A49088008460088B0F5004F0CDB30
:10D6D00008460088B0F5803F07DA084600884FF614
:10D6E000FF71081A1149088008E0104800884FF6B9
:10D6F000FF71884202DB00200C4908800B4800883B
:10D70000FBF70BF806460A4A1B4BFAF717FF0446CD
:10D710000022094BFAF784FF8046FBF795F807498A
:10D72000086000BF05480068BDE8F087CA00002017
:10D73000FCA9F1D24D622040E0FFEF40CC00002078
:10D74000D0000020F308CA40F6285C8FC2F51340D1
:10D75000E40000204E6567617469766520766F6C21
:10D76000746167652073616D706C65206661756CAE
:10D7700074210D0A000000004D6210400146087D32
:10D7800070470146087C70470146C87C032801D1D8
:10D7900001207047C87C042801D10020F9E700204F
:10D7A000F7E70146887C012800D17047887C08B9DA
:10D7B0000020FAE70020F8E70148B0F90A007047B6
:10D7C000A00D00200148406870470000A00D002017
:10D7D000F8B5044600200090554A106F126FD16BC7
:10D7E000884707465348007830B101283BD00228CB
:10D7F0004DD003287CD169E02046FAF7E1FF0546C9
:10D800004D4A4E4BFBF708F80BD22046FAF7D8FFEB
:10D8100005464B4A4B4BFAF7E7FF02D20320009034
:10D8200020E049492046FBF72BF80BD22046FAF7B7
:10D83000C7FF0546454A464BFAF7EEFF02D20120E4
:10D8400000900FE04FF081412046FBF723F807D20C
:10D8500040492046FBF714F802D20220009001E074
:10D860000020009059E038492046FBF709F80BD218
:10D870002046FAF7A5FF0546374A384BFAF7CCFFA2
:10D8800002D20120009001E00020009045E04FF01E
:10D890007F512046FAF7F4FF07D231492046FAF7C4
:10D8A000F9FF02D2032000900FE04FF081412046A3
:10D8B000FAF7F0FF07D227492046FAF7E1FF02D234
:10D8C0000220009001E00020009026E04FF07F5100
:10D8D0002046FAF7D5FF0CD22046FAF771FF05462D
:10D8E0001D4A1E4BFAF798FF03D20320009010E068
:10D8F00010E04FF081412046FAF7CCFF07D21949DA
:10D900002046FAF7BDFF02D20220009001E000207D
:10D91000009002E00020009000BF00BF694612485E
:10D92000FFF76AF80349087008460078F8BD000060
:10D93000F0070020600C00208195438B6CE7E73FE7
:10D940009EEFA7C64B37ED3F333373409A999999B1
:10D950009999B93F0000C0407B14AE47E17A843FFB
:10D960000AD7233C0000E040602600202DE9FC4758
:10D970001848046801681848FAF7C3FC05461549B9
:10D9800008681649FAF7C3FC06462946FAF7F1FC7F
:10D9900004462046FAF714FF07460022104BFAF718
:10D9A000CAFD05460E462046FAF70AFF0746002242
:10D9B0000B4BFAF7C3FD81462A463346FAF730FE91
:10D9C000CDE90001FAF740FF04460648046020460E
:10D9D000BDE8FC87A00D00200000A0403333A34029
:10D9E000000024406C0000200148B0F90800704796
:10D9F000A00D00200146487C012800D17047487CDA
:10DA000008B90020FAE70020F8E700000148007894
:10DA100070470000AD00002010B56B480088401C26
:10DA200080B2694908800A287EDB002008806748A8
:10DA3000B0F84000B0F5FA7F33DA6448B0F840003F
:10DA4000401C6249A1F840000846B0F84000B0F51B
:10DA5000FA7F26D1002008720846407F032803D0B1
:10DA60000846407F02281CD1002058490877012031
:10DA70004877002081F8220088714874A1F840009E
:10DA800081F8240081F8250081F82700C8735048E8
:10DA90000079012803D100204D498861087100F008
:10DAA0003DFC4A4890F8240058B14A48007820F0DC
:10DAB0000100484908700846007820F0020008700C
:10DAC0000CE04448007820F00100401C41490870F7
:10DAD0000846007820F00200801C08703B4890F84F
:10DAE000250058B13B48007820F0040039490870FF
:10DAF0000846007820F0080008700CE035480078EF
:10DB000020F00400001D334908700846007820F01A
:10DB10000800083008702D48B0F8540070B12B4848
:10DB2000B0F85400401E00E04CE02849A1F8540031
:10DB30000846B0F8540008B90020C8732648008889
:10DB4000401C80B224490880642800DA10BD0020FF
:10DB5000214908801D4890F82900D8B11B4890F849
:10DB60002900401E194981F82900084690F829002B
:10DB700080B90846C07801280CD10020C87008463A
:10DB800090F82800002805DD084690F82800401E7F
:10DB900081F828000D48007A30B10E48007820F056
:10DBA00010000C4908700DE00A48007820F01000C1
:10DBB00010300849087000204877FF208877887067
:10DBC00000F0ACFB00BFC1E7560D0020FC48002070
:10DBD000C4480020680C0020540D0020014601F0CC
:10DBE0000F01092903DD01F13700C0B2704701F1CF
:10DBF0003000C0B2FAE701460911092903DD01F13D
:10DC00003700C0B2704701F13000C0B2FAE7704788
:10DC100070B505460E4608480670002404E0285DED
:10DC200006490855601CC4B2034800788442F6DBFC
:10DC300003F0C4FF70BD0000610D0020580D0020EE
:10DC40000146002004E0054A125C0A54421CD0B28E
:10DC5000034A12789042F6DB70470000580D00200E
:10DC6000610D002070B504460D4604F0B3F8064679
:10DC700032462946204606F035FA70BD70B5054695
:10DC80000E4608480670002404E0285D0649085541
:10DC9000601CC4B2034800788442F6DB04F012F83A
:10DCA00070BD0000610D0020580D002010B504F07B
:10DCB00023F910BD10B5044606F0A8FA002001496A
:10DCC000087010BD600D002001480078704700000A
:10DCD000610D00207FB505460E48006800900E4893
:10DCE00000788DF80400002405E0295D0DF10500A1
:10DCF0000155601CC4B2084800788442F5DB01205D
:10DD00008DF80D00054948709DE80F0005F0E0F919
:10DD10007FBD0000640D0020620D0020FC48002043
:10DD20000149087070470000620D002020B940F2E0
:10DD3000B471044A116003E040F2B471014A116009
:10DD400070470000640D0020704700002DE9F0418D
:10DD500005460E4604F03EF804460A48007878B9B5
:10DD60007F2020706570A67003270020FFF7DEFF7C
:10DD700004F02AFC384604F08DF8012001490870AF
:10DD8000BDE8F081600D00202DE9F04105460E460A
:10DD900004F020F880460D480078A8B9A5B1002409
:10DDA00004E0305D08F80400601C84B2AC42F8DB8B
:10DDB0002F460020FFF7BAFF04F006FC384604F0B7
:10DDC00069F8012001490870BDE8F081600D00206C
:10DDD00010B503F095FE10BD014608787047014666
:10DDE0000878704700BFFEE770B50446002500BF05
:10DDF00000259120005D06281ED2DFE800F0031EFA
:10DE00004C4D5C7094F85400032815DB04F170004D
:10DE10000DF092FC80B904F1940104F170000DF052
:10DE2000ABFC40B1012191200155002084F8900005
:10DE30000021AC200155012567E094F89930942227
:10DE40001159207804F19A02A668B04784F8980026
:10DE500094F89000401C84F8900094F89800FF28F3
:10DE60000ED00221912001550021AC200155012541
:10DE700094F8540081280DD1032084F8540009E05F
:10DE800094F8901094F84400814203DB042191201F
:10DE90000155012539E038E094F8901094F84400D9
:10DEA000814203DB04219120015502E001219120F0
:10DEB0000155012529E0002191200155D4F8A80041
:10DEC00020B10121D4E92902904706E0206D20B15C
:10DED0000121226DD4F8A4009047012515E000210E
:10DEE00091200155D4F8A80028B10220D4E92921B5
:10DEF00009F058FD07E0206D28B10220D4F8A420D5
:10DF0000216D09F04FFD012500BF00BF012D04D197
:10DF10009120005D04287FF46BAF25B122780421A5
:10DF2000012009F03FFD70BD10B504469120005D51
:10DF3000022811D194F8901094F84400814203DB38
:10DF400004219120015502E00321912001552278FE
:10DF50000421012009F026FD10BD70B504460D46D0
:10DF60009120005D022803D09120005D03280DD18F
:10DF700094F89800A84209D105219120015594F800
:10DF80005400032802DB2046FFF72EFF70BD00007F
:10DF900070B50024002515E001201B49086005200C
:10DFA000FAF754FF6006040E1848D0F81C0108B1B7
:10DFB00044F001040020144908600520FAF746FFE8
:10DFC000681CC5B2082DE7DB00200F49086005205A
:10DFD000FAF73CFF00200D49C1F89C010520FAF733
:10DFE00035FF0120084908600520FAF72FFF0020BF
:10DFF0000649C1F898010520FAF728FF01200249D7
:10E00000091D0860204670BD988121420080214290
:10E0100010B501200C4908600520FAF717FF012010
:10E020000A49C1F898010520FAF710FF00200649B7
:10E0300008600520FAF70AFF00200449C1F898019A
:10E040000520FAF703FF10BD9C8121420080214288
:10E0500010B50020094908600520FAF7F7FE0120F5
:10E060000749C1F898010520FAF7F0FE012003499D
:10E0700008600520FAF7EAFE10BD00009C812142ED
:10E080000080214270B50446002018490860002530
:10E090001CE004F0800020B101201449091D086033
:10E0A00003E000201149091D086001200F490860A4
:10E0B0000520FAF7CBFE00200D49C1F89801052094
:10E0C000FAF7C4FE6006040E681CC5B2082DE0DB3A
:10E0D00001200649091D08600549C1F8980105207D
:10E0E000FAF7B4FE00200149086070BD9881214212
:10E0F0000080214210B54FF400600B4908600AF01F
:10E1000032FD4FF480600849091F08600AF02BFDBA
:10E110004FF48060044908600AF025FD4FF4006068
:10E120000149091F086010BD140C014010B54FF4DF
:10E130000060094908600AF016FD4FF48060064946
:10E1400008600AF010FD4FF480600349091D086063
:10E150000AF009FD10BD0000100C014070B5054625
:10E160000024002618E06006040E4FF480600F497A
:10E1700008600AF0F8FC0D480838006800F40060F8
:10E1800008B1601CC4B24FF480600849091D0860E2
:10E190000AF0E9FC701CC6B2082EE4DB15B9FFF7E3
:10E1A000C5FF01E0FFF7A6FF204670BD100C01403F
:10E1B00070B50446002524E004F0800020B14FF43F
:10E1C00000601149086004E04FF400600E49091D29
:10E1D00008600AF0C8FC4FF480600B4908600AF040
:10E1E000C2FC4FF480600849091D0860072D02D168
:10E1F0004000091F08606006040E0AF0B4FC681CA9
:10E20000C5B2082DD8DB70BD100C014010B54FF41D
:10E2100000600A490860401008600AF0A4FC4FF44E
:10E2200000600649091D08600AF09DFC4FF48060FB
:10E230000249091D08600AF096FC10BD100C01404F
:10E2400010B54FF40060074908604010091F0860CE
:10E250000AF089FC4FF400600249091F08600AF0C7
:10E2600082FC10BD140C014010B54FF400600E4943
:10E2700008600AF078FC4FF480600B4908600AF0EF
:10E2800072FC09480838006800F4006008B10124F5
:10E2900000E000244FF480600349091D08600AF083
:10E2A00062FC204610BD0000100C014001460A88A7
:10E2B000002000BF064BB3F83530934206DB00BFA9
:10E2C000034BB3F843301433934200DC0320704710
:10E2D000F00700202DE9F04104462568002600BF24
:10E2E0000D48B0F839008046FAF712FA0746294679
:10E2F000FAF7C6FA01D201260BE000BF0648C08F2C
:10E300008046FAF705FA07462946FAF7C3FA00D21B
:10E3100002263046BDE8F081F0070020704700007B
:10E320007F20034908600020024908707047000000
:10E33000002C0040E901002010B51748C06940F4E6
:10E3400000601549C86140F2FF30144908607F2021
:10E35000091F08600846006840F08000086000203F
:10E360000146002807DA0A07140E0D4A00F00F03D1
:10E370001B1FD45403E00A07130E0A4A135400BFAC
:10E380000020012181404209920002F1E022C2F8FE
:10E39000001100BF10BD000000100240042C00401E
:10E3A00018ED00E000E400E00EB541F28730ADF872
:10E3B00000006748019069466648FAF701FE42F29C
:10E3C0000F70ADF800006448019069466148FAF7A3
:10E3D000F7FD40F6C310ADF800005F4801906946B4
:10E3E0005C48FAF7EDFD40F6C310ADF800005B485D
:10E3F000019069465748FAF7E3FD41F28730ADF8DE
:10E4000000005348019069465248FAF7D9FD42F29C
:10E410002730ADF800005048019069464D48FAF7A2
:10E42000CFFD40F2E730ADF800004D48019069465D
:10E430004848FAF7C5FD41F28730ADF8000046487C
:10E44000019069464348FAF7BBFD40F6C310ADF8AA
:10E4500000003F48019069463E48FAF7B1FD40F69A
:10E46000C310ADF800003D48019069463948FAF7FD
:10E47000A7FD42F20F70ADF80000374801906946E1
:10E480003448FAF79DFD41F28730ADF8000032487C
:10E49000019069462F48FAF793FD41F28730ADF8B5
:10E4A00000002B48019069462A48FAF789FD40F69A
:10E4B000C310ADF800002848019069462548FAF7D6
:10E4C0007FFD41F64B50ADF80000244801906946AD
:10E4D0002048FAF775FD41F28730ADF800001E487C
:10E4E000019069461B48FAF76BFD40F69F70ADF846
:10E4F00000001748019069461648FAF761FD40F29E
:10E50000E730ADF800001648019069461148FAF767
:10E5100057FD41F64B50ADF800000F480190694699
:10E520000C48FAF74DFD40F6C310ADF800000B485B
:10E53000019069460748FAF743FD41F28730ADF88C
:10E5400000000548019069460248FAF739FD0EBD02
:10E550009D120108C43700207512010889120108B4
:10E56000D112010810B5002414E004EB440101EBC2
:10E57000C4010F4A02EB0110B021F9F73FFEFF2062
:10E5800004EB440101EBC401094A02EB01110870DC
:10E59000601CC4B2022CE8D303F08CF805490120BA
:10E5A00009F01AFA0449022009F016FA10BD000019
:10E5B0002C150020B3A600089BA6000810B5482122
:10E5C0000E48F9F71BFE28210D48F9F717FE0D48F4
:10E5D00002F0C2F8044624B1142221460848F9F793
:10E5E000F4FD0848203002F0B7F804462CB114229C
:10E5F000214603481430F9F7E8FD10BD5C110020F6
:10E6000034110020F0C0010810B5204800F0FCF9DA
:10E610001F4800F0F9F91F4800F0F6F91E4800F015
:10E62000F3F91E4800F0F0F91D4800F0EDF91D481F
:10E6300000F0EAF91C4800F0E7F91C4800F0E4F9A2
:10E640001B4800F0E1F91B4800F0DEF91A4800F021
:10E65000DBF91A4800F0D8F9194800F0D5F9194843
:10E6600000F0D2F9184800F0CFF9184800F0CCF9C2
:10E67000174800F0C9F9174800F0C6F9164800F02D
:10E68000C3F9164800F0C0F910BD00009C0A002034
:10E69000B00A0020C40A00202C0C0020D80A002058
:10E6A000EC0A0020000B0020140B0020280B002097
:10E6B0003C0B0020500B0020640B0020780B002046
:10E6C0008C0B0020A00B0020B40B0020C80B0020F6
:10E6D000DC0B0020F00B0020040C0020180C0020A4
:10E6E00010B528480078052848D2DFE800F0030C70
:10E6F000391B2A002448C07B08B1032000E0012018
:10E70000204908703BE021480078072804D02049C0
:10E7100008698047022801D1022000E00120194940
:10E7200008702CE019480078072804D018490869B7
:10E730008047022801D1032000E00420114908701D
:10E740001DE012480078072804D011490869804765
:10E75000022801D1022000E004200A4908700EE0DE
:10E76000002009494860487301F0F8FE06498860B6
:10E770000020044908700749087000E000BF00BF8E
:10E7800010BD000074090020600900203026002020
:10E790006C0000205C0900202DE9F04180460D4608
:10E7A000164600244046FEF7C7FE04460CB105B1EC
:10E7B00016B90020BDE8F081287818B194F854000B
:10E7C000012801D00020F5E795F8200000F00100B5
:10E7D00018B1A86A08B90020ECE795F8251084F86C
:10E7E000451094F8450010B9322184F8451094F88A
:10E7F000451001EB4101C80007F050F8C4F88C0047
:10E80000D4F88C0048B194F84530182204F1700017
:10E81000D4F88C100CF0A2FF01E00020CAE795F8B4
:10E82000200000F00100D8B994F84510080107F065
:10E8300035F8C4F88800D4F8880048B194F8453019
:10E84000102204F15800D4F888100CF087FF07E07C
:10E85000D4F88C0006F0F4FF0020C4F88C00A9E77F
:10E86000296A216404F1200720213846F9F7C6FC03
:10E870001F2229463846F9F7A8FCE86AF862A86A18
:10E88000B86295F8240087F82400286B386308489C
:10E8900030610848F0600848B06008487060084877
:10E8A000306008487061022084F85400012081E73C
:10E8B00075930108A1910108219201083B9201087A
:10E8C000C5920108BD90010838B5054601213C20DC
:10E8D00001F0CEFC0121084601F0CAFC01211348D9
:10E8E000FEF796FAAC681CB911A006F085FF38BD9A
:10E8F0002088ADF8000010208DF8030002208DF86C
:10E90000020069466068FEF7F7F9207A012804D111
:10E9100021886068FEF7CDFA05E0207A18B92188D1
:10E920006068FDF76AFB00BFE1E70000000230000D
:10E930004F5053206973204E554C4C0D0A00000077
:10E9400010B5034800F0CEF8024800F0F6F810BD0C
:10E95000A00B0020B40B002010B5034800F0C2F853
:10E96000024800F0EAF810BDB40B0020A00B002014
:10E9700010B5034800F0B6F8024800F0B3F810BD37
:10E98000A00B0020B40B002010B5054800F0AAF839
:10E99000044800F0A7F804A006F02EFF10BD000008
:10E9A000A00B0020B40B0020414320C8ABB5CD0024
:10E9B00010B5054800F0C1F8044800F0BEF804A006
:10E9C00006F01AFF10BD0000A00B0020B40B0020C1
:10E9D000414320C8ABB8DF0038B5054601211020FF
:10E9E00001F046FCAC6804B938BD2088ADF80000E1
:10E9F00004208DF8030003208DF80200694660684A
:10EA0000FEF77AF900BFEFE770B505462C6820687D
:10EA100000B970BD20462168884700BFF9E70000B3
:10EA200038B5054601213C2001F022FCAC681CB938
:10EA300010A006F0E1FE38BD2088ADF800001020DF
:10EA40008DF8030002208DF8020069466068FEF729
:10EA500053F9207A012804D121886068FEF729FA49
:10EA600005E0207A18B921886068FDF7C6FA00BF72
:10EA7000E1E700004F5053206973204E554C4C0D78
:10EA80000A00000038B505460121042001F0F0FB22
:10EA9000AC6804B938BD2088ADF8000010208DF8AE
:10EAA000030003208DF8020069466068FEF724F930
:10EAB000207A012804D121886068FEF7FAF905E080
:10EAC000207A18B921886068FDF797FA00BFE1E75E
:10EAD00010B5044621886068FDF78FFA0020207287
:10EAE000012010BD70B5044620684568686808B903
:10EAF000002070BD22689068696888470120F8E7A7
:10EB000010B5044621886068FEF7CAF910BD70B5DB
:10EB1000044620684568A86808B9032070BD2268CB
:10EB20009068A9688847F9E710B5044621886068AD
:10EB3000FEF7BFF90120207210BD70B504462068B1
:10EB40004568286808B9002070BD22689068296867
:10EB500088470120F8E738B505460121102001F06B
:10EB600087FBAC6804B938BD2088ADF800004820A8
:10EB70008DF8030003208DF8020069466068FEF7F7
:10EB8000BBF800BFEFE7000070B50A48C4880A4A26
:10EB90000221204606F0ECFC084907480068F9F716
:10EBA000B6FB05464FF07A51F9F759FB0449486026
:10EBB00070BD000060000020B40000200000304163
:10EBC000A00D002070B50446002000BF14F8016BB2
:10EBD0008E4204D1012A00D108E0551EEAB203B9E1
:10EBE00004E0451CA8B25D1EABB2EFE700BF70BDEC
:10EBF00010B517480078072804D0164908698047DF
:10EC0000022801D1642001E04FF47A7012490860B3
:10EC100008460168114804F079F9012816D1104816
:10EC200001780068401C0E4A106001F0010020B11C
:10EC300000BF0C48FFF756FF04E000BF0948FFF78C
:10EC40007CFF00BF0021054804F060F910BD000002
:10EC5000302600206C00002008000020000000206A
:10EC600004000020280B00201048807A08B90020FA
:10EC700070470E480B300E490978405C30B10B48A4
:10EC80000B300B490978405C0A4908800848007835
:10EC9000401C074908700548807A0978884202DCE0
:10ECA00000200349087003480078E1E7680C002061
:10ECB000AB060020AC06002003A006F09DFD06F088
:10ECC000C5FC00F04DFE0000476F20746F20536CB0
:10ECD0006565700D0A00000000BFFEE7704710B5C3
:10ECE0004FF4A06000F046F810BD000000F01F02D5
:10ECF00001219140024A430942F823107047000065
:10ED000080E100E070B5002100230F22C47804B335
:10ED1000154C246804F4E064C4F5E064210AC1F1F0
:10ED20000403CA40447804FA03F184781440214370
:10ED300009010E4C0678A155047804F01F05012442
:10ED4000AC4005786D11AD0005F1E025C5F8004136
:10ED500009E0047804F01F050124AC40044D067856
:10ED6000761145F8264070BD0CED00E000E400E0AF
:10ED700080E100E002490143024A1160704700004F
:10ED80000000FA050CED00E0024A0A400243024B83
:10ED90001A60704780FFFF1F08ED00E0064800681A
:10EDA00000F4E06005490843001D03490860BFF313
:10EDB0004F8F00BFFEE700000CED00E00000FA05F9
:10EDC0000648006800F4E06005490843001D034957
:10EDD0000860BFF34F8F00BFFEE700000CED00E0BE
:10EDE0000000FA0510B54FF400720021014805F04B
:10EDF00059FC10BD5C49002010B50848FFF79DFE86
:10EE00000120FDF7C0F80648FFF797FE4FF4FA70AF
:10EE1000FDF7B9F80248FFF765FE10BDA00B002012
:10EE2000B40B002010B5FFF797FD6420FDF7ABF899
:10EE3000FFF79EFD00200349487103A006F0DCFCAB
:10EE400010BD0000EC2500204F50454E5F4143525D
:10EE500065616C790D0A000010B5012004498871C4
:10EE600004A006F0C9FC0748FFF767FE10BD0000CC
:10EE7000EC2500204F50454E5F44435265616C794C
:10EE80000D0A00009C0A002010B50B48008848B904
:10EE900001200949088000200849887308A006F06D
:10EEA000ABFC08E000200449088001200349887376
:10EEB00007A006F0A1FC10BD52050020D4250020BB
:10EEC000B4F2BFAAC0CFBBAFC4A3CABD0D0A000035
:10EED000B9D8B1D5C0CFBBAFC4A3CABD0D0A00001D
:10EEE00001460A780AB9012070470020FCE70000BB
:10EEF000014908627047000000000E42034909689A
:10EF000041EA8001014A1160704700000070004032
:10EF100010B5044604F10B0318460CF097FC186872
:10EF2000C0F3093081B20F4881871868C0F30930F7
:10EF30000A2190FBF1F00B4981F86C005868800CB5
:10EF400081B20848C1875868800C0649A1F846007C
:10EF500018791968890D60F38D210248A0F84810CE
:10EF6000012010BDF007002070B5054605F10B0427
:10EF700020460CF06BFC6268C2F3C262D0B20A4A4F
:10EF8000126F116B88472268C2F30262D0B2064A40
:10EF9000126F916B88472068C0F34070C1B202487D
:10EFA00080F85910012070BDF007002010B504460C
:10EFB00004F10B0318460CF049FC988880B20A2132
:10EFC00090FBF1F081B20F48A0F866105868000C71
:10EFD0000A2190FBF1F081B20A48A0F86810586845
:10EFE000000C0A2190FBF1F080B240F480510548FA
:10EFF000A0F84A101868000C024981F84F0001205F
:10F0000010BD0000F007002010B5044604F10B030A
:10F0100018460CF01BFC9888000A0A30C1B20F4851
:10F0200080F86A105868000E0A30C1B20B4880F8A8
:10F030006B109888010A094880F850105868010E32
:10F04000064880F852105868010C044880F85110A6
:10F05000197980F85310012010BD0000F00700203E
:10F0600070B50546FAF7CCF805F10B0420460CF014
:10F07000EDFB6068C0F3892000EB80004FF6FF7164
:10F0800001EA40000549A1F841006068000D81B225
:10F090000248A0F84310012070BD0000F0070020D6
:10F0A00070B50546FAF7ACF805F10B0420460CF0F4
:10F0B000CDFB2088C0F305202168C1F30441C1EBDA
:10F0C000011100EB810081B20248A0F84D1001202F
:10F0D00070BD0000F007002010B5044604F10B03DA
:10F0E00018460CF0B3FB04491868086302485968D5
:10F0F0004163012010BD00004825002010B50446E2
:10F1000004F10B0318460CF0A1FB0449186888634E
:10F1100002485968C163012010BD00004825002045
:10F1200010B5044604F10B0318460CF08FFB04499C
:10F1300018680864024859684164012010BD000045
:10F140004825002070B5054605F10B0420460CF05B
:10F150007DFB2068C0F34040C1B21A4880F84510DA
:10F160006068000C0A2190FBF1F01649A1F8330009
:10F17000A088C0F38D000880217812484171208852
:10F18000010A104880F83B10A088C0F38D0081B2BE
:10F190000C48A0F839102268C2F30042D0B2094AE4
:10F1A000126F916988472068C0F30040C1B20548DA
:10F1B00080F85A102068800C81B202480181012039
:10F1C00070BD0000F007002010B5044604F10B03E9
:10F1D00018460CF03BFB9888C0F38D0081B20648BE
:10F1E000C1805868000DC0F57A6081B20248A0F86D
:10F1F0003510012010BD0000F007002010B50446B6
:10F2000004F10B0318460CF021FB1868C0F3893099
:10F2100081B20548A0F83710044918688866034889
:10F220005968C166012010BDF00700204825002064
:10F230002DE9F041274805880126274827494860DD
:10F24000002008702B46324620212348FFF7BAFCE5
:10F25000044622494C70AC4202D10120BDE8F08145
:10F26000701CC6B231E01C48005D202802D1601C31
:10F2700084B22AE027461848011918480278083055
:10F2800040F822102B46324620211348FFF79AFC03
:10F290000446E01BC1B21148027818308154183876
:10F2A0000378083050F82320083801780CA006F0C5
:10F2B000A3FA0A480078401C0849087008460078FC
:10F2C000042800DB03E0701CC6B2AC42CBD100BF07
:10F2D0000120C3E71E020020661E002060210020DE
:10F2E000256420706172616D3A25730A0000000088
:10F2F0007CB5002000900190009001904FF4457083
:10F300007E490860486000200872487208208872B0
:10F310006C4601F0F1FC054601F004FD0646D4E917
:10F32000000165F31961C4E90001D4E9000165F346
:10F330009B61C4E90001D4E9000166F31D71C4E9D1
:10F340000001D4E9000166F39F71C4E900016C4833
:10F35000007A08B9012000E00020D4E9001260F32F
:10F360001142C4E900126648C07908B9012000E0E2
:10F370000020D4E9001260F39342C4E9001260480F
:10F38000407A08B9012000E00020D4E9001260F3BF
:10F390004922C4E90012FCF70DFC0246D4E9000141
:10F3A00062F38B20C4E90001FCF734F80246D4E98B
:10F3B000001062F31550C4E90010524908698047F3
:10F3C000022814D15049898989B20A2291FBF2F1AD
:10F3D00088B2C82801DA002101E0A0F1C80188B292
:10F3E000D4E9002160F35D52C4E9002106E0002267
:10F3F000D4E9000162F35D50C4E90001434800789C
:10F4000005280FD14248006FB0F902000A2190FB95
:10F41000F1F000F5FA70D4E9002160F31432C4E988
:10F42000002107E04FF4FA72D4E9001062F31431BE
:10F43000C4E90010FCF78CF90246D4E9000162F33C
:10F44000DF70C4E900012420FDF776F9D4E9001249
:10F4500060F39E71C4E900122E48807C58B12D489B
:10F46000007B40B12648817AD4E9002061F34F3017
:10F47000C4E9002006E00022D4E9000162F34F3124
:10F48000C4E900011E484178D4E9002061F3D75057
:10F49000C4E900201A488078D4E9001260F30822F9
:10F4A000C4E900121C480078401C1B49087008463B
:10F4B0000078042802DB0020087001E0164800787C
:10F4C000D4E9001260F30921C4E90012072168465B
:10F4D00008F0AAFD0246D4E9001062F30701C4E96E
:10F4E000001020460CF0B9F904480B300099016077
:10F4F000019941600B3808F0ADFB7CBDC0250020B0
:10F50000EC2500206C000020A00D002030260020FB
:10F51000F007002060090020AE0600207CB5002026
:10F5200000900190009001904FF47A704E4908606D
:10F530004860002008724872082088726C462820B3
:10F54000FDF7FAF858B92620FDF7F6F838B91C206F
:10F55000FDF7F2F818B92120FDF7EEF808B1012007
:10F5600000E00020D4E9001260F38E32C4E90012FA
:10F570003E48007804280DDB3C480078062809DC6A
:10F580003A48C07C30B10122D4E9001062F3CF3098
:10F59000C4E90010FBF73EFF022803D0FBF73AFF57
:10F5A000032806D10022D4E9000162F3CF31C4E977
:10F5B00000012F49486880472830D4E9001260F3E1
:10F5C0001F62C4E900122B4800782830D4E90012E9
:10F5D00060F31742C4E90012254908682649F8F784
:10F5E00096FE0646F9F7BFF8054642F210718D42C5
:10F5F00001D90A4600E02A46D4E9000162F30D0170
:10F60000C4E900011D48807C98B11C48007B80B192
:10F610001B48827AD4E9001062F30B21C4E9001080
:10F62000FFF722FBD4E9002160F30702C4E90021BF
:10F630000CE00022D4E9001062F30B21C4E90010B1
:10F64000D4E9001062F30701C4E9001020460CF071
:10F6500004F905480B3000990160019941600B38AD
:10F6600008F0F8FA7CBD0000C025002030260020FC
:10F670006C000020EC25002000007A446009002086
:10F68000680C002010B5044604F10B0318460CF07A
:10F69000DDF85868C0F317000249096F486001207F
:10F6A00010BD0000F007002010B5044604F10B0364
:10F6B00018460CF0CBF85868800EC1B21348006FA2
:10F6C00001725868C0F30550C1B21048006F417212
:10F6D0005868C0F3C430C1B20C48006F817298887A
:10F6E000C0F38420C1B20948006FC1729888C0F38A
:10F6F0008310C1B20548006F01731879C0F305008B
:10F70000C1B20248006F4173012010BDF007002014
:10F710001CB50020009001900090019040F23F4005
:10F7200017490860486000200872487208208872F3
:10F730006C463F22D4E9000162F31F61C4E9000175
:10F7400010480078072804D00F490869804702282C
:10F7500001D1012000E00220D4E9001260F3070289
:10F76000C4E9001220460CF078F805480B300099E7
:10F770000160019941600B3808F06CFA1CBD000073
:10F78000C0250020302600206C0000201FB501207D
:10F79000134908720020A1F840000098A0F23470CC
:10F7A00010B1AB2818D10BE040F234700C49A1F82D
:10F7B0004E009DF804100DF10500FEF75FFA0CE015
:10F7C00040F2DF700649A1F84E009DF804100DF1DB
:10F7D0000500FEF71DFA00E000BF00BF1FBD0000DE
:10F7E000FC48002010B5044604F10B0318460CF049
:10F7F0002DF806491868086104485968416158683D
:10F80000000C0349096F0880012010BD4825002025
:10F81000F007002070B5054605F10B0420460CF0FA
:10F8200015F82268C2F30362D0B2064A126F916AD9
:10F8300088476268920FD0B2024A126F116A8847F5
:10F84000012070BDF00700207CB50025002000904D
:10F8500001900090019040F276503D490860486068
:10F86000002008724872082088726C463948007877
:10F87000D4E9001260F31F62C4E900120122D4E946
:10F88000000162F30A21C4E900013248006858B15E
:10F8900030480068052807D800BFD4E9000162F3AA
:10F8A0001541C4E9000119E02A48006805280ED96D
:10F8B000F9F7D0FB0546002D01DD022000E0012014
:10F8C000D4E9001260F31542C4E9001206E00022F8
:10F8D000D4E9000162F31541C4E900011E48425D0C
:10F8E000D4E9000162F30701C4E90001681C1A4968
:10F8F000095CD4E9000261F31F60C4E90002A81C9E
:10F9000015490A5CD4E9000162F31740C4E900011B
:10F91000E81C11490A5CD4E9000162F30F20C4E934
:10F920000001281D0C490A5CD4E9001062F30701AC
:10F93000C4E9001020460BF090FF05480B300099F9
:10F940000160019941600B3808F084F97CBD00002A
:10F95000C025002058090020002700207047000023
:10F960004FF0E020006920F002004FF0E021086134
:10F970000220FFF7BBF90320FFF7B8F90420FFF7D7
:10F98000B5F90520FFF7B2F90620FFF7AFF9072018
:10F99000FFF7ACF90820FFF7A9F90920FFF7A6F94E
:10F9A0000A20FFF7A3F90B20FFF7A0F90C20FFF7BF
:10F9B0009DF90D20FFF79AF90E20FFF797F90F2018
:10F9C000FFF794F91020FFF791F91120FFF78EF956
:10F9D0001320FFF78BF91420FFF788F91520FFF7A4
:10F9E00085F91620FFF782F91720FFF77FF9182015
:10F9F000FFF77CF91920FFF779F91A20FFF776F95C
:10FA00001B20FFF773F91C20FFF770F91D20FFF78B
:10FA10006DF91E20FFF76AF91F20FFF767F9202014
:10FA2000FFF764F92120FFF761F92220FFF75EF963
:10FA30002320FFF75BF92420FFF758F92520FFF773
:10FA400055F92620FFF752F92720FFF74FF9FEF767
:10FA500067FC2820FFF74AF92920FFF747F92A20F9
:10FA6000FFF744F93220FFF741F93320FFF73EF961
:10FA70003420FFF73BF93520FFF738F93620FFF740
:10FA800035F93720FFF732F93820FFF72FF9392001
:10FA9000FFF72CF93A20FFF729F93B20FFF726F969
:10FAA0003C20FFF723F93D20FFF720F93E20FFF728
:10FAB0001DF93F20FFF71AF94020FFF717F9412001
:10FAC000FFF714F94220FFF711F94320FFF70EF971
:10FAD00000BF002005E04FF0FF32134941F820201D
:10FAE000401C0828F7DB00BF0120FFF707FAFEF7EC
:10FAF00017FC00BF0D48FEF7F5FF4FF4FA70FCF756
:10FB000042FA0B48FFF719F80A48C07B18B10A48B7
:10FB1000FFF713F802E00848FEF7E4FF41F28830EF
:10FB2000FCF731FAFFF74CF980E100E02C0C0020E3
:10FB3000180C002060090020040C002070B56F48EC
:10FB40000068401C6D490860084600680521B0FB4C
:10FB5000F1F201FB1200052873D2DFE800F003394F
:10FB60005188A30066A005F047FE7048007A08B1EE
:10FB70006FA005E0714908698047714951F820007C
:10FB8000044621466FA005F037FE754A106F126FCC
:10FB9000D16A8847734951F82040214672A005F088
:10FBA0002BFE6F4890F86C2075480078754B53F821
:10FBB000201075A005F020FE694890F8450008B1B6
:10FBC00079A000E07CA001467FA005F015FE93E03F
:10FBD0006348B0F84320B0F8411081A005F00CFE56
:10FBE0008A48B0F81D20B0F81B1089A005F004FE6B
:10FBF0005B48006FB0F9021090A005F0FDFD7BE0BE
:10FC00004E498868804704464C4948688047054605
:10FC1000224629468FA005F0EFFD00BF9548FEF76C
:10FC200076FF08B194A000E096A004469748FEF73E
:10FC30006EFF08B193A000E08FA00546224629463A
:10FC400000E058E092A005F0D7FD3848007A08B1EE
:10FC500097A000E097A002463448C07908B196A06A
:10FC600000E096A0014696A005F0C6FD44E09C4940
:10FC70004868F8F7A5FD044622460B4699A005F012
:10FC8000BBFD9748B0F90C109BA005F0B5FD2B49C2
:10FC90000868F8F795FD044622460B469CA005F03F
:10FCA000ABFD29E02E4A106F126FD16B88479E4939
:10FCB00051F8204021469DA005F09EFD1B4880780C
:10FCC00008B1A0A000E0A1A002461848407808B101
:10FCD0009CA000E09DA001469EA005F08DFDF9F7D7
:10FCE000BBF828B9A14802684168A1A005F084FDCD
:10FCF00000F054F900E000BF00BF70BDD80800203C
:10FD00000D0AA1AAA1AAA1AAA1AAA1AAA1AAA1AACF
:10FD1000A1AAA1AAA1AAA1AAA1AAA1AAA1AAA1AA8B
:10FD2000A1AAA1AAA1AAA1AA0D0A0000EC2500205F
:10FD300041435F4368617267696E67006C00002031
:10FD4000640800200D0A4443555F576F726B696E5B
:10FD5000674D6F6465203C25733E0D0A000000006E
:10FD6000F0070020A80800205643555F576F726BBC
:10FD7000696E674D6F6465203C25733E0D0A000077
:10FD800030260020700800204368617267696E6742
:10FD90005F5374616765203C25733E09534F4320D0
:10FDA0003C25643E0D0A0000436F6E7374616E74EF
:10FDB000566F6C7461676500436F6E7374616E7427
:10FDC00043757272656E74004368617267696E672D
:10FDD0005F4D6F646520203C25733E0D0A000000D6
:10FDE00044656D616E645F766F6C74616765203C1D
:10FDF00025643E0944656D616E645F63757272656A
:10FE00006E74203C25643E0D0A000000380E002070
:10FE10004F75747075745F766F6C74616765203CA4
:10FE200025643E094F75747075745F6375727265F1
:10FE30006E74203C25643E0D0A0000004368617228
:10FE400067696E6743757272656E74203C25643E07
:10FE50000D0A000054656D7031202020203C25647F
:10FE60003E092047554E5F54454D50203C25643E89
:10FE70000D0A00003C0B0020446973636F6E6E65D1
:10FE8000637400004F70656E00000000500B00208E
:10FE900044435F52656C6179203C25733E202041CC
:10FEA000435F52656C6179203C25733E0D0A00006A
:10FEB00043430000434332004343310043500000BA
:10FEC00043502D4343312020203C25733E092043DD
:10FED000432D4343322020203C25733E0D0A000071
:10FEE000A00D00204B4C33305F566F6C74203C25C6
:10FEF000663E0D0A0000000053616D706C5F766F06
:10FF00006C74616765202020203C25643E0D0A004A
:10FF100043435F522069732020202020202020208E
:10FF2000203C25663E0D0A00900800204F42435FAA
:10FF300047756E436F6E6E6563742020203C257399
:10FF40003E0D0A004E4F5F4C6F636B004C6F636B4E
:10FF5000000000004856494C203C25733E2048567E
:10FF6000494C5F32203C25733E0D0A006009002099
:10FF7000456E7465722046616C7365536C6565707F
:10FF80002049646C6520636F756E74202564204D74
:10FF900041582069732025640D0A000070B50024C3
:10FFA0001DE01048005D002817DD3726002511E010
:10FFB0000D4810F835000B49095D884208D1094801
:10FFC000025D094800EBC500416808A005F014FC7B
:10FFD000681CC5B2B542EBDB00BF601CC4B20A2C82
:10FFE000DFDB70BD0027002048C401084572726F36
:10FFF0007220436F646520496E466F206973202527
:020000040801F1
:10000000732D25640D0A000010B500242F480078D8
:1000100030B101280BD0022820D0032850D14DE068
:10002000F8F71AFF80F00100284908704CE00BF047
:10003000DFFB04461CB90120244908700DE0012CA7
:1000400003D100202149087007E0022C05D10120CE
:100050001F49487302201D49087035E01D4800689B
:10006000401C1C4908601A48807B012809D00846BA
:100070000068052805D30020086003201349087094
:1000800005E014480068012801D1F9F7D9FDFEF711
:1000900027FB0F48007B50B904F056FB38B90E48D7
:1000A0000078022809DD0C480078062805DA0020CF
:1000B0000749486048730549087005E0FEF7FCFDF4
:1000C00006A005F099FB00BF00BF10BD5C09002031
:1000D0006009002078090020302600204552522077
:1000E000536C6565700D0A0030B53D4C647A04EBC5
:1000F00084046300B3F5AF7F00DA30BD1A46394C93
:100100002178394C04EBC1046488944226DA08460D
:100110000DE0354C34F83040944206DA324C04EBB2
:10012000C0046488944200DD03E0441CE0B205286A
:10013000EFDB00BF052800DB042000242B4D2C70D2
:100140002B4C247844B90124294D2C70264C04EB07
:10015000C104E488274D2C8001462DE0224C34F860
:100160003140944223DD08460DE01F4C34F8304006
:10017000944206DA1C4C04EBC0046488944200DD0F
:1001800003E0441EE0B20028EFDC00BF0024184D5D
:100190002C70164C247844B90124144D2C70124C48
:1001A00004EBC104E488134D2C80014604E00024D4
:1001B0000E4D2C700E4D2C700E4C24882CB10D4C15
:1001C0002488641E0B4D2C8007E0064C24788C425A
:1001D00003D0322A01DD034C217000BF8DE70000FF
:1001E000CC380020F00C002058C60108FA0C002082
:1001F000F90C0020FC0C002001460020034A506846
:1002000020F4404008435060704700000010024056
:1002100029B1064A52690243044B5A6104E0034A79
:1002200052698243014B5A6170470000001002403E
:1002300029B1064AD2690243044BDA6104E0034A59
:10024000D2698243014BDA6170470000001002401E
:1002500029B1064A12690243044B1A6104E0034AB9
:1002600012698243014B1A6170470000001002407E
:1002700029B1064A92690243044B9A6104E0034A99
:1002800092698243014B9A6170470000001002405E
:100290000149086070470000400442422DE9F041E6
:1002A00000210022002500230026002400278C4680
:1002B000DFF86081D8F8048008F00C0121B104292E
:1002C00007D0082959D109E0DFF84C81C0F8008037
:1002D00058E0DFF84481C0F8008053E0DFF8348153
:1002E000D8F8048008F47012DFF82881D8F8048068
:1002F00008F48035920C0D2A01D0921C00E00622F1
:1003000035B9DFF8188102FB08F8C0F8008033E047
:10031000DFF80081D8F82C8008F48036DFF8F4800C
:10032000D8F82C8008F00F0808F1010446B9DFF86E
:10033000E880B8FBF4F808FB02F8C0F800801BE086
:10034000DFF8D080D8F82C80C8F3031808F1010733
:10035000DFF8C080D8F82C80C8F3032808F1020C1D
:10036000DFF8B480B8FBF7F808FB0CF8B8FBF4F83A
:1003700008FB02F8C0F8008004E0DFF89C80C0F8B9
:10038000008000BF00BFDFF88C80D8F8048008F040
:10039000F0010909DFF8888018F80130D0F80080F2
:1003A00028FA03F8C0F80480DFF86880D8F80480E1
:1003B00008F4E061090ADFF8688018F80130D0F825
:1003C000048028FA03F8C0F80880DFF84880D8F8DD
:1003D000048008F46051C90ADFF8448018F801303D
:1003E000D0F8048028FA03F8C0F80C80DFF82480E5
:1003F000D8F8048008F44041890BDFF8288018F809
:100400000130D0F80C80B8FBF3F8C0F81080BDE8DC
:10041000F08100000010024000127A0000093D0047
:10042000F10500200106002010B50146002200233E
:1004300000204A11012A02D1094C236806E0022A51
:1004400002D1074C236A01E0054C636A01F01F02E8
:10045000012494401C400CB1012000E0002010BD9C
:1004600000100240014908607047000080044242C9
:1004700001490860704700003C0442420249096A91
:100480000143014A116270470010024010B50D4847
:10049000008F00F4804058B90A4890F8380000F006
:1004A000200028B9074890F8380000F0400030B12B
:1004B0002F20FCF75BF900200249886310BD012062
:1004C000FCE70000380E002070B505460E460024FB
:1004D00000BF03E0285D03F0E3FE641CB442F9DBD7
:1004E00070BD70B505460E46002400BF03E0285DD0
:1004F00003F0D6FE641CB442F9DB0D2003F0D0FEFD
:100500000A2003F0CDFE002403E0285D02F04AFE3D
:10051000641CB442F9DB70BD70B505460E4600247C
:1005200000BF03E0285D02F03DFE641CB442F9DB2D
:1005300070BD00000348008840F0100001490880A9
:100540007047000004280040034800884FF6EF7110
:1005500008400149088070470428004000210348F2
:100560000188001F008841EA004070471C280040B5
:1005700010B501214FF0C050FFF75AFE4FF4007044
:10058000FFF77CFF0120FFF773FF0120FEF7B0FCAF
:10059000F8F77AFD0120FFF765FF00BF6120FFF744
:1005A00043FF0028FAD04FF40070FFF767FF0120E7
:1005B000FFF75EFF00F024F800F018F849F63F401E
:1005C00000F004F800F012F810BD000000B502467B
:1005D000FFF7B0FFC2F3034003490880091D0A80FA
:1005E000FFF7B2FF00BD00000828004000BF03482D
:1005F000008800F020000028F9D07047042800404F
:10060000074800884FF6F77108400549088000BF89
:100610000348008800F008000028F9D07047000067
:100620000428004010B5012013490860FDF7F0FCD4
:100630009020FDF727FD0020FDF724FDFDF708FDC4
:10064000FDF7E6FC9120FDF71DFDFDF7A1FC0B4930
:100650000880FDF79DFC09494880FDF7F9FC074833
:1006600040880649098840EA012000B20349088011
:100670000846008880B210BD98812142C400002045
:1006800010B505A005F0B8F812210648FFF744FFA1
:1006900005A005F0B1F810BD4F726465725F436F3D
:1006A00064652000CC2600200D0A000010B5274804
:1006B0000078052845D2DFE800F003123F21300022
:1006C00023480078072804D0224908698047022877
:1006D00001D1032000E001201C49087032E01C48D1
:1006E0000078072804D01B4908698047022801D1F7
:1006F000022000E001201549087023E0144800782A
:10070000072804D0134908698047022801D1032033
:1007100000E004200D49087014E00D480078072817
:1007200004D00C4908698047022801D1022000E06A
:1007300004200649087005E00020044908700120E3
:1007400010BD00BF00BF0020FAE70000A606002091
:10075000302600206C00002070B505461DB1686889
:1007600008B1A86808B9002070BD00240EE004EBB1
:10077000440000EBC4001B4901EB0010007829780D
:10078000884201D10020EFE7601CC4B2022CEED3F6
:10079000002422E004EB440000EBC400114901EB0B
:1007A00000100078FF2816D104EB440101EBC401CE
:1007B0000C4A02EB011020222946F7F706FD012022
:1007C00004EB440101EBC401064A02EB011181F87C
:1007D00054000548C8E7601CC4B2022CDAD30020DC
:1007E000C2E700002C150020440100200020014930
:1007F000088070471E02002070B504460D46494827
:100800000078062871D2DFE800F0031F23437180CF
:1008100045480078072804D04449086980470228E1
:1008200001D1012000E002203E490870002040492B
:100830000870404901EBC50000F029FA3D4901EB81
:10084000C40000F024FA6AE003203649087066E02C
:1008500035480078072804D03449086980470228C1
:1008600003D100202F49087011E0324901EBC40088
:100870000A2100F0F9F910B9FEF74AFF07E02D4907
:1008800001EBC40000F003FA05202649087046E099
:10089000284901EBC5004FF4967100F0E5F940B12D
:1008A000244901EBC50000F0F2F905201D4908704C
:1008B0001AE01D480078022807DD1B48007806284A
:1008C00003DA0420174908700EE01748007807285B
:1008D00008D0164908698047022803D00020114932
:1008E000087001E0FEF714FF19E017E00E480078E9
:1008F000022803DD0C480078062803DB00200949A4
:10090000087001E0FEF704FF09E0FFF7CFFE08B131
:10091000002000E005200349087000E000BF00BF90
:1009200070BD0000A8060020302600206C000020CA
:10093000A60600200C37002070B504460D46494835
:100940000078062871D2DFE800F0031F234371808E
:1009500045480078072804D04449086980470228A0
:1009600001D1012000E002203E49087000204049EA
:100970000870404901EBC50000F089F93D4901EBE1
:10098000C40000F084F96AE003203649087066E08C
:1009900035480078072804D0344908698047022880
:1009A00003D100202F49087011E0324901EBC40047
:1009B0000A2100F059F910B9FEF7AAFE07E02D4907
:1009C00001EBC40000F063F905202649087046E0F9
:1009D000284901EBC5004FF4967100F045F940B18C
:1009E000244901EBC50000F052F905201D490870AB
:1009F0001AE01D480078022807DD1B480078062809
:100A000003DA0420174908700EE017480078072819
:100A100008D0164908698047022803D000201149F0
:100A2000087001E0FEF774FE19E017E00E48007848
:100A3000022803DD0C480078062803DB0020094962
:100A4000087001E0FEF764FE09E0FFF72FFE08B131
:100A5000002000E005200349087000E000BF00BF4F
:100A600070BD0000A7060020302600206C0000208A
:100A7000A60600200C37002030B5002300200021FE
:100A80000022354CA47A1CB90024344DAC7230BD20
:100A90000024334D2C704FE02F4C0B34304D2D780B
:100AA000645D002C43D02C4C0B342D4D2D78645DAF
:100AB0002C4D2C802C462488102C01D1012036E0AE
:100AC000284C2488012C0FD0264C2488022C0BD0D3
:100AD000244C2488052C07D0224C2488082C03D0D1
:100AE000204C2488092C01D1022120E01D4C2488AF
:100AF000032C1BD01B4C2488042C17D0194C2488A1
:100B0000062C13D0174C24880A2C0FD0154C24889F
:100B10000B2C0BD0134C24880C2C07D0114C2488A0
:100B20000E2C03D00F4C2488112C00D103220C4C26
:100B30002478641C0A4D2C70074CA47A084D2D783B
:100B4000AC42A9DC00B1034601B10B4602B1134629
:100B5000024CA37200BF9AE7680C0020EC2500202D
:100B60004D0900204E090020704772B6704762B6EA
:100B70007047000070B505460C46122C00D070BDC1
:100B8000224629460448F7F720FB0120024981F854
:100B9000220000BFF3E70000CC260020F0B502469B
:100BA0000B4600210020132B00D0F0BD002110E0E7
:100BB000545C202C0BD0565C0446C51700EB157511
:100BC0002D11A0EB0517074DEE55441CE0B24C1C4F
:100BD000E1B29942ECDB0124024D123D85F823403D
:100BE00000BFE2E7DE26002070B5FCF7BFFE064638
:100BF000FCF7EEFD04460025012C01D1012506E09D
:100C0000022C01D0032C01D1022500E0002512485E
:100C10000078854205D00020104908600E48057014
:100C200019E00F480078854203D100200B49086085
:100C300011E00A480068401C08490860084600683E
:100C4000022808D304480078054908700548047054
:100C500000200249086070BDAC000020C0000020E8
:100C6000AD000020AE00002070B504460D46FFF731
:100C700075FC0646206818B9266020682844606024
:100C80006068B04201D8012070BD0020FCE7014639
:100C900000200860486001207047000010B5022461
:100CA0001348B0F8410018B11148B0F84300A0B99A
:100CB0003C211048FFF7D8FFC0B10E48FFF7E7FF0F
:100CC0000B48B0F8410018B90920FBF74FFD02E0CE
:100CD0000A20FBF74BFD012408E00548B0F841006D
:100CE00020B10348B0F8430000B10024204610BDF5
:100CF000F00700206437002010B503240848C078AE
:100D0000012801D1012403E00548C07800B900247E
:100D10000420FBF711FD00B10224204610BD0000A5
:100D2000EC25002010B5032408480079012801D1E2
:100D3000002403E00548007900B901240320FBF7F3
:100D4000FBFC00B10224204610BD0000EC25002071
:100D50002DE9F04104460D460027002660782178F1
:100D600000EB012086B24948008AB04216D14848BB
:100D7000007AA84210D1474890F8220050B1FAF703
:100D800094FC28B12A46A11C4348F7F71EFA76E0E6
:100D9000222774E0332772E0132770E03B48408A33
:100DA000B04217D13A48407AA84211D1394890F858
:100DB000220058B1FAF779FC30B12A46A11C364816
:100DC0001330F7F702FA5AE0222758E0332756E0AB
:100DD000132754E02D48C08BB04217D12C48C07B5C
:100DE000A84211D12B4890F8220058B1FAF75DFCC7
:100DF00030B12A46A11C28487730F7F7E6F93EE0E3
:100E000022273CE033273AE0132738E01F48008CC4
:100E1000B04217D11E48007CA84211D11D4890F85D
:100E2000220058B1FAF741FC30B12A46A11C1A48F9
:100E30007B30F7F7CAF922E0222720E033271EE0B3
:100E400013271CE01148408CB04217D11048407C59
:100E5000A84211D10F4890F8220058B1FAF725FCAA
:100E600030B12A46A11C0C487F30F7F7AEF906E0F6
:100E7000222704E0332702E0132700E0312717B9C7
:100E80003046FBF707F93846BDE8F081BAC60108DD
:100E9000A6C60108FC480020453800202DE9F04F87
:100EA0008DB0044692469B464FF00008C14600258F
:100EB000002600279B48B0F84200042803DA1320DC
:100EC0000DB0BDE8F08F94F80090A078617840EA0A
:100ED000012571223046711C8EB20DF80020227857
:100EE0003046711C8EB20DF8002062783046711CBD
:100EF0008EB20DF80020A2783046711C8EB20DF82B
:100F00000020B9F1010F6BD1A078617840EA01258A
:100F10008449B1F842000421FAF7C1FB18B140F24C
:100F20000320854220D07F49B1F842000421FAF71E
:100F3000B6FB10B1B5F5017F16D07A49B1F8420081
:100F40000521FAF7ACFB18B140F2052085420BD021
:100F50007449B1F842000521FAF7A1FB00285CD0E2
:100F600040F20720854258D16E4890F822000028B0
:100F700050D0FAF79AFB002843D0A5F2032070B3B3
:100F8000012804D002280CD0042838D118E000270A
:100F90000220654948773046711C8EB20DF800700A
:100FA0002EE0E078012804DC0027E0785E498877AD
:100FB00000E001273046711C8EB20DF800701FE072
:100FC000E078012804DC0027E0785749887000E0C9
:100FD00001273046711C8EB20DF8007010E000E061
:100FE0002BE001204F49C8734FF4FA70A1F8540068
:100FF00000273046711C8EB20DF8007000E000BF73
:1010000001E04FF02208B8F1000F7FD101204749DD
:1010100008707BE04FF0330878E040F2032085420F
:1010200005D0B5F5017F02D0001D854202D14FF0F9
:1010300013086BE04FF0310868E0B9F1030F30D1CD
:10104000A078617840EA01253649B1F842000421D0
:10105000FAF725FBE0B1B5F5017F19D1314890F8D9
:10106000220090B1FAF721FB60B1B5F5017F07D1FD
:101070002D48477F3046711C8EB20DF8007000E09D
:1010800000BF43E04FF0220840E04FF033083DE05E
:10109000B5F5017F02D14FF0130837E04FF031086A
:1010A00034E0B9F1020F28D11E49B1F84200042101
:1010B000FAF7F5FAC0B1B5F5017F15D1194890F8E6
:1010C000220070B1B5F5017F09D100270020164933
:1010D00048773046711C8EB20DF8007000E000BFFA
:1010E00014E04FF0330811E0B5F5017F02D14FF065
:1010F00013080BE04FF0310808E00A480079012896
:1011000004D10020074908714FF01208ABF80060C5
:10111000B8F1000F04D1324669465046F7F755F84A
:101120004046CDE6FC480020680C0020A60C0020BC
:101130004BF65C20034908804AF65520091D0880BB
:1011400070470000B06C004010B500F001F810BD11
:101150000CB50020019000904048006840F48030B9
:101160003E49086000BF3D48006800F40030009030
:101170000198401C0190009820B94FF6FF7101982A
:101180008842F0D13548006800F4003010B10120E9
:10119000009001E000200090009801285CD13048C8
:1011A000006840F010002E4908600846006820F0F2
:1011B000030008600846006840F002000860274805
:1011C00040682649486008464068486008464068CC
:1011D00040F4806048600846C06A224908401F49C0
:1011E000C8620846C06A204908431C49C8620846CC
:1011F000006840F08060086000BF1848006800F098
:1012000000600028F9D01548406820F47C1013498C
:1012100048600846406840F4E810486008460068A6
:1012200040F08070086000BF0C48006800F000705B
:101230000028F9D00948406820F0030007494860B9
:101240000846406840F00200486000BF034840681C
:1012500000F00C000828F9D10CBD0000001002407D
:101260000020024000F0FEFF1408010010B5FFF757
:101270005FFF10BD10B50348407B012801D0FEF789
:1012800037F810BD6009002010B50348407B0128E5
:1012900001D0FEF743F910BD6009002010B50948E0
:1012A000007B38B900200849087014211320FFF78B
:1012B00043FB06E000200549087016211520FFF7C2
:1012C0009BFA10BD60090020A8060020A706002098
:1012D00010B50348407B012801D0FEF7B5FA10BDD8
:1012E0006009002001460248017501207047000096
:1012F000B007002001460248017401207047000039
:10130000B00700200146032903D0042901D00020A2
:1013100070470248C1740120FAE70000B0070020BE
:101320000146012902D009B10020704701488174AB
:101330000120FAE7B0070020002201490A54704753
:1013400050260020014602484174012070470000E9
:10135000B007002010B5FDF76BFF08B9002010BDE5
:10136000FBF79EFC0020134908801DE0114A1288FB
:1013700002EB4202104B03EB820251680F4A5068A5
:10138000F6F747FF58B10B48008800EB40000A49C8
:1013900001EB8000846804B1A0470120DFE7054825
:1013A0000088401C03490880024800881528DDD3C6
:1013B0000020D4E72802002048C101086021002055
:1013C0001FB500BF2748FDF7A2FB08B1012000E0D0
:1013D0000020039000BF2448FDF799FB08B10120CD
:1013E00000E00020029000BF2048FDF790FB08B10C
:1013F000012000E00020019000BF1D48FDF787FBA1
:1014000008B1012000E00020009003A91948FBF773
:10141000F3FA08B1012000E000201749C87002A9C2
:1014200014480C38FBF7E8FA08B1012000E000206E
:101430001149087101A90F480C30FBF7DDFA08B11A
:10144000012000E000200C49487069460948183026
:10145000FBF7D2FA08B1012000E0002006498870AD
:101460001FBD00003C0B0020500B0020DC0B0020B7
:10147000F00B002090260020EC25002070B50246DD
:1014800000204FF44F431E120546401C565505469A
:10149000401C53550E780546401C5655DB1C1E1249
:1014A0000546401C56550546401C53554E7805468A
:1014B000401C56558E780546401C5655CE7804463D
:1014C000451CE8B216559B1C1E120446451CE8B28A
:1014D00016550446451CE8B213550E790446451CC2
:1014E000E8B216554E790446451CE8B216558E7979
:1014F0000446451CE8B21655CE790446451CE8B2B0
:1015000016550E7A0446451CE8B216554E7A044626
:10151000451CE8B216554FF43E531E120446451CB6
:10152000E8B216550446451CE8B213558E7A0446B7
:10153000451CE8B21655CE7A0446451CE8B216554D
:101540005B1C1E120446451CE8B216550446451C99
:10155000E8B213550E7B0446451CE8B216554E7B87
:101560000446451CE8B216555B1C1E120446451C79
:10157000E8B216550446451CE8B213558E7B044666
:10158000451CE8B216555B1C1E120446451CE8B209
:1015900016550446451CE8B21355CE7B0446451C3F
:1015A000E8B216555B1C1E120446451CE8B21655DF
:1015B0000446451CE8B213550E7C0446451CE8B2AF
:1015C00016555B1C1E120446451CE8B2165504460F
:1015D000451CE8B213554E7C0446451CE8B216552E
:1015E0008E7C0446451CE8B216555B1C1E12044650
:1015F000451CE8B216550446451CE8B21355CE7C8E
:101600000446451CE8B2165570BD000010B50446EE
:1016100014220249A01CF6F7D8FD10BDD5380020D1
:101620002DE9F04104460023002000250027177013
:1016300000BF17E003EBC30707EB470727447F789A
:1016400077B103EBC30707EB470727447F7847EAE7
:10165000032C92F8008008F10107177021F818C0D8
:101660005F1CFBB2122BE5DB177807B300251AE0ED
:10167000002011E011F810C0471C11F81770BC458C
:1016800008DD471C31F8176031F810C021F817C089
:1016900021F81060471CF8B217787F1B7F1E874225
:1016A000E8DC6F1CFDB217787F1EAF42E0DCBDE8BE
:1016B000F081000010B50948006820B9084806F01C
:1016C00003FA064908600548006806F090FA20B958
:1016D0000A210248006806F07DFA10BD580100207A
:1016E000E9BA010810B5F7F705FD20B90FA004F01D
:1016F00083F8002010BDFAF78FFA08B90020F9E747
:10170000FAF79AF908B90020F4E7134890F838007E
:1017100000F0100038B1F9F7C5FA20B90FA004F0B5
:101720006BF80020E6E70120E4E70000424D53207B
:10173000546865204368617267696E67205068610C
:1017400073652053746F70732041626E6F726D61A8
:101750006C6C790A0D000000380E002043435320C2
:101760004E6F204368617267696E6720416C6C6FD1
:101770007765646E0D0000000F480068401C0E493C
:1017800008600E480068401C0C4908600A48006860
:101790004FF47A71B0FBF1F201FB1200012804D181
:1017A00007480068401C064908600648007810B9E0
:1017B0000120044908707047F4010020EC0100206A
:1017C000F8010020F001002030B5164800684FF401
:1017D0007A72B0FBF2F1B1F1807F01D301201DE0FC
:1017E00021F07F40401E4FF0E022506150170F2241
:1017F000002807DA13071D0E0B4B00F00F04241FFF
:101800001D5503E013071C0E084B1C5400BF00209D
:101810004FF0E022906107201061002008B100BF66
:10182000FEE730BD0C00002018ED00E000E400E011
:1018300010B5FCF775FD4FF417720249024805F028
:10184000F5FD10BD1017002000F0010810B5164876
:10185000006840F0010014490860084640681349D8
:1018600008401149486008460068114908400E497F
:1018700008600846006820F4802008600846406838
:1018800020F4FE0048600846006820F0A050086080
:101890004FF47F0088600020C862FFF755FC4FF0CE
:1018A00000600449086010BD001002400000FFF015
:1018B000FFFFF6FE08ED00E02DE9F05F1048B0F8FC
:1018C00000A0104A0021504603F052FE0D48006867
:1018D000F6F776FF804642460B460B480B49F6F773
:1018E0009FFE064600220A4BF6F722FE0446F6F754
:1018F000ABFF8346FBF7A0F806490881BDE8F09FDF
:1019000060000020B00000209A999999999913409D
:101910000000F03FA00D002010B50121054800F0A7
:101920004AF828B101F012FB0121024800F034F816
:1019300010BD0000000400407FB505460C460121A3
:101940000220FEF775FCADF80850ADF80440002009
:10195000ADF80A00ADF8060001A90E4800F048F8FD
:10196000012211460B4800F037F81D208DF80000C9
:1019700001208DF8010003208DF8020001208DF870
:1019800003006846FDF7BEF90121024800F007F8A0
:101990007FBD000000040040CA430282704721B1AD
:1019A000028842F00102028004E002884FF6FE73D2
:1019B0001A400280704730B5024600200023002400
:1019C000158A05EA0103958905EA010413B10CB1F2
:1019D000012000E0002030BD1AB183890B438381D0
:1019E00002E083898B4383817047818570470000C3
:1019F000002202881D4B98420ED01D4B98420BD0FE
:101A0000B0F1804F08D01B4B984205D01A4B98423A
:101A100002D01A4B984204D14FF68F731A404B886C
:101A20001A43174B984207D0164B984204D04FF6F2
:101A3000FF431A40CB881A4302808B8883850B882A
:101A400003850A4B98420BD0094B984208D00E4BA5
:101A5000984205D00D4B984202D00D4B984201D1CF
:101A60000B7A03860123838270470000002C01401B
:101A7000003401400004004000080040000C004019
:101A800000100040001400400040014000440140AC
:101A90000048014010B51248008888B9002011495B
:101AA00008701149087011490870114908701149EE
:101AB00008700846017810480088FCF7D3F80DE05C
:101AC0000720094908700D480078401C0B49087030
:101AD00008460078102801D10020087010BD0000D1
:101AE000C40C0020E00C0020CE0C0020B70C00201D
:101AF000DC0C0020D50C0020BC0C0020BA0C00200F
:101B000010B50120214908700020214908702148A2
:101B10000078012805D120480078102801D1FAF773
:101B20006EFA1C480078012803D11B480078102861
:101B300005D01A48007858B11948007840B9962065
:101B400018490880012018490870022017490870B8
:101B500016480078012802D11548007848B10E488F
:101B6000007830B10B480078042804D1114800886F
:101B700008B900F0FDFC10480078012805D105489F
:101B80000078062801D100F0F3FC10BDD80C00202D
:101B9000DD0C0020CE0C0020B20C0020AA0C00208E
:101BA000A90C0020CA0C0020DF0C0020A80C00208B
:101BB000AB0C0020B00C0020B70C002070B53648EC
:101BC0000078012866D035480079012804D13448CE
:101BD0000078012800D170BDFCF776F83149088003
:101BE0003148FCF72DF83048007800F0F0002F491C
:101BF000087000202E4908802E4800882749A1F847
:101C00004200002008712848007800F00F052248A3
:101C10000078022803D115B901201F490870204817
:101C20000078012801D100F0A3FC2048007820BBF7
:101C30001D48007800F00F001E49088001240CE0C8
:101C40001948005D1C491A4A1288885418480088AF
:101C5000401C17490880601CC4B2164800888442A2
:101C6000EEDD00F03DFA48B9092014490870084635
:101C7000017810480088FBF7F5FF0BE001201049C0
:101C8000087000200D49087008460178094800884E
:101C9000FBF7E8FF00BF9EE7A80C0020FC480020EF
:101CA000B70C0020C20C0020E20C0020BE0C00206B
:101CB000C00C0020BC0C0020EA3C0020D50C002009
:101CC000D70C002010B51F480078012824D001202F
:101CD0001D490870FBF7F8FF1C4908801C48FBF7FA
:101CE000AFFF1B48007800F00F0416480078022868
:101CF00003D114B90120134908701648007801284F
:101D000001D100F035FC002013490870012013496F
:101D100008701349087114E00F480078401CC0B2E5
:101D20000D49087002280CDB02F080F900F064F81D
:101D3000002009490870034908700A4908700A49D7
:101D4000087010BDA80C0020D90C0020C20C002087
:101D5000E20C0020B70C0020EB0C0020EA0C002065
:101D6000FC480020CE0C0020600D002010B511486A
:101D7000007838B1104840781049087000F0EAFB4C
:101D80000F4908700D4800780E4908700C4800781B
:101D90000D49087000200D49087000F029FC0B481F
:101DA000007818B904200A49087002E003200849A5
:101DB000087010BDE10C0020E20C0020AA0C0020ED
:101DC000AB0C0020A90C0020AC0C0020AE0C0020B5
:101DD000CE0C002000487047EA3C002010B50548B2
:101DE0000078012804D100200249087000F050F961
:101DF00010BD0000D90C002000200D4908700D49CD
:101E000008700D4908700D4908700D4908700D499A
:101E100008700D4908700D4908700D4908700D498A
:101E200008700D4908700D4908700D490870704719
:101E3000CE0C0020A80C0020B70C0020DB0C0020EA
:101E4000DC0C0020D80C0020D90C0020DD0C002078
:101E5000DE0C0020DF0C0020E00C0020D40C002061
:101E6000DA0C002010B507480078FBF759FF064848
:101E7000FBF730FF4620054908800120044908701F
:101E800010BD0000B60C0020E20C0020C60C0020A3
:101E9000DD0C002010B50446114804800088072896
:101EA00003DC00200F49087002E010200D49087083
:101EB00001200D49087000200C4908800C4800786A
:101EC000012802D100F054FC09E00C2009490870F7
:101ED00008460078FBF7EEFE00200349087010BDAD
:101EE000B00C0020B20C0020A80C0020B40C002084
:101EF000DB0C0020D50C002010B500F03DFE00F0FA
:101F000037FB10BD10B50A48007820B1012805D074
:101F1000022809D105E000F091FA06E000F0AAFAE3
:101F200003E000F0DDFA00E000BF00BF10BD0000DC
:101F3000BB0C002010B52E4840782D49097801F0DF
:101F40000F0140EA01202B490880084600882A49F1
:101F500008802848008840F60201884213DD0D20E1
:101F6000264908700846017822480088FBF77AFE67
:101F700002202349087000F083FB002020490870EC
:101F80002049087032E01B48008808282EDB00F04A
:101F9000A7F848B90920194908700846017815487A
:101FA0000088FBF75FFE21E0022411E01048005D8D
:101FB0001549164A128888540F480088401E0E4959
:101FC000088012480088401C10490880601CC4B278
:101FD000072CEBDD01200E49087006480088FBF74E
:101FE00016FE01200B49087000F04AFB10BD0000EE
:101FF000E20C0020BC0C0020C40C0020D50C0020FA
:10200000D40C0020CE0C0020EA3C0020C00C0020A4
:10201000BA0C0020B70C002010B51848007800F06A
:102020000F001749088001240CE01448005D154991
:10203000154A1288885414480088401C12490880A8
:10204000601CC4B20E4800888442EEDD00F048F8FF
:1020500048B909200D4908700846017808480088E9
:10206000FBF700FE08E000200849087008460178E8
:1020700003480088FBF7F6FD10BD0000E20C0020CD
:10208000BC0C0020EA3C0020C00C0020D50C002035
:1020900010B50E48007800F0F0000D4908700020DF
:1020A0000C4908800C490870094800780B49C8762B
:1020B0000748007810B9FFF7AFFF05E00448007843
:1020C000102801D1FFF736FF10BD0000E20C002000
:1020D000BE0C0020C00C0020D70C0020FC480020C3
:1020E00000202149097831B1102912D0202918D0B7
:1020F000302935D12CE01D49098849B11C490A888D
:102100001A490988491C8A4201DA002000E00120AE
:1021100027E017490988082901DA002000E001209A
:102120001FE014490988072907DB11490988082994
:1021300001DA00200BE0012009E00D490A880D4971
:102140000988491C8A4201DA002000E0012008E0E9
:1021500007490988032901DA002000E0012000E096
:1021600000BF00BF70470000BE0C0020BC0C002068
:10217000C20C0020C40C00202C490988072933DA3E
:1021800001212B4A1180012016E02A49095C2A4AC4
:102190002A4B1B88D15429490988491C274A118098
:1021A00027490988491E264A118021490988491C66
:1021B0001F4A1180411CC8B21C4909888842E4DDCD
:1021C0001F49098819B901211E4A82F821100121ED
:1021D0001D4A117008211D4A117001211C4A1170FD
:1021E0000021164A118020E01049098807291CDBCC
:1021F000012011E00F49095C0F4A104B1B88D15494
:102200000E490988491C0D4A11800D490988491E4B
:102210000B4A1180411CC8B20728EBDD0849098828
:1022200019B90121074A82F821107047D00C00200B
:10223000D20C0020E20C0020EA3C0020C00C002060
:10224000C40C0020FC480020BB0C0020CE0C002059
:10225000DC0C002010B52D48008838B903202C492B
:1022600008700846007800F0D1F84EE02948007860
:1022700001284AD1002027490870274908702748BB
:10228000007800F0F000264908700846007818B180
:1022900008460078102809D106201D490870084614
:1022A000007800F0B3F8FFF7F3FE2EE01C4800784A
:1022B00020282AD1FFF714FF38B9092014490870E3
:1022C0000846007800F0A2F81FE01448007800F0FB
:1022D0000F0014490978884210D100201249087073
:1022E000FFF710FE96200949088001200A4908706E
:1022F0000D48007848B9FFF7CDFB06E004200449FB
:1023000008700846007800F081F810BDCC0C002061
:10231000D50C0020D90C0020E00C0020E20C00209D
:10232000BE0C0020BA0C0020BB0C002010B52D4ABA
:1023300012882D4B1B889A4220DB2B4A11780120F2
:1023400011E02A4A125C2A4B2A4C24881A55294A41
:102350001288521C274B1A80234A1288521E224B85
:102360001A80421CD0B28842EBDD1F4A1288002A34
:1023700036D10122204B83F8212031E0194A1288FE
:10238000194B1B889A422BDA01221C4B1A80012020
:1023900016E0164A125C164B164C24881A55154A3C
:1023A0001288521C134B1A800F4A1288521E0E4B71
:1023B0001A80124A1288521C104B1A80421CD0B24A
:1023C000084A12889042E4DD02220D4B1A7008225E
:1023D0000C4B1A7001220C4B1A700022054B1A800C
:1023E00010BD0000D00C0020C40C0020E20C002026
:1023F000EA3C0020C00C0020FC480020D20C002049
:10240000BB0C0020CE0C0020DC0C002010B50446D4
:10241000214606480088FBF725FC00200449087087
:10242000044908700449087010BD0000BC0C00206D
:10243000CE0C0020B70C0020DC0C002010B50A48A0
:10244000008840F60201081A0849088008480088F8
:10245000072802DBFFF790FE05E005480088072803
:1024600001DAFFF763FF10BDC00C0020D00C002084
:10247000C40C00201248007808BB16E0114812492D
:102480000988405C1149124A128888541048008813
:10249000401C0F4908800F480088401E0D490880E5
:1024A00009480088401C0849088007480088072818
:1024B000E4DD0020084908700720084908707047CB
:1024C000DC0C0020E20C0020D20C0020EA3C0020B2
:1024D000C00C0020C40C0020BB0C0020CE0C00203F
:1024E0001449097821BB1449087816E01349144AA5
:1024F0001288895C134A144B1B88D15412490988ED
:10250000491C114A11800C490988491E0A4A118048
:102510000B490988491C0A4A118009490A88411C4B
:102520008A42E3DD0021094A11700721084A11702F
:1025300070470000DC0C0020C40C0020E20C0020DE
:10254000D20C0020EA3C0020C00C0020BB0C002074
:10255000CE0C0020054A917831B17F2900DD7F2122
:10256000C8B2421CD0B200E001207047E20C00204B
:1025700010B514480078092821D2DFE800F00508DA
:102580000B0E1114171A1D00FFF728FC18E000F0BD
:102590006BFC15E000F0D6FB12E000F01BF80FE03A
:1025A00000F030FB0CE000F099FC09E000F02EFC9C
:1025B00006E0FFF74FFE03E000F098FB00E000BFED
:1025C00000BF10BDCE0C00200120014908707047EB
:1025D000DB0C002010B500F00BF80348007810B9B0
:1025E00004200249087010BDAE0C0020CE0C002063
:1025F00010B50A48007820B1012805D0022809D179
:1026000005E000F0CBF906E000F0EEF903E000F0A1
:102610002DFA00E000BF00BF10BD0000AE0C00208E
:1026200012490988C1F3032141F01001104A1170C9
:102630000E4909785170022011E00E490E4A1288A5
:10264000895C0B4A11540C490988491C0A4A1180BB
:1026500006490988491E054A1180411CC8B207284D
:10266000EBDD0821054A117070470000B00C002016
:10267000E20C0020EA3C0020B40C0020B60C002044
:1026800010B51848007840F0300017490870002055
:1026900048701420887000201449088003201449D1
:1026A0000870032404E0CC200F490855601CC4B214
:1026B000072CF8DD08200E4908700020FBF736FBD8
:1026C0000B480078FBF72CFB0748FBF703FB0620C1
:1026D0000849087046200849088001200749087009
:1026E00010BD0000D40C0020E20C0020B80C00202B
:1026F000B60C0020CE0C0020C80C0020DE0C002000
:10270000164A1278164B1A70012001210EE0154A64
:10271000154B1B88D25C124B5A54134A1288521C18
:10272000114B1A80421CD0B24A1CD1B20B4A1288FB
:102730009142ECDD094A1278521C0C4B1A700728A2
:102740000ADC04E0CC22064B1A54421CD0B2072803
:10275000F8DD0822054B1A7070470000B00C00200D
:10276000E20C0020EA3C0020B40C0020B60C002053
:1027700010B51048007810B9FFF7C2FF05E00D480A
:102780000078102801D1FFF74BFF01200A4908709B
:102790000A480078FBF7C4FA0948FBF79BFA0120C6
:1027A0000849087046200849088001200749087038
:1027B00010BD0000B20C0020AD0C0020B60C0020B3
:1027C000E20C0020CE0C0020C60C0020DD0C002006
:1027D00010B52A48008807282BDA012028490880EC
:1027E000012416E0274828490988405C27490855F4
:1027F00025480088401C2449088025480088401E40
:10280000234908801E480088401C1D490880601C20
:10281000C4B21A4800888442E4DD01201D490870D2
:1028200000201D490870FBF78FFA00201649088028
:1028300023E01248008807281FDB012411E011481B
:1028400011490988405C114908550F480088401C0F
:102850000D4908800E480088401E0D490880601C04
:10286000C4B2072CEBDD08200C490870FFF7FAFA18
:1028700004200B49087000F065F910BDD00C002051
:10288000D20C0020EA3C0020B40C0020E20C002016
:10289000B00C0020AE0C0020DB0C0020B60C002099
:1028A000CE0C002070B5334800883349098888422F
:1028B0002DDB012530480678012413E02F483049EC
:1028C0000988405C2F4908552D480088401C2C4938
:1028D000088029480088401E27490880681CC5B226
:1028E000601CC4B2B442E9DD2748067004E0CC2085
:1028F00024494855681CC5B2072DF8DD0820224937
:102900000870FFF7AFFA04202049087030E019483A
:1029100000881949098888422ADA01201C49088060
:10292000012416E0154816490988405C15490855E8
:1029300013480088401C124908800F480088401E38
:102940000D49088012480088401C11490880601C0D
:10295000C4B2084800888442E4DD02200D490870B2
:1029600000200D490870FBF7EFF9002004490880AA
:1029700070BD0000D00C0020B00C0020EA3C00200C
:10298000B40C0020E20C0020B60C0020CE0C00207D
:10299000D20C0020AE0C0020DB0C002010B50D483E
:1029A000007840F020000C4908700C48008840F680
:1029B0000201081A0A4908800A480088072802DB31
:1029C000FFF706FF05E007480088072801DAFFF750
:1029D00069FF10BDAD0C0020E20C0020B40C0020FB
:1029E000D00C0020B00C002010B51748007801284A
:1029F00028D116E0154816490988405C1549164A41
:102A00001288885412480088401C114908801348D5
:102A10000088401E114908800F480088401C0E495C
:102A200008800D4800880728E4DD08200C4908705C
:102A3000FFF718FA00200B49087004200A490870B3
:102A400000F080F810BD0000DB0C0020EA3C002004
:102A5000B40C0020E20C0020D20C0020B00C0020AE
:102A6000B60C0020AE0C0020CE0C002010B5204883
:102A7000007801283AD11F48047800781E49097867
:102A800008441E49087018E01D481E490988405C2A
:102A90001D49184A128888541A480088401C194950
:102AA000088015480088401E13490880601CC4B285
:102AB00010480088401C0F4908800E4800880F49C4
:102AC00009788842E0DB04E0CC200F490855601CFF
:102AD000C4B2072CF8DD082008490870FFF7C2F9D6
:102AE00000200A49087004200949087010BD000040
:102AF000DB0C0020D20C0020B00C0020B60C002013
:102B0000EA3C0020B40C0020E20C0020AE0C0020B7
:102B1000CE0C002010B504462046FBF7CBF8002071
:102B20000449087004490870044908700449087091
:102B300010BD0000CE0C0020A80C0020DB0C0020F3
:102B4000D80C002009480078401C08490870084645
:102B50000078102801D1002008700548007820B1C5
:102B600004480078401E034908707047AD0C0020EF
:102B7000AA0C0020A90C00201A480078012808D1CE
:102B800019480088002804DD17480088401E1649AF
:102B9000088016480078012808D1154800880028C8
:102BA00004DD13480088401E114908801148007850
:102BB000012808D110480088002804DD0E4800884C
:102BC000401E0D4908800D480078012808D10C48A6
:102BD0000088002804DD0A480088401E0849088053
:102BE00070470000DD0C0020C60C0020DE0C002029
:102BF000C80C0020DF0C0020CA0C0020E00C0020D4
:102C0000CC0C002010B52C48008838B901202B4985
:102C1000087008460078FFF77DFF4CE028480078F0
:102C2000012803D027480078012844D100202649F4
:102C30000870234908702548008838B900201F49CA
:102C4000087008460078FFF765FF34E020480078F8
:102C500048B12048007830B900201F490870022090
:102C60001E49087027E01E48007818B11C480078FB
:102C700001280CD1FFF7BCFC1A48007818B90020D5
:102C80001049087017E001200E49087013E014483D
:102C90000078022803D10320104908700BE0104887
:102CA0000078022807DD10480078401E0E490870A1
:102CB00005200A49087010BDC60C0020D50C002064
:102CC000D80C0020DA0C0020DD0C0020B00C002015
:102CD000AA0C0020A90C0020E10C0020CE0C002042
:102CE000AB0C0020AE0C0020AC0C002010B511483D
:102CF000008838B903201049087008460078FFF7AB
:102D000085FB15E00D48007801280AD100200B4909
:102D100008700B200849087008460078FFF776FB1A
:102D200006E0FFF7EFF80648007808B9FEF7B2FEB4
:102D300010BD0000CC0C0020D50C0020D90C0020C8
:102D4000BB0C002010B52B48008838B902202A4956
:102D5000087008460078FFF7DDFE49E02748007854
:102D6000012845D10020254908702548007800F049
:102D7000F0002449087008460078302838D1002037
:102D8000214908701E48007800F00F04FFF7A8F9E9
:102D900038B909201849087008460078FFF7BAFECC
:102DA00026E0032C07DB052013490870084600784D
:102DB000FFF7B0FE1CE0022C07D108200E49087076
:102DC00008460078FFF7A6FE12E0012C0DD107207F
:102DD0000949087008460078FFF79CFE95200549D0
:102DE000088001200849087002E00CB9FEF7BEFF18
:102DF00010BD0000CA0C0020D50C0020D90C00200A
:102E0000E20C0020BE0C0020DF0C002010B50F48A3
:102E1000007801280ED100200C4908700C49087078
:102E200007200C49087096200B49088001200B49A7
:102E3000087009E00A48008830B901200949087083
:102E400008460078FFF7E2FA10BD0000D80C002019
:102E5000DE0C0020CE0C0020CC0C0020E00C00206A
:102E6000C80C0020D50C002010B51548008838B9D2
:102E700001201449087008460078FFF74BFE1DE05A
:102E800011480078012819D100200F4908700F4916
:102E900008700F48007838B900200A4908700846C1
:102EA0000078FFF737FE09E009480078102805D1BF
:102EB00001200849087002200749087010BD000071
:102EC000C60C0020D50C0020D80C0020DD0C002002
:102ED000B20C0020E10C0020CE0C00200848007845
:102EE000401E0749087008460078012806DC0320C8
:102EF00004490870044800780149087070470000D0
:102F0000AC0C0020CE0C0020AB0C002002460023AD
:102F100021B90D4800681060012070470A48036815
:102F20001068984205D81068181A884209D3012001
:102F3000F3E71068C0F1FF301844884201D3012044
:102F4000EBE70020E9E70000F401002010B5322093
:102F5000F9F7F2FB90B92A20F9F7EEFB70B90848AF
:102F6000006801880748FEF740FD05490968486880
:102F700080470348006880680149086010BD000070
:102F8000C4370020000400404F48007801280AD1CF
:102F90004E48C068401C4D49C860012008700020A0
:102FA0004949087000E070474848C0680521B0FBF7
:102FB000F1F201FB120030B94448C06818B1012099
:102FC0004249487000E0EEE74048C0680A21B0FB83
:102FD000F1F201FB120028B93C48C06810B1012091
:102FE0003A4988703948C0681421B0FBF1F201FBFE
:102FF000120028B93548C06810B101203349C870A3
:103000003248C0683221B0FBF1F201FB120028B94E
:103010002E48C06810B101202C4908712B48C068A7
:103020006421B0FBF1F201FB120028B92748C06807
:1030300010B10120254948712448C0684FF4FA7145
:10304000B0FBF1F201FB120028B92048C06810B1B2
:1030500001201E4988711D48C0684FF47A71B0FB89
:10306000F1F201FB120028B91848C06810B1012024
:103070001649C8711548C06840F2DC51B0FBF1F246
:1030800001FB120028B91148C06810B101200F4996
:1030900008720E48C0684FF4FA61B0FBF1F201FB10
:1030A000120028B90948C06810B1012007494872C8
:1030B0000648C06841F27071884202D3002003497B
:1030C000C86000BF6FE70000F0010020001700207B
:1030D0000FB5184800880A2802DB0020154908802F
:1030E00014480288001D00EB0210009901609DF851
:1030F000041010480288001D00EB021001719DF8B9
:103100000D100C480288001D00EB021041730948A5
:103110000188001D00EB0110DDF8051040F8051FC7
:10312000DDF80910416003480088401C014908800F
:103130000FBD0000EC44002010B51748006800B136
:1031400010BDF8F763F900B9FAE71BE013484088AF
:103150000A2802DB00201149488010484188001DE0
:1031600000EB011494E80F0001F017FB01200C495B
:103170008870002081F82A0008484088401C0749D0
:10318000488005E005480088044949888842DDD127
:1031900000BF00BFD4E70000640C0020EC44002016
:1031A000FC48002010B504462146054801F059FAB4
:1031B00000BF0348008800F080000028F9D010BD4F
:1031C000004C004010B540F22551394801F089F912
:1031D000F8B1374801F040FAC4B236480088C82830
:1031E00008DA344801880088401C324A108032488E
:1031F000445402E000202F4908800A2C04D1FEF735
:10320000A9F8FDF7F3FA10BD40F22551284801F066
:1032100040F940F22441264801F063F948B1FDF736
:10322000E5FA234801F018FA40F22441204801F061
:1032300030F940F227711E4801F053F920B140F2F5
:1032400027711B4801F025F940F22661184801F06A
:1032500048F920B140F22661154801F01AF9082119
:10326000134801F031F9012806D10821104801F076
:1032700007F90F4801F0F0F904210D4801F024F995
:10328000012806D104210A4801F0FAF8084801F0A3
:10329000E3F90221064801F017F9012806D10221BD
:1032A000034801F0EDF8024801F0D6F900BFAAE7A3
:1032B000004C00401E020020661E002010B540F2A7
:1032C0002551334801F00DF9E8B1314801F0C4F956
:1032D000C4B230480088C82808DA2E48018800881F
:1032E000401C2C4A10802C48445402E000202949FC
:1032F00008800020294908802949087040F225519A
:10330000234801F0C6F840F22441214801F0E9F8D1
:1033100050B11F4801F0A0F901202149087040F286
:1033200024411B4801F0B5F840F22661184801F02D
:10333000D8F820B140F22661154801F0AAF808211A
:10334000134801F0C1F8012806D10821104801F006
:1033500097F80F4801F080F904210D4801F0B4F806
:10336000012806D104210A4801F08AF8084801F032
:1033700073F90221064801F0A7F8012806D10221BD
:10338000034801F07DF8024801F066F910BD000025
:1033900000500040240200202E1F002020020020A8
:1033A0002202002010B50948007F70B10748C07F95
:1033B00010280AD10549887F00F0AAFA00200349A5
:1033C0000877FF210248F4F719FF10BDFC480020E0
:1033D000EA3C002010B50748007F50B10548C07F87
:1033E000112806D103482B3000F03EFB0020014994
:1033F000087710BDFC48002010B50A48007F78B15E
:103400000848C07F14280BD1032106482B3000F058
:1034100087FB002003490877FF210348F4F7EEFEFD
:1034200010BD0000FC480020EA3C002010B5064812
:10343000007F40B10448C07F192804D100F014F97E
:1034400000200149087710BDFC48002010B506484F
:10345000007F40B10448C07F222804D100F0AAF9BF
:1034600000200149087710BDFC48002010B5154820
:10347000007F28B31348C07F272821D1114890F836
:103480002B00022809D0104A0E492B31012000F0F0
:103490008BFB00200B49087712E00A4890F82B00BC
:1034A00002280DD1084A07492B3100F07DFB00208E
:1034B0000449087781F82100034800210160416038
:1034C00010BD0000FC480020180D002010B50A486F
:1034D000007F78B10848C07F28280BD10221064818
:1034E0002B3000F079FC002003490877FF210348C6
:1034F000F4F784FE10BD0000FC480020EA3C0020E8
:1035000010B50A48007F78B10848C07F2E280BD13B
:1035100007480088401E81B2064800F07FF900206D
:10352000024981F82100087710BD0000FC48002006
:10353000C00C0020EB3C002010B50A48007F78B199
:103540000848C07F31280BD1032106482B3000F0FA
:10355000CDFC002003490877FF210348F4F74EFE15
:1035600010BD0000FC480020EA3C002010B50748D0
:10357000007F50B10548C07F3E2806D103482B305C
:1035800000F08CF900200149087710BDFC480020AC
:1035900010B50A48007F78B10848C07F85280BD154
:1035A000012106482B3000F0DBFC0020034908779E
:1035B000FF210348F4F722FE10BD0000FC48002064
:1035C000EA3C00208178064A1170C178517011469A
:1035D0000978491C117011464978891C517070474F
:1035E000180D002010B50948007801280DD10748B2
:1035F00040780C2806DA05484078054951F8204003
:10360000A04702E000200149087010BD200D0020F5
:10361000240D002010B501200249087000F006FDBD
:1036200010BD0000200D002010B5002002490870D8
:1036300000F0FCFC10BD0000200D002070470000D1
:10364000012008494877002081F8220088714874D9
:10365000A1F8400081F8240081F8250081F82700B6
:1036600070470000FC48002070B5002400250026AB
:103670004D484078012870DD19204B490870002022
:1036800048704A48B0F84200022878DB474890F872
:103690002B0000F07F060B2E67D2DFE806F06606EF
:1036A0000745256626666666460000BF3046F7F782
:1036B000E3FFB8B13D49B1F842000321F7F7EFFF4E
:1036C00070B13A4A2B3231463948F9F7D5FC0446F5
:1036D00024B137492046FAF757FB04E0312502E0D0
:1036E000132500E0122549E000BF3046F7F7C4FF7C
:1036F000C0B12E49B1F842000621F7F7D0FF78B1EA
:103700002A4A2B3231462A48F9F7B6FC0446032CE4
:1037100004DD27492046FAF737FB04E0312502E0B3
:10372000132500E0122529E000BF3046F7F7A4FF7B
:10373000C8B11E49B1F842000221F7F7B0FF80B1CD
:103740001A4A2B3231461A48F9F796FC044634B12E
:1037500017492046FAF718FB06E023E00FE0312571
:1037600002E0132500E0122508E01048B0F84200FE
:10377000022801DA132500E0122500BF00E013251E
:10378000122D01D0312D04D108480079012800D034
:1037900000251DB129461920FAF7D8FA0A20034955
:1037A000A1F8460070BD0000680D0020FC48002014
:1037B000CC4B002070B50024002515484078012826
:1037C00024DD1449B1F842000321F7F768FF98B1EE
:1037D0001148F9F7F9FC0546032D04DB0E4928468C
:1037E000FAF7D2FA09E00B480079012805D1002048
:1037F00008490871312400E013241CB1214622201D
:10380000FAF7A4FA1E200349A1F8460070BD000093
:10381000680D0020FC480020CC4B00202DE9F04131
:1038200004460D46002600271948407801282CDD63
:1038300018480079012828D11649487F0022032121
:10384000F7F7FAFEB8B1032D01DA132714E0A81E2A
:1038500081B22046FDF77CFA064656B96E200E4925
:10386000087020784870607888700320FAF78CFA26
:1038700002E0374600E07F271FB139462E20FAF7D5
:1038800065FA28200349A1F84600BDE8F081000050
:10389000680D0020FC480020CC4B002070B5044689
:1038A000002500261748407801282ADD1649B1F87E
:1038B00042000221F7F7F3FEC8B1207800F07F063E
:1038C00066B92078F7F7E4FE90B17E200F490870C2
:1038D000207848700220FAF757FA09E00A48007980
:1038E000012805D1002008490871122500E01325A0
:1038F0001DB129463E20FAF729FA0A200249A1F80B
:10390000460070BD680D0020FC480020CC4B002014
:103910002DE9F04105460227002600244F48407853
:1039200001287CDD10204D490870002048704C496A
:10393000B1F842000221F7F7B2FE00287ED005F070
:103940007F04012C03D0022C01D0032C6DD14448FC
:10395000407F03281AD1022C18D141480079012850
:103960006DD1F7F7A2FE78B13D48C07B60B13C480D
:103970004477FDF77BFC0120394908730870C820A3
:1039800081F8200078265AE0222658E03448407F0B
:10399000012801D1022C05D03148407F022807D1EF
:1039A000032C05D12E480079012848D17E2646E017
:1039B000032C03D0012C01D1FAF7B0FC012C02D169
:1039C00000202749C8732648447700202449A1F8DD
:1039D000400081F82200887148740846407F03281F
:1039E00001D1032C07D000201D4981F8240081F863
:1039F000250081F827002846F7F74AFEF8B1502045
:103A00001849087008464570002088703220C87038
:103A100001200871F42048710627384602E01BE0B7
:103A20000CE002E0FAF7B0F909E00D48007901284E
:103A300005D100200A490871122600E013261EB1A4
:103A400031461020FAF782F90A2004498880084696
:103A500080880349A1F84600BDE8F081680D002088
:103A6000FC480020CC4B002070B504460025002601
:103A70002748407801284ADD112025490870002098
:103A800048701E2088802349B1F842000221F7F7D0
:103A900006FE002831D0207800F07F063046F7F788
:103AA000E3FD08B3F7F701FEE0B12078F7F7F0FD8A
:103AB00038B1512018490870207848700220FAF770
:103AC00063F916480079012805D1002013490871CF
:103AD00011490870487001200E490870C82081F80B
:103AE00020000BE0222509E00A480079012805D1D1
:103AF000002008490871122500E013251DB1294650
:103B00001120FAF723F90A200249A1F8460070BDF6
:103B1000680D0020FC480020CC4B0020C448002049
:103B20002DE9F04104460F4600251C484078012845
:103B300032DD1420194908701E2088802078000486
:103B4000617800EB0120A17846181549B1F84200D0
:103B50000421F7F7A4FDA8B16FF07F40864208D199
:103B6000F7F7A6FD54200F4908700120FAF70CF969
:103B700009E00B480079012805D1002008490871A7
:103B8000312500E013251DB129461420FAF7DEF88F
:103B90000A200349A1F84600BDE8F081680D002025
:103BA000FC480020CC4B00202DE9F04180460C461B
:103BB00015460026FF2782484078012872DD81489B
:103BC000007901286ED17F49487F01221146F7F71D
:103BD00033FD002867D02078012842D100207A499F
:103BE00008707849B1F842000221F7F758FDA8B3F0
:103BF0007448C078012801D13726D4E06720734982
:103C00000870207848706F4890F82200012808D189
:103C10006C488079012804D108460021C0F80210C0
:103C20000DE06848407C50B96948F9F70FFA012067
:103C300064494874654866490968C0F80210012063
:103C4000614908705F49887167205D4908700020EC
:103C500048705E490620FAF797F8A4E0FFE71326BC
:103C6000A1E0207802287BD1002056494874B1F8A1
:103C700042000621F7F713FD002872D0514890F852
:103C80002800032802DC5048007868B94D4890F8B5
:103C90002800032800DB36264B4800780028ACD1EA
:103CA000242680E08AE07DE047480078012802D1A0
:103CB00000204549087045480021016081800422A8
:103CC0004349F4F7BFFA00285BD02178491EC8B2F7
:103CD000404A3F49F9F746F90746002F4FD160782F
:103CE0002870A0786870E078A8702079E8700422C5
:103CF00038492846F4F7A6FAF8B90020314981F886
:103D00002800672031490870207848702078022800
:103D100001D1012000E002202A4981F82300672018
:103D200027490870002048700120264981F82200A8
:103D300026490220FAF728F824E0224890F82800C3
:103D4000FF2806DA1F4890F82800401C1D4981F81A
:103D500028001C4890F82800022803DC352611E0D2
:103D600017E014E0174890F8280003280AD13626F7
:103D70000A20144981F829000120C87002E01226A7
:103D800000E0242612480021016081800BE0132608
:103D900009E00C48B0F84200022801DA132602E0DC
:103DA000122600E07F261EB131462720F9F7CEFF0C
:103DB0001E20034988800349A1F84600BDE8F08130
:103DC000680D0020FC480020760D0020CC4B002020
:103DD0006E0D0020720D00202DE9F041044688464A
:103DE00000270025002668203D4908703D4840789E
:103DF000012873DD28203B4908701E2088803A493D
:103E0000487F01221146F7F717FC002855D03649A4
:103E1000B1F842000321F7F742FC00284BD0F7F736
:103E200044FC002845D0207800F07F0566780DB16D
:103E3000032D35D1012E01D0032E28D16DB9012ECD
:103E400004D10020284981F8240015E000202649EB
:103E500081F8240081F825000EE0032D0CD1012EFD
:103E600004D10120204981F8240005E001201E49E9
:103E700081F8240081F825002078F7F709FC20B3A9
:103E80002078174948700220F9F77EFF1DE0164898
:103E90000079012819D1002013490871312714E055
:103EA00011480079012810D100200F49087112270C
:103EB0000BE0222709E0132707E00B4800790128CF
:103EC00003D10020084908717F271FB139462820F7
:103ED000F9F73CFF0A200449A1F84600BDE8F0814B
:103EE000CC4B0020680D0020FC480020F8B50546AA
:103EF0000E4600240020009016484078012827DD57
:103F00003120144908701E20888013480079012848
:103F10001ED11149487F01221146F7F78DFB38B1B8
:103F20006B460E4A31462846FCF7B8FF044600E0CF
:103F30007F2424B121463120F9F708FF04E0074926
:103F4000BDF80000F9F720FF0A200349A1F8460058
:103F5000F8BD0000680D0020FC480020CC4B00207C
:103F60002DE9F04104460F46002600252C484078F4
:103F7000012853DD85202A4908701E2088802949A0
:103F8000487F01221146F7F757FB002835D0254915
:103F9000B1F842000221F7F782FB60B3F7F785FB27
:103FA00008B9222631E0207800F07F05012D01D0EC
:103FB000022D17D1012D04D100201A4981F82700C4
:103FC00003E00120174981F827002078F7F760FB0C
:103FD000D8B1C52014490870207848700220F9F73C
:103FE000D3FE12E00F48007901280ED100200D49C0
:103FF0000871122609E0132607E00A480079012813
:1040000003D10020074908717F261EB13146852063
:10401000F9F79CFE0A200349A1F84600BDE8F081AB
:10402000680D0020FC480020CC4B002000200449F3
:104030000870022048700120887000208880704736
:10404000680D002010B50848007F58B10649C87FA8
:1040500000F014F8002004490877C877FF210348CE
:10406000F4F7CCF810BD0000FC480020EA3C00202A
:1040700010B50446FFF7D8FA10BD000070B505462C
:1040800000240B484078012810DD0A4800790128F7
:1040900003D100200749087111241CB1214628468C
:1040A000F9F754FE0A200349A1F8460070BD00004C
:1040B000680D0020FC4800201E20014988807047C0
:1040C000680D002070B505460C4605480078272885
:1040D00005D16078012802D12046FFF773FA70BD40
:1040E000680D00202DE9F04107460E4614464EBBF0
:1040F0003F484078012825D13D480078403021785C
:10410000884207D121463846FFF7DCFF02203849B4
:1041100048706BE020787F2868D135480078617856
:10412000884263D1A078782805D1FFF7C5FF042025
:104130002F4948705AE0A078FFF79AFF03202C49D6
:10414000487053E0002E44D129484078022840D1DD
:104150002078102805D1022025494870607825492B
:10416000887720782349C877002518E02248405DE9
:104170002049C97F884210D11E48C07F342803D00F
:104180001C48C07F362805D11C48008820B91C482F
:10419000457001E01A48457003E0681CC5B20C2D5B
:1041A000E4DB00BF0C2D02D10B201549487014210F
:1041B00010482B30F4F722F81422611C0D482B30E4
:1041C000F4F703F801200B4908770846A0F842707D
:1041D0000CE0092E0AD10B480078012806D10020F6
:1041E00008490870FF210848F4F708F8BDE8F08195
:1041F000680D0020FC4800202AC70108C40C0020DC
:10420000200D0020EA0C0020EA3C0020012001499A
:1042100048707047680D002010B540F225511D48C8
:1042200000F05FF910B31B4800F016FAC4B21A4848
:10423000008800F40040C8B91748008800F48040A6
:1042400060B10A2C03D000201349088020E01248F6
:10425000008840F400401049088019E00D2C06D178
:104260000D48008840F480400B49088010E00A485F
:104270000088C0F30D0009490C5407480088401C11
:104280000549088008460088C72801DD002008800D
:1042900010BD0000003801400E020020D81B002095
:1042A00010B504462146054800F0DBF900BF03487D
:1042B000008800F080000028F9D010BD00440040C4
:1042C00010B540F22551304800F00BF9C0B12E482E
:1042D00000F0C2F9C4B22D480088FE2808DA2B4845
:1042E00001880088401C294A10802948445402E073
:1042F00000202649088040F22551234800F0C9F8E3
:1043000040F22441204800F0ECF850B11E4800F083
:10431000A3F901201F49087040F224411A4800F017
:10432000B8F840F22661184800F0DBF820B140F2FE
:104330002661154800F0ADF80821134800F0C4F8D4
:10434000012806D10821104800F09AF80E4800F024
:1043500083F904210C4800F0B7F8012806D10421A4
:10436000094800F08DF8084800F076F90221064867
:1043700000F0AAF8012806D10221034800F080F8D5
:10438000014800F069F910BD00440040100200200F
:10439000A01C00201202002010B540F22551334825
:1043A00000F09FF8E8B1314800F056F9C4B2304847
:1043B0000088C82808DA2E4801880088401C2C4A4A
:1043C00010802C48445402E0002029490880002035
:1043D000294908802949087040F22551234800F0F6
:1043E00058F840F22441214800F07BF850B11F48B2
:1043F00000F032F901202149087040F224411B48A5
:1044000000F047F840F22661184800F06AF820B141
:1044100040F22661154800F03CF80821134800F0EE
:1044200053F8012806D10821104800F029F80F4858
:1044300000F012F904210D4800F046F8012806D1D9
:1044400004210A4800F01CF8084800F005F9022190
:10445000064800F039F8012806D10221034800F08F
:104460000FF8024800F0F8F810BD000000480040C6
:10447000180200209E1D00201402002016020020B9
:1044800001F40072B2F5007F00D100BFCA43028080
:10449000704710B50022002340F66A14A14200D1F3
:1044A00000BF0A1201249440A3B2DC43048010BD73
:1044B00021B1828942F40052828104E082894DF662
:1044C000FF731A408281704702460020B1F5007FD9
:1044D00000D100BF13880B400BB1012000E0002089
:1044E000704770B50246002400230025002040F6E6
:1044F0006A16B14200D100BFC1F3421501F01F039B
:10450000012606FA03F3012D02D19689334006E015
:10451000022D02D1168A334001E0968A33400C12F4
:10452000012606FA04F41688344013B10CB10120B8
:1045300000E0002070BDF0B50346002400260025F1
:10454000002040F66A17B94200D100BF1846C1F3F7
:10455000421401F01F06012707FA06F5012C01D1CC
:104560000C3004E0022C01D1103000E014301AB1FC
:1045700007682F43076002E00768AF430760F0BD9C
:104580002DE9F04786B005460E460024A24600BF3E
:10459000A1460027B08900B100BF2F462C8A4CF6F7
:1045A000FF700440F08804432C82AC894EF6F3106F
:1045B0000440B08831890843718908430443AC81C1
:1045C000AC8A4FF6FF400440B0890443AC8201A896
:1045D000FBF764FE1F48874202D1DDF810A001E01E
:1045E000DDF80CA0A88900F4004040B10AEBCA0035
:1045F00000EB0A1031684900B0FBF1F807E00AEB64
:10460000CA0000EB0A1031688900B0FBF1F86420A1
:10461000B8FBF0F004012009642101FB1089A8898E
:1046200000F4004040B1322000EBC900B0FBF1F0D3
:1046300000F00700044308E0322000EB0910642179
:10464000B0FBF1F000F00F0004432C8106B0BDE890
:10465000F08700000038014001468888C0F3080058
:104660007047C1F308028280704710B500F072F9FC
:10467000FBF73AFD10BD10B500F048FB10BD00007F
:1046800006480088064908600448001F0088098819
:1046900040EA01400249086070470000BC6C0040DD
:1046A000EC0C002070B504460D46164632462946ED
:1046B000204603F004FD70BD70B504460D46164655
:1046C00032462946204603F03DFD70BD1149096878
:1046D00051B94FF0E02189690E4A1160114609680D
:1046E0000D4A51430B4A11604FF0E0218969094A94
:1046F000126888180749096843F285621144054A1F
:10470000116080B21146098801EB810140EA014045
:1047100070470000F40C00200DE37A05704700009C
:1047200000200349097801F0010101B1012070471F
:10473000680C0020002003490978C1F3400101B151
:1047400001207047680C0020002003490978C1F35C
:10475000001101B901207047680C002001460020BB
:1047600040F2B472914200D1012070470FB41FB5DE
:10477000069800909DF822008DF804009DF8042012
:104780000DF123010DF10500F3F71FFD9DE80F006A
:1047900000F026FB1FBC5DF814FB0FB585B00020B0
:1047A0008DF80800059800909DF818008DF80A0013
:1047B00000208DF809009DF80A200DF119010DF176
:1047C0000B00F3F702FD684603F044FA09B000BDA0
:1047D00010B50648007840B9012004490870FAF77E
:1047E00001FBF7F741FAF7F771FB10BDF80C002059
:1047F00010B53C48C2793C4801683C48F3F7E5FCF9
:10480000384802783AA139486B38F3F7DEFC35486E
:1048100042783BA135485D38F3F7D7FC31488278C0
:104820003AA132485138F3F7D0FC2E4802793AA128
:104830002E482B38F3F7C9FC2A48C27839A12B48F7
:104840004538F3F7C2FC2748427933A1274821387D
:10485000F3F7BBFC2348827939A124481738F3F7D2
:10486000B4FC2048827A38A120485F30F3F7ADFCD1
:104870001C48017A1D480A30F3F7C0FC00201B4990
:104880006B3981F8E800002118486B3880F8E9108E
:104890008C2016496B3981F8EC00A02113486B3845
:1048A00080F8ED10142011496B3981F8F000502187
:1048B0000E486B3880F8F11013200C496B3981F8E1
:1048C000F400882109486B3880F8F5101920074951
:1048D0006B3981F8F800192104486B3880F8F91019
:1048E00010BD0000A6C60108EC0C00203B380020DB
:1048F000323130393134302D535A3032000000001B
:104900003839323620202020202000004443552012
:10491000202020202020000048573A432E312E30FE
:104920000000000053573A312E30302E435F3234AE
:10493000303831325F383932365F303000000000B5
:10494000413430553630000052325830303030313A
:104950000000000010B5B648007820F00100401CAF
:10496000B3490870B3494868B349F3F7D0FC04462B
:10497000F3F7F9FEAE494872B048007C087200BFF8
:10498000AF48808F0112AA48C17400BFAC4890F8AC
:104990003C00C1B2A6480175A6488089010AA44816
:1049A0004175A448017BA2488175A548006F406805
:1049B000010C9F488172A248006F8088010A9C48C0
:1049C000C1729F48006F0179994801739C48006F3C
:1049D000417B974841739A48006F017B94488173EB
:1049E0009748006FC17A9248C1739548006F817AE9
:1049F0008F4801749248006F417A8D484174904805
:104A0000006F017A8A4881748E480078072803D1A4
:104A100001218748C1750BE08B490869804702284E
:104A200003D102218248C17502E000218048C1758E
:104A30008648C078012803D100217D4841760DE0E9
:104A40008248C07818B901217948417606E00420EF
:104A5000F7F772FE10B10221754841767B48007964
:104A6000012803D10121724801760DE077480079D1
:104A700018B900216E48017606E00320F7F75CFEC6
:104A800010B102216A4801766F4908687049F3F74E
:104A90003EFC0446F3F767FE010A654881766A49E1
:104AA00008686B49F3F733FC0446F3F75CFEC1B2C8
:104AB0005F48C1766148807B08B9012100E0002190
:104AC0005B4801770120F7F737FEC043C0435849E0
:104AD000097860F3041156480170007820F0200036
:104AE000534908703320F7F727FEC043C0435049AD
:104AF000097860F386114E4801703420F7F71CFEE8
:104B0000C043C0434A49097860F3C711484801705F
:104B10003020F7F711FEC043C0434549497860F3A0
:104B20000001434841703120F7F706FEC043C043FF
:104B30003F49497860F341013D4841700320F7F750
:104B4000FBFDC043C0433A49497860F382013848CD
:104B500041700320F7F7F0FDC043C0433449497862
:104B600060F3C301324841700420F7F7E5FDC0430C
:104B7000C0432F49497860F304112D484170042047
:104B8000F7F7DAFDC043C0432949497860F345117E
:104B9000274841702D48407810B92C48807808B1DA
:104BA000012000E000202249497860F38611204866
:104BB00041703520F7F7C0FDC043C0431C49497818
:104BC00060F3C7111A4841703620F7F7B5FD184950
:104BD00088701848808988801C48007888711A4934
:104BE000486880471249C8711A480078022806DAD6
:104BF0000846007820F00200801C087005E00C4890
:104C0000007820F002000A49087012480078022853
:104C100007DD0748007820F00400001D04490870F3
:104C200005E00348007820F004000149087010BD39
:104C3000CC380020A00D0020000020416009002099
:104C4000F0070020302600206C000020EC2500201A
:104C500000401C46F00C00200E4890F8EC000E4975
:104C6000C8700C4890F8ED0008710A4890F8F100FF
:104C7000084991F8F01000EB01200749C880054869
:104C800090F8F500034991F8F41000EB0120024977
:104C900008817047D0370020680C002030B585B0FF
:104CA0001648006816490968884225D013481449F7
:104CB000096801600025002410E004EBC40000EB4B
:104CC00040011048405C092806D1601CC2B2284649
:104CD000691CCDB20DF80020601CC4B2122CECDBB4
:104CE0000948857212210B30F3F788FA2A46694683
:104CF00005480B30F3F769FA05B030BD9C0C002075
:104D00008C0C0020F8380020680C002010B52D48CD
:104D1000007830B9FFF76CFDFEF792FC01202949BD
:104D2000087029480078F0B1274890F8200038B181
:104D3000254890F82000401E234981F8200011E00A
:104D400000202149087000BF2048006800F4E0609E
:104D50001F490843001D1D490860BFF34F8F00BF66
:104D600000BFFEE710BD1B480088401C80B21949F7
:104D7000088002280DDB00200880FEF74BFC012094
:104D80001149C8710020C87600F06CF80020124963
:104D9000088012480088401C80B210490880012811
:104DA00005DB00200880FEF71DFCF8F77FFFFEF70B
:104DB000C3F9F8F731FEF6F7B9FBFEF73FFC00BF89
:104DC000D0E70000160D0020FC4800200CED00E0AC
:104DD0000000FA05100D0020140D0020120D002017
:104DE0001FB540F2DF710098884204D040F2347160
:104DF000009888422FD11A480088322802DB002010
:104E00001749088016480288001D00EB021000991F
:104E100001609DF8041012480288001D00EB02108A
:104E200001719DF80D100E480288001D00EB021064
:104E300041730B480188001D00EB0110DDF80510DF
:104E400040F8051FDDF80910416005480088401C46
:104E50000349088003E0009988B200F031F81FBDD3
:104E60009045002010B51DE012484088322802DB32
:104E70000020104948800F4880780F4908700D487D
:104E80004188001D00EB011494E80F00FAF77EFC46
:104E900008484088401C0749488008480068401C72
:104EA0000649086003480088024949888842DBD1E6
:104EB00010BD000090450020010D00200C0D0020C9
:104EC0001249097801F0010101B97047B0F5827FFC
:104ED00003D0A0F21111A1B909E00D49096821F030
:104EE00001010B4A116000210A4A11800AE00849B9
:104EF000096821F00201064A11600021064A11806A
:104F000000BF00BF00BF00BFDFE70000680C00204B
:104F10008C0C0020960C0020980C00202DE9F74FF7
:104F200084B00C4617460026F9F7FAF904980028D1
:104F300056D12079D349087060794870A07900066D
:104F4000E17940EA0140217A40EA0120617A084390
:104F5000CC494860A07AE17A40EA0120C949088139
:104F6000E07B0006A17B40EA0140617B40EA012032
:104F7000217B0843C349C860207C617C40EA012052
:104F8000C0490882701E88610020C86148624FF6DF
:104F9000FF7008840020BC490870BA48008AB949EB
:104FA000C968B84A1289CDE900210290B548436822
:104FB00042780178B5A000F01FFCB248008AB149E0
:104FC000C968B04A1289CDE900210290AD48436812
:104FD00042780178BC4800F00FFCF4F75FF94EE12D
:104FE00004980128FBD1A848007810B107B0BDE8AB
:104FF000F08FE0780006A17840EA0140617840EA4D
:105000000120217808439F494861F4F707F9F9F72F
:1050100087F99C483A464169ACA000F0EDFB9948FD
:10502000806998494969884272D096484069954993
:1050300088610846C169A7F10D0008449149C8611B
:105040000846C369808BC0F30A020846C069C10ADA
:10505000A4A000F0D1FBF7F751FC8A48008C8949E5
:10506000C969B0EBD12F14D08648C069C0F3CF20F6
:10507000844908840846C069A64908444FEAD028F4
:105080004FEAC8284146A4A000F0B6FB4046F7F717
:1050900091FB04F1040AA7F10D00C11700EB917117
:1050A000C1F3870BC11700EB91718910A0EB81014F
:1050B00069B1A0A000F0A0FBA7F109010819032223
:1050C000FF21F3F794F80BF1010000F0FF0B6D489E
:1050D000406A904900EB01086A48C0696949486222
:1050E000002540E0002614E05AF825104046F7F766
:1050F000CDFB042800D10DE0701CC6B2032E08DBE6
:10510000414692A000F078FB01205F4908706DE7EE
:10511000B3E0E9E700BFD8F80090012D03DBABF165
:105120000100A84206DC5AF825204B46414690A0D3
:1051300000F062FB5AF8250048450DD094A000F01D
:105140005BFB5AF825204B46414689A000F054FBF2
:1051500001204D49087049E708F10408032E00DBDF
:1051600003E0681CC5B25D45BCDB00BFF9F7D8F8A9
:10517000A7F10D0081B28F480288201DF4F730F9A5
:105180008C4908803F4801898A4802888AA000F03B
:1051900033FBF9F7C5F83B4840693A49C96888428A
:1051A00069D13848008983490988884203D08BA097
:1051B00000F022FB1AE700263248C16891A000F0F7
:1051C0001BFB9948F7F7F6FA0FE098499648F7F76E
:1051D0005DFB042800D109E0701CC6B2032E04DB7D
:1051E000914993A000F008FB00E0EEE700BF8E4875
:1051F000D0F800904B468D4A01465DA000F0FCFAC5
:105200008A48814503D001201F490870EEE6002638
:1052100012E01C4841688448001DF7F737FB04285A
:1052200000D10AE0701CC6B2032E05DB7E49091DC1
:1052300088A000F0E1FA00E0EBE700BF7A48001D2B
:10524000D0F800900F484B467749091D42688BA063
:1052500000F0D2FA0B484068484503D001200A49C3
:105260000870C3E6F9F75CF8F3F7D8FF8CA000F0FC
:10527000C3FAF9F793FDF7F7DDFAF9F751F800BF34
:10528000B4E60000B01B00206A0500200D0A363687
:10529000365570642D2D747970653A2564202C760E
:1052A00065723A25642C54627974653A25642C2021
:1052B0004372633A25642C5061673A25642C506C24
:1052C000656E3A25640D0A0038C701080A0D43755A
:1052D0007272204261673A25642C206C656E20252D
:1052E000640A0D0057726974652D616464723A2016
:1052F000736563746F722025642C2C6F666673650A
:1053000074202564202C7265636C656E20253064E2
:105310000D0A0000006002083434437572722045A3
:10532000726173652D2D616464723A202530780DA9
:105330000A0000000A0D6C6173742D2D2D2D2D6255
:105340006167212121212121210A0D0021323221F1
:10535000212121212121212157726974652D466166
:10536000696C2D616464723A202530780D0A000062
:1053700061646472202530782C2C57726974652022
:105380002530782C2C72656164202530780D0A0058
:105390000A0D207265616476616C20213D20557094
:1053A00064646174615B695D2921212121210A0DF9
:1053B00000000000680500203132325570644865F5
:1053C00061642E46696C654372633D2530782C54C8
:1053D0004372633D2530780D0A0000005570644823
:1053E0006561642E46696C6543726320213D2054DB
:1053F000437263202121212072657475726E210D24
:105400000A0000002121217570642D696E666F21EC
:10541000212057726974652D746F7470616720253F
:1054200064200D0A000000000058020844332211D5
:1054300055706444617461466C61672120577269DC
:1054400074652D4661696C2D616464723A20253063
:10545000780D0A002121217570642D696E666F2117
:10546000212057726974652D4661696C2D616464F1
:10547000723A202530780D0A000000003161646422
:1054800072202530782C2C5772697465202530786D
:105490002C2C72656164202530780D0A0000000014
:1054A00032327570642D616C6C207772697465207E
:1054B0004F4F4B4B2121726573746172742121210E
:1054C00021212121212121210D0A000070B5C2B026
:1054D00005460C46002641F20D000849A1F80500DA
:1054E000224629460548C01DF2F76FFE0348448056
:1054F00001AA02A9F6F748FC42B070BDF61F0020D1
:1055000000BFFEE710B502240E4A106F126F516BF8
:10551000884760B905210C48FBF7A6FB78B1262027
:10552000F7F724F90848FBF7B2FB012407E0054A26
:10553000106F126F516B8847012800D1002420465C
:1055400010BD0000F0070020343700202DE9F041A5
:1055500004460E461546601BF3F7D1F880463146E7
:10556000F2F707FF0746F3F7FEF880B2BDE8F081D7
:105570002DE9FC4781460C469246314800EB041069
:105580000078C0B32E4800EB0410406848B32C48A4
:1055900000EB041040681421B0FBF1F0284901EB46
:1055A00004114860264901EB04114868F3F7B5F887
:1055B00007464FF06632234BF2F7C0FF0546002244
:1055C000214BF3F72DF8CDE90001F3F73DF91C4924
:1055D00001EB0411C8601A4800EB0410C068CAF857
:1055E00000000020164901EB04114860144901EB4A
:1055F0000411087022E0FFE7114800EB0410007A64
:10560000401C0F4901EB041108720D4800EB041017
:10561000406848440A4901EB04114860084800EB1F
:105620000410007A142809D10120054901EB041166
:1056300008700020024901EB04110872BDE8FC87E4
:10564000B00D002066660A400000B04010B5012190
:10565000C802FAF7FDFD00214FF40060FAF7F8FDEB
:1056600010BD000000200849086008480078401C70
:1056700006490870084600781E2803DC7F2002498E
:105680000839086070470000082C0040E90100203C
:1056900044E032213EE000BF00BF00BF00BF00BFBA
:1056A00000BF00BF00BF00BF00BF00BF00BF00BF02
:1056B00000BF00BF00BF00BF00BF00BF00BF00BFF2
:1056C00000BF00BF00BF00BF00BF00BF00BF00BFE2
:1056D00000BF00BF00BF00BF00BF00BF00BF00BFD2
:1056E00000BF00BF00BF00BF00BF00BF00BF00BFC2
:1056F00000BF00BF00BF00BF00BF00BF00BF00BFB2
:1057000000BF00BF00BF00BF00BF00BF00BF00BFA1
:105710004A1ED1B20029BEDC421ED0B20028B8DC3D
:105720007047000010B51E4890F82200012817D1DC
:105730001C4801780078401C1A4A107005290FDDBA
:10574000F8F7EEFD0020164981F8220012221648D3
:1057500001F06CFE00201349087014A000F04CF812
:105760000F4890F82300012818D10E4801780078DE
:10577000401C0C4A1070052910DDF8F7D1FD0020FF
:10578000074981F8230010221231114801F04EFE22
:105790000020044908700FA000F02EF810BD000092
:1057A000CC2600205009002000F001084F726465EB
:1057B000725F436F64652057726974652073756307
:1057C0006365737366756C6C79210D0A00000000C7
:1057D00000F8010850726F647563745F436F64650D
:1057E000205772697465207375636365737366759A
:1057F0006C6C79210D0A00000FB4054B10B503A99C
:10580000044A029800F044F910BC5DF814FB000053
:10581000F1810108080200200FB4084B10B504A95B
:1058200002AA039800F034F9044602A9002000F00F
:10583000B2FC204610BC5DF814FB00009761010823
:1058400030B528B1144C031F002021680A4605E03A
:10585000084630BD9A4203D810465268002AF9D152
:10586000002800D041680BD00468A3EB0005A542D6
:1058700004D11B681C440346046002E0436000E05E
:1058800023603AB11C68D51AA54203D115682C448F
:105890001C6052685A6030BD780D00202DE9F04739
:1058A00082460F4C10480D4E0E4F001B4FF0000863
:1058B00020F007054FF0010900221146504603F081
:1058C00049FA002802D1306810B10020BDE8F08705
:1058D0003C60C4E90058C6F80090EDE77C0D00205C
:1058E000544C0020780D0020506C002002E008C8C5
:1058F000121F08C1002AFAD170477047002001E04A
:1059000001C1121F002AFBD1704700002DE9FF5F83
:1059100082B00021DDE90430020DDDF840B0034320
:1059200018D044F61050A2F2FF32424315141198D9
:1059300001281FD0A5EB0B00401C5FEA000A4FF0C6
:1059400000064E4FDFF83891B046504615D5CAF1E3
:10595000000413E0119801244AA3012801D16FEA41
:105960000B010298119AC0E90031C0E9024206B069
:10597000BDE8F09FCBF10000DFE704460021404A7C
:10598000491842EB0450CDE9001012E0E00707D0BF
:1059900032463B4640464946F2F7D0FD80468946AE
:1059A00032463B4610461946F2F7C8FD06460F46FA
:1059B0006410002CEAD1DDE90401DDE90023BAF12D
:1059C000000F06DAF2F7BAFD42464B46F2F7B6FD93
:1059D00005E0F2F725FE42464B46F2F721FE04466B
:1059E0000E460022284BF2F717FF03D84FF0FF3086
:1059F000014607E00022254B20463146F2F7F7FC2E
:105A0000F3F73FF8102409E0002C0ADB0A220023F8
:105A1000F2F760FF039B30321A55641E50EA010210
:105A2000F2D1641C039AC4F111031444119A012A9F
:105A300003D0012208430DD10AE0084304D000201E
:105A40004FF0110B119072E7A3EB0B056D1E0DE0EB
:105A50005B4504DD4FF0000205F1010504E003DAC7
:105A60004FF00002A5F10105002AECD0029811992F
:105A7000C0E90231C0E9004579E7000000001440A8
:105A80000000F03F300000000000F0430000E03F65
:105A90002DE9FF4F95B09A46884606460025EEE16F
:105AA000252877D100242746F94A0121039400E0F4
:105AB000044316F8013F203B01FA03F01042F7D1EE
:105AC00030782A2811D06FF02F033078A0F13002FF
:105AD000092A16D8039A44F0020402EB820203EB6F
:105AE00042021044761C0390EFE758F8042B03920F
:105AF000002A03DA504244F40054039044F00204B4
:105B0000761C30782E2816D116F8010F44F00404C4
:105B10002A280DD06FF02F023078A0F13003092B26
:105B200009D807EB870302EB4303C718761CF3E79A
:105B300058F8047B761C30786C280FD006DC4C2893
:105B400017D068280DD06A2814D104E0742810D02A
:105B50007A280FD10DE044F400140AE044F48014D4
:105B600001E044F440147278824202D104F58014BA
:105B7000761C761C307866280BD013DC582877D03A
:105B800009DC002875D04528F6D04628F4D04728EF
:105B90001AD193E118E0632835D0642879D06528BC
:105BA00012D18BE1702873D008DC6728F1D0692806
:105BB0006FD06E280DD06F2806D1ACE073282CD0A2
:105BC000752874D0782853D05246179990476D1C89
:105BD00054E1C4F30250022809D003280DD0D8F8AC
:105BE000001004280DD00D6008F1040846E1D8F833
:105BF0000010EA17C1E90052F6E7D8F800100D804E
:105C0000F2E70D70F0E718F8041B8DF80010002083
:105C10008DF80100EB46012003E058F804BB4FF07B
:105C2000FF3061074FF0000102D40DE009F10101DE
:105C30008946B9420FDA8145F8DB1BF809100029C3
:105C4000F4D108E009F1010189468142FADB1BF831
:105C500009100029F6D103985346A0EB0907214605
:105C60003846179A00F080FA284400EB090507E04F
:105C700044E008E10DE01BF8010B524617999047EC
:105C8000B9F10109F7D2534621463846179AF2E096
:105C900039E00A21C4F302524FF0000B0091022AAE
:105CA00006D058F8040BC117032A09D00AE023E0F4
:105CB00008F1070020F00702F2E80201904605E033
:105CC00000B2C117042A01D140B2C117002906DA77
:105CD0000A460021404261EB02012D2202E022052A
:105CE00004D52B228DF80420012203E0E20701D025
:105CF0002022F7E7914657E00A2100E010214FF0FB
:105D0000000B00910BE010214FF0000B44F0040455
:105D10000827009103E008204FF0000B0090C4F327
:105D20000252022A05D058F8040B0021032A08D099
:105D300008E008F1070020F00702F2E802019046AF
:105D400003E080B2042A00D1C0B24FF0000922075C
:105D50002AD53278702A07D0DDF800C08CF0100CFC
:105D60005CEA0B0C05D00EE040228DF804200122E5
:105D700008E050EA010306D030238DF804308DF896
:105D8000052002229146009B83F0080353EA0B038F
:105D90000AD150EA010201D1620705D530228DF8FF
:105DA00004204FF001097F1E3278582A04D039A20E
:105DB0000C920CAA02920BE03BA2F9E75B46009A18
:105DC000F2F788FD0C9B9B5C029A521E02921370A4
:105DD00050EA0102F2D1029804A9081A00F1200B3E
:105DE000600702D524F4803400E001275F4502DD1E
:105DF000A7EB0B0000E0002000EB0B0100900398E4
:105E00004944401A0390E00306D453462146179AAA
:105E1000039800F0A9F90544002706E001A85246BE
:105E2000C05D179990476D1C7F1C4F45F6DBE00362
:105E30000CD553462146179A039800F095F905446E
:105E400004E030205246179990476D1C0099481E77
:105E500000900029F5DC08E002980299524600788B
:105E6000491C0291179990476D1CBBF10001ABF1E1
:105E7000010BF1DC5BE100F065F90544761C30783C
:105E800000287FF40DAE19B02846BDE8F08F000061
:105E90000928010030313233343536373839616200
:105EA00063646566000000003031323334353637C4
:105EB000383941424344454600000000600700D4A1
:105EC000062708F1070020F00700F0E802238046CB
:105ED00003F0004C5FEA0C0001D097A009E0200518
:105EE00001D596A005E0E00701D095A001E0AFF252
:105EF0004C001390307823F0004365280CD006DC6A
:105F0000452809D046281DD047287FD13BE0662888
:105F100018D067287AD136E00021112F01DB11203B
:105F200000E0781CCDE9000104A90CA8FFF7EEFC05
:105F3000DDE90D010C9A4FF0000B07F101091092F9
:105F400000914EE04FF000400097CDE9011004A908
:105F50000CA8FFF7DBFCDDE90D020C9B0F994FF05D
:105F6000000B91461093009211B9791C00EB0109C6
:105F7000B7EB090003D4C0F1FF3B07F10109A9EB1E
:105F80000700019042E0012F00DA01270021112FC4
:105F900001DD112000E03846CDE9000104A90CA87C
:105FA000FFF7B4FCDDE90D010C9A00914FF0000BF6
:105FB000B946109221070FD4009A4A4503DA914658
:105FC00001E0A9F10109B9F1010F05DD109AA9F16C
:105FD0000101515C3029F4D0B84202DA10F1040F0B
:105FE00003DA0121CDE9011010E0002803DC83442D
:105FF000A9EB000102E0411C494500DD8946A0EB08
:106000000B00401C01904FF000400290200705D487
:106010000198484502DB4FF0FF30019000208DF8D9
:106020004B0002980DF14B07B0F1004F25D0022034
:106030000C902B200D90029800280CDA4042029020
:106040002D200D9007E00A210298F2F72DFC303147
:10605000029007F8011D0C99481E0C900029F2DCF3
:1060600002980028EFD1791E0D980870307800F062
:10607000200040F0450007F8020D11A8C01BC01D0C
:1060800002901398007800B1012000EB09010198FB
:1060900001EBE071029801440398401A401E0390FE
:1060A000E00306D453462146179A039800F05CF8A3
:1060B00005441398007818B15246179990476D1C03
:1060C000E00323D553462146179A039800F04CF875
:1060D00005441BE0BBF1000F07DB0098584504DDC9
:1060E0001098179910F80B0001E0179930205246CC
:1060F000904701980BF1010B401E05F1010501903D
:1061000004D12E205246179990476D1CB9F1000119
:10611000A9F10109DEDC05E017F8010B52461799D9
:1061200090476D1C0299481E02900029F4DC5346EA
:106130002146179A03989EE62D0000002B000000D0
:10614000200000002DE9F041044600251E461746B8
:10615000880404D405E039462020B0476D1C641E35
:10616000F9D52846BDE8F0812DE9F0410446002527
:106170001E469046C80301D5302700E0202788043A
:1061800004D505E041463846B0476D1C641EF9D57C
:106190002846BDE8F0810A68531C0B6010707047F8
:1061A0000749084A1268885406490968491C0A22A6
:1061B000B1FBF2F302FB1311024A116070470000B9
:1061C000002700205809002010B5044602F0F8FD11
:1061D00018B10AA0FFF710FB10BD0E480E49096860
:1061E00044540D480068401C052190FBF1F201FB6E
:1061F00012000949086000BFEEE700004576656EB1
:10620000742071756575652069732066756C6C0AFC
:10621000000000003C0C0020380C002010B58CB0B1
:1062200001F0D4FB26E09DF80C3004AA07A80699DB
:10623000F3F73FFF00208DF82F000120264908705A
:106240000B98009007A80FC800F0FCF901280FD1A7
:10625000142207A92148F1F7B8FF1F480021CDE912
:1062600001101E48006900901C480FC800F086F914
:10627000F8F756F81A48406840B1194803AB04AA29
:1062800006A944680020A0470128CCD014E09DF85E
:106290000C3004AA07A80699F3F70BFF00208DF82D
:1062A0002F00FEF73DFA28B10B98009007A80FC801
:1062B00000F03CF9F8F734F80948C06940B10848E3
:1062C00003AB04AA06A9C4690120A0470128DED0B7
:1062D00001F054FA0CB010BDE8010020EC160020CB
:1062E0009C16002010B520211A48F1F787FF3021B5
:1062F0001948F1F783FF01F063FBF8F733F9F8F77A
:106300005DF9154A15490020F8F746FA10B114A0B6
:10631000FFF772FA104A183217490120F8F73CFAD1
:1063200010B116A0FFF768FA0B48C06830B10A48F0
:1063300000231A461946C4681846A0470648406A12
:1063400030B1054800231A461946446A0120A04787
:1063500010BD0000CC1600209C160020B0010020CB
:1063600063616E3120D0ADD2E9B3F5CABCBBAFB327
:10637000C9B9A60D0A0000007C01002063616E32DD
:1063800020D0ADD2E9B3F5CABCBBAFB3C9B9A60D35
:106390000A00000010B5A2B0002441F20B000D4924
:1063A000A1F8050000BF01E0601C84B2282CFBDBD3
:1063B0005020084948800848007C401C0649087461
:1063C00006A0FFF719FA01AA02A90248F5F7DCFCBA
:1063D00022B010BDF61F00207C21002053656E64A2
:1063E0002063656C6C2074656D70200A0D000000E0
:1063F00010B5A2B0002441F20C001049A1F805002C
:1064000000BF06E00E48015D0C48C01D0155601C30
:1064100084B2082CF6DB0820084948800948007C33
:10642000401C0849087408A0FFF7E6F901AA02A970
:106430000248F5F7A9FC22B010BD0000F61F0020AD
:10644000452400207C21002073656E6420626D73FA
:106450005F73746174655F696E666F0A0D0000009A
:1064600010B5A2B0002441F20A001149A1F80500BC
:1064700000BF09E004EB44010E48084481780C4851
:10648000C01D0155601C84B2282CF3DB282008496C
:1064900048800948007C401C0749087407A0FFF7A2
:1064A000ABF901AA02A90248F5F76EFC22B010BDB3
:1064B000F61F0020CD2300207C21002053656E6450
:1064C0002063656C6C2074656D70200A0D000000FF
:1064D00070B50546002400BF1FE0114951F8341083
:1064E0002868884217D10E4800EBC400406828B1E4
:1064F0000B4800EBC40041682846884740F227411A
:106500002868884205D10748FAF7C1FB01200649EF
:10651000087300202860601C44B2132CDDD370BDCA
:106520000C0600207C370020600900200FB410B555
:10653000142202A90D48F1F748FE0C480468142201
:1065400001460B48F1F741FE80210A48F6F7B1FCFD
:10655000094801680548884714210448F1F74EFEB0
:1065600000200249086010BC5DF814FB20110020D7
:10657000E410002000100140080600200FB470B5A0
:10658000DDE9095429484078142810DA2749497868
:1065900001EB81022549091D01EB8200142204A9A7
:1065A000F1F713FE21484078401C204948700598B7
:1065B0006FF30F001E49884218D19DF81B00102868
:1065C00003D09DF81B00132804D19DF81E00194923
:1065D000087007E09DF81B00112803D19DF81C00EE
:1065E000144908700A201449086015E005986FF3F3
:1065F0000F00124988420FD19DF81B000D49097800
:10660000884206D114200C4908600020094908700E
:1066100002E032200849086000210948FCF776FCB6
:106620000020207070BC5DF814FB0000180F0020E3
:106630000000EC1C08010020F00000200000EB1C12
:10664000EC0000200FB410B5142202A93848F1F76D
:10665000BCFD37484068374908603548808880B2BB
:106660004FF25641884204D04FF0FF3010BC5DF825
:1066700014FB2F4840686FF30F002F49884207D161
:1066800014222B492D48F1F7A0FD4FF0FF30EDE724
:10669000274840686FF30F002949884207D1142228
:1066A00023492648F1F791FD4FF0FF30DEE72148FE
:1066B0000068244988422CD01E480068224988423C
:1066C00027D01C4800682149884222D01948006818
:1066D0001F4988421DD0174800681E49884218D0BB
:1066E000144800681C49884213D0124800681B49AE
:1066F00088420ED00F4800681949884209D00D48D9
:1067000000681849884204D00A480068164988423F
:106710000BD1142206491548F1F757FD04498A7A2E
:10672000002348680B3100F04FFD00209EE7000079
:106730000C110020040100200000EC1CC80E0020F9
:106740000000EB1C56F4261856F4011856F40718EE
:1067500056F4081856F40A1056F4121856F41D1878
:1067600056F41F0856F41A1056F41A18040F002095
:106770002DE9F05F0020294908602948486004207D
:1067800008720020487205208872FF2208212348E1
:106790000B30F1F72CFD3320F5F7CEFF18B934207C
:1067A000F5F7CAFFB8B11F48B0F841A00146B1F8EB
:1067B0004300F1F7B2FF80461B4A1C4BF1F7BEFEC7
:1067C000064600221A4BF1F7B6FE0446F1F7DFFF4A
:1067D0001FFA80FB08E01348B0F841A0B0F843006E
:1067E000C0F57A601FFA80FB0C4981F80BA04FEAD4
:1067F0001A210A48017380F80DB04FEA1B218173FA
:10680000084890F8450008B1022100E00121034842
:10681000C17301F0F7F9BDE8F09F0000DC0E002025
:10682000F4561018F00700209A9999999999E93F20
:106830000040AF4010B50446012C25D100204B4943
:1068400008604B4848600420087200204872082005
:106850008872FF22082145480B30F1F7C8FC102050
:106860004249C8720D214148017300214173022140
:106870008173FF21C173002101740621417400213D
:10688000817401F0BFF970E0022C6ED1002037490D
:1068900008603848486004200872002048720820C8
:1068A0008872FF22082131480B30F1F7A0FC01204B
:1068B0002E49C872304890F833102C4801732E4886
:1068C000B0F83300010A294841732B48B0F835006D
:1068D000C0F57A60C1B2254881732748B0F8350009
:1068E000C0F57A60010A2148C173234890F8371037
:1068F0001E4801742048B0F83700010A1B48417453
:106900001D4890F839101948817401F07BF9032073
:10691000F5F739FB02201549C8721748B0F839005D
:10692000010A12480173144890F83B000A30C1B2C2
:106930000E48417300BF104890F83C00C1B20B48AC
:10694000817300BF0C48808F010A0848C1730A4850
:1069500090F83E10054801740748C08F010A0348AB
:1069600041740021817401F04DF910BDDC0E00204E
:10697000F456EC1CF456EB1CF007002010B504464E
:10698000012C25D100203E4908603E484860042083
:1069900008720020487208208872FF2208213848B7
:1069A0000B30F1F724FC10203549C8720921344816
:1069B00001730021417302218173FF21C173002102
:1069C0000174112141740021817401F01BF956E01A
:1069D000022C54D100202A4908602B48486004202A
:1069E00008720020487208208872FF22082124487B
:1069F0000B30F1F7FCFB01202149C872234890F8C5
:106A000046101F4801732148B0F84600010A1C488F
:106A100041731E4890F84810194881731B48B0F81C
:106A20004800010A1648C173184890F84A101448E3
:106A300001741648B0F84A00010A1148417413481D
:106A400090F86C100E48817401F0DCF80320F5F723
:106A50009AFA02200A49C8720C4890F84D1008486A
:106A600001730A48B0F84D00010A0548417300213E
:106A70008173C17301744174817401F0C3F810BD56
:106A8000DC0E0020F456EC1CF456EB1CF007002042
:106A900010B5044600200C4908600C4848600420EA
:106AA00008720020487202208872FF2208210648DE
:106AB0000B30F1F79CFB0449CC72210A02480173A8
:106AC00001F0A0F810BD0000DC0E0020F4562718DD
:106AD00010B586B00446142101A8F1F78FFB012CF4
:106AE00025D100209249086092484860042008722D
:106AF0000020487208208872FF2208218C480B3041
:106B0000F1F775FB10208A49C8723121884801735A
:106B10000021417307218173FF21C173002101749A
:106B2000022141740021817401F06CF8FEE0022C16
:106B3000FCD100207E4908607F484860042008722C
:106B40000020487208208872FF22082178480B3004
:106B5000F1F74DFB01207649C87200BF7748807875
:106B6000087300BF7548C078487300BF7348007948
:106B7000887300BF71484079C87300BF6F4880793F
:106B8000C1B26B48017400BF6C48C088010A6848F4
:106B9000417400BF6948007AC1B26548817401F050
:106BA00031F80320F5F7EFF902206149C87200BF00
:106BB00062480089010A5E4801736048817A5C4836
:106BC00041735E48C17A5A4881735C48017B5848DA
:106BD000C1735A48417B5648017400214174817445
:106BE00001F010F80320F5F7CEF903205049C872E0
:106BF00001214F480173022141735048817C4C4868
:106C000081734E48C17C4A48C1734C48017D484855
:106C100001744A48417D464841744848817D444852
:106C2000817400F0EFFF0320F5F7ADF9002044492F
:106C300081F88701084690F88701012806D11222C1
:106C40003E491A3101A8F1F7C0FA04E0FF221121F0
:106C500001A8F1F7CCFA04203549C8723748C17D44
:106C6000334801733548017E3148417300218173F7
:106C70009DF80410C1739DF8051001749DF806106D
:106C800041749DF80710817400F0BCFF0320F5F7F4
:106C90007AF905202649C8729DF808102448017326
:106CA0009DF8091041739DF80A1081739DF80B102F
:106CB000C1739DF80C1001749DF80D1041749DF87E
:106CC0000E10817400F09EFF0320F5F75CF906209A
:106CD0001749C8729DF80F10154801739DF81010E0
:106CE00041739DF8111081739DF81210C1739DF8C6
:106CF000131001749DF8141041741021817400F078
:106D000081FF0320F5F73FF907200949C8720A21DE
:106D1000074801730B21417307218173E021C1737F
:106D2000FF2101744174817400F06CFF06B010BD46
:106D3000DC0E0020F456EC1CF456EB1CF00700208F
:106D40001017002010B5044600200A4908600A48C0
:106D50004860042008720020487201208872FF22D7
:106D6000082104480B30F1F742FA0248C47200F0DF
:106D700049FF10BDDC0E0020F456091010B5044682
:106D80000020204908602048486004200872002044
:106D9000487207208872FF2208211A480B30F1F749
:106DA00026FA1A4890F86C001649C87200BF1748B6
:106DB00090F86600C1B21348017300BF1348B0F8E1
:106DC0006600010A0F48417300BF104890F8680040
:106DD000C1B20C48817300BF0C48B0F86800010ACA
:106DE0000848C17300BF094890F86A000549087453
:106DF00000BF064890F86B004874084600F002FF98
:106E000010BD0000DC0E0020F4561C18F007002016
:106E10002DE9F04781460024002500260027A046E2
:106E200000207E4908607E484860042008720020E7
:106E3000487207208872FF22082178480B30F1F74A
:106E4000D6F9784890F89701012806D105244B25FA
:106E500004264A274FF0030805E005244B250426A5
:106E60004A274FF003082B20F5F766FC18B92C20B1
:106E7000F5F762FC48B16C4890F85B0020F0030025
:106E8000401C694981F85B0007E0674890F85B00A7
:106E900020F00301644880F85B102D20F5F74CFCCE
:106EA00018B90C20F5F748FC48B15F4890F85B0032
:106EB00020F00C00001D5C4981F85B0007E05A4897
:106EC00090F85B0020F00C01574880F85B102E20F2
:106ED000F5F732FC48B1544890F85B0020F03000E0
:106EE0001030514981F85B0007E04F4890F85B0093
:106EF00020F030014C4880F85B100B20F5F71CFCAB
:106F000048B1494890F85B0020F0C0004030464945
:106F100081F85B0007E0444890F85B0020F0C00176
:106F2000414880F85B100E20F5F706FC18B91A20CE
:106F3000F5F702FC48B13C4890F85C0020F00301F2
:106F4000491C394880F85C1007E0374890F85C002D
:106F500020F00301344880F85C1000BF324890F8FC
:106F60005900012809D1304890F85C0020F00C014C
:106F7000091D2D4880F85C1007E02B4890F85C0054
:106F800020F00C01284880F85C1000BF264890F8DB
:106F90005A00012809D1244890F85C0020F0300103
:106FA0001031214880F85C1007E01F4890F85C0021
:106FB00020F030011C4880F85C1000BF1A4890F89F
:106FC0004F001649C87200BF174890F850000A30A9
:106FD000C1B21248017300BF134890F851000F4925
:106FE000487300BF104890F852000A30C1B20B48F5
:106FF000817300BF0C4890F853000849C8730A48D1
:1070000090F85B1005480174074890F85C1003483D
:10701000417400F0F7FDBDE8F0870000DC0E0020B1
:10702000F456131810170020F007002010B504467E
:10703000002062490860624848600420087200200D
:107040004872042088725F4890F86C00642809D167
:107050005C4890F8610020F00300401C594981F819
:10706000610007E0574890F8610020F0030155489F
:1070700080F861102F20F5F75FFB48B1514890F878
:10708000610020F0C00040304E4981F8610007E007
:107090004C4890F8610020F0C0014A4880F8611027
:1070A0001A20F5F749FB18B90E20F5F745FB48B152
:1070B000444890F8620020F00301491C414880F8E0
:1070C000621007E03F4890F8620020F003013D485D
:1070D00080F862100B20F5F72FFB48B1394890F883
:1070E000630020F00301491C364880F8631007E074
:1070F000344890F8630020F00301324880F86310B0
:107100000320F5F719FB18B90420F5F715FB48B172
:107110002C4890F8630020F00C01091D294880F8E4
:10712000631007E0274890F8630020F00C01254821
:1071300080F863102E20F5F7FFFA48B1214890F847
:10714000640020F00301491C1E4880F8641007E029
:107150001C4890F8640020F003011A4880F864107D
:107160000120F5F7E9FA48B1164890F8640020F0DC
:107170000C01091D134880F8641007E0114890F8CD
:10718000640020F00C010F4880F864100D4890F85E
:1071900061000A49C8720B4890F8621007480173F1
:1071A000084890F8631005484173064890F8641049
:1071B0000248817300F026FD10BD0000DC0E0020A7
:1071C000F4561910F00700202DE9F04105460E464F
:1071D000174698460024F3F7ADFF5649681A8D42CA
:1071E0004CD015DC5449A5EB01008D4273D008DC6E
:1071F0005248284400286CD051490844002869D1DD
:107200004AE050490844E8B1B0F5C02FF7D127E073
:10721000B0F5202F4ED0B0F5901F5DD0B0F5A81F6F
:1072200068D0B0F5F01FEAD1424639463046F3F750
:1072300099FD04462CB14448806B40F4804042499B
:10724000886374E0424639463046F3F7CFFD044682
:107250002CB13D48806B40F001003B49886366E0FB
:10726000424639463046F3F711FE04462CB1364803
:10727000806B40F002003449886358E0424639464A
:107280003046F3F77FFD04462CB12F48806B40F069
:1072900004002D4988634AE0424639463046F3F7F8
:1072A000C3FD04462CB12848806B40F008002649F5
:1072B00088633CE0424639463046F3F701FD044618
:1072C0002CB12148806B40F010001F4988632EE0EC
:1072D00001E01DE02AE000BF424639463046F3F7A0
:1072E000C1FD04462CB11848806B40F020001649BF
:1072F00088631CE0424639463046F3F79FFD04465A
:107300002CB11148806B40F040000F4988630EE0BB
:10731000424639463046F3F711FD04462CB10A487F
:10732000806B40F080000849886300E000BF00BF28
:10733000BDE8F08156F4081856F41A10AA0BE0F7CD
:10734000000015F8000019F8380E0020F0B50346CB
:1073500098180F4FB84201D90320F0BD0AB9002098
:10736000FBE7012600240BE01D780878A84204D032
:10737000FF2D01D00220F0E700265B1C491C641C95
:107380009442F1D3012E01D10020E6E70120E4E789
:107390000000020801460020C80AC0027047000031
:1073A00008B501210820F8F763FF03208DF80200DB
:1073B00014208DF803004FF48060ADF8000069469A
:1073C0000D48F5F799FC03208DF802004FF400609A
:1073D000ADF8000014208DF8030069460648F5F763
:1073E0008BFC4FF480610448F5F763FD4FF40061B6
:1073F0000148F5F75EFD08BD000C014030B50346BD
:107400009818094DA84201D9012030BD0AB90120C0
:10741000FBE7002404E013F8010B01F8010B641CE6
:107420009442F8D30020F0E7000002082DE9F84F5D
:1074300006460F4614464FF0040B30192A4988427D
:1074400002D90120BDE8F88F0CB90020FAE704F05A
:10745000010000B1641C224639463046FFF776FF32
:107460008046B8F1000F01D10020EBE7012080F346
:10747000108800BFF5F742FA3520F5F795F9304648
:10748000FFF788FF0090F5F795F983464FF47A7A75
:1074900000BFBAF10000AAF101011FFA81FAF8D188
:1074A000002511E017F815906800401C385C49EA87
:1074B000002949463046F5F7C7F98346BBF1040F6A
:1074C00000D004E0B61C6D1CB5EB540FEAD300BF2E
:1074D000F5F7B0F9002080F3108800BFBBF1040F6E
:1074E00000D1AFE70220ADE70000020810B5044666
:1074F0003CB900210748F3F7B1F90648F2F796FDC9
:1075000006E000210448F3F7A9F90348F2F78EFDDD
:10751000012010BD006400400068004070B50546C1
:107520000C46022D00DB70BD05EB85000D4901EB1B
:107530008000006988B1A37A207A042801D16068AC
:1075400000E02068014605EB8500064A02EB80005A
:1075500004F10B0206692846B047284600F0DCF922
:1075600000BFE0E73411002070B505460E460DB9A6
:10757000064900E0064908463146F3F753FA044647
:10758000042C00D1FF24204670BD000000640040A0
:107590000068004070B504460D461646022C00DB1C
:1075A00070BD04EBC400144901EB8000C0680121E8
:1075B000A9400840F0B104EBC4000F4901EB800082
:1075C000C0680121A940884304EBC4010A4A02EBC8
:1075D0008101C860204600F09FF904EB8400074950
:1075E00051F8200030B104EB840051F820202946E6
:1075F0002046904700BFD3E75C11002034110020E3
:1076000070B504460D4614B9F3F76CF801E0F2F7D3
:1076100017FB012070BD000010B50446832C00D07C
:1076200010BD0A48007C01280ED00948C06A18B174
:107630000748C16A012088470120044908740021D5
:1076400002481430FBF762FC00BFE9E7CC160020CB
:107650009C1600202DE9F04105460E4626BB2F461C
:1076600000240FE0124800EB04100068B84207D174
:107670000F4901EB041101F10C000021FBF746FC5E
:10768000601C84B2022CEDD300BF0A48807F002822
:107690000BDD0848007C022807D1002105488177CE
:1076A0001830FBF733FC00E000BFBDE8F0810000BC
:1076B0005C010020CC16002010B50446002004EB2D
:1076C000C401044A02EB810188602046FFF70EFFE7
:1076D00010BD00005C11002010B50446022C00DB38
:1076E00010BD04EB84000D4901EB8000806890B16F
:1076F00004EBC4000A4B03EB8000C06808B1012012
:1077000000E00020014604EB8400044B03EB800002
:1077100082682046904700BFE2E700003411002055
:107720005C11002010B50446022C00DB10BDF9F7F7
:107730001CFA04EB84000F4901EB8000C06838B1EB
:1077400004EB84000A4602EB8000C16820468847AB
:10775000F9F70DFA04EBC400074901EB8000C0689B
:1077600030B1002004EBC401034A02EB8101C86080
:1077700000BFDBE7341100205C1100207CB5002045
:107780000090019000246CE0374800EB0410007872
:1077900001284CD1344800EB04108089062807D218
:1077A000314800EB04108089304931F8105001E075
:1077B0002E4845892C4901EB0411081D2946FBF789
:1077C000A5FB00284BD0F9F7D0F9274800EB0410AF
:1077D0008089401C244901EB0411888104EB44009A
:1077E000234901EBC000C06848B104EB440001EB41
:1077F000C00000231A461946C6682046B04702203A
:10780000194901EB0411087001208DF80000F9F707
:10781000AEF9154901EB041101F108000021FBF755
:1078200075FB0120104901EB0411887317E00E4825
:1078300000EB04100078022811D10B4901EB041170
:1078400001F108006721FBF761FB40B10020064908
:1078500001EB04118881044901EB04110870601CDC
:10786000C4B2022C90DB7CBDCC16002030C10108D4
:107870009C1600202DE9F04104460D4616461F4691
:10788000022C02DB0020BDE8F081012004EBC401E2
:10789000204A02EB81018860002004EBC40102EB66
:1078A0008101487104EBC400114601EB80000771AF
:1078B00004EBC40001EB8000C67004EBC40021F8A7
:1078C0002050002004EBC40102EB8101C86004EBEE
:1078D000C40002EB80012046FFF792FE38B102207F
:1078E00004EBC4010B4A02EB8101886006E0002032
:1078F00004EBC401074A02EB8101886004EBC40079
:10790000044901EB80008068022801D10120BAE718
:107910000020B8E75C110020022800DB704700BFA0
:10792000FCE700002DE9F04104460E461746984654
:10793000022C07DA04EBC400194901EB80008068CF
:10794000022802D00020BDE8F08104EBC401144AF3
:1079500002EB810101F1100043463A463146F2F74D
:1079600081FB04EBC4000E4A02EB800000F1100121
:107970002046FFF7F9FD0546FF2D0ED004EBC400AD
:10798000074901EB8000C1680120A840014304EBD6
:10799000C400034A02EB8000C1602846D3E7000020
:1079A0005C110020FEB504460D4616460094019574
:1079B00002966946014803F0FCFEFEBD2414002037
:1079C00010B500F0A9F800F047F810BD10B500F0B0
:1079D00055F800F0ABF810BD10B502460B4612B9D1
:1079E0004FF0FF3010BD002114E01A4850F831006C
:1079F00090420ED1174800EBC1004360154800EBE0
:107A0000C100406818B90020124C44F83100002031
:107A1000E8E7491C1429E8D313B94FF0FF30E1E738
:107A2000002111E00B4850F8310020B1094800EB6B
:107A3000C100406838B9074840F8312000EBC10068
:107A400043600020CEE7491C1429EBD34FF0FF30F0
:107A5000C8E70000A411002010B54FF426710648B5
:107A6000F0F7CCFB28230C220349A03101F5F0707C
:107A700003F074FE002010BDA41100203EB518E0F4
:107A800069460F4803F078FE00240FE00D4850F8D7
:107A900034000099884208D10A4800EBC4004568C8
:107AA00015B19DE80700A84702E0641C142CEDD333
:107AB00000BF034803F040FE0028E1D000203EBD97
:107AC00024140020A411002010B502460AB9002099
:107AD00010BD002119E001EB41000E4B03EB8000CB
:107AE000806880B901EB410003EB800082600020D8
:107AF00001EB4103074C44F8230001EB410023460E
:107B000003EB8000E4E7481C81B21429E3D3002092
:107B1000DEE700003C14002010B5F0210248F0F729
:107B20006DFB002010BD00003C140020F8B50027BC
:107B300000216846FBF7EAF90098B84203D0781CA8
:107B40000099814201D10020F8BD009F00243BE054
:107B500004EB44001E4901EB8000866804EB4400FE
:107B600051F820507DB376B304EB4401184A02EB80
:107B70008101081D2946FBF7C9F9012823D104EB2F
:107B80004400134901EB80008068A8B104EB440075
:107B900001EB800040680099081AB0FBF5F004EB97
:107BA00044010B4A02EB8101496800FB051004EB1C
:107BB000440102EB810148602EB104EB4401044A08
:107BC00002EB8100B047641C142CC1D30020BBE73A
:107BD0003C14002070B504460E46254605B970BD1C
:107BE0002E600021281DFBF791F900BFF7E7014641
:107BF0000A460AB900207047106808B10120FAE768
:107C00000020F8E77CB50446002611480068E0B182
:107C10000021207A042801D1606800E02068CDE9C5
:107C20000001607A08B9A07A00E000200346207ABB
:107C3000042801D1606800E020680146044804F18E
:107C40000B0205680020A8477CBD0020FCE700006F
:107C50009C1600202DE9FC4104460027FCF76AFD34
:107C600060B9217A042901D1616800E021680846E1
:107C7000FCF774FD10B90120BDE8FC812048806943
:107C800000283AD00021207A042801D1606800E061
:107C90002068CDE90001607A08B9A07A00E00020F0
:107CA0000346207A042801D1606800E0206801467C
:107CB000134804F10B0285690120A847E8B1207A36
:107CC000042801D1606800E02068064600250FE026
:107CD0000C4800EB05100068B04207D1094901EBE0
:107CE000051101F108000021FBF710F9681C85B2AD
:107CF000022DEDD300BF0020BEE70020BCE700004E
:107D00009C1600205C01002010B50F48008868B95F
:107D100001200D49088000BF00200C4948720C4822
:107D2000F6F7E0FE0BA0FDF767FD0CE0002006492A
:107D3000088000BF0120054948720548F6F7FDFE9E
:107D400009A0FDF759FD10BD50050020EC250020CD
:107D5000000B0020B9D8B1D54443CEC2B6C8BCCCC4
:107D6000B5E7C6F70D0A0000BFAAC6F44443CEC269
:107D7000B6C8BCCCB5E7C6F70D0A000010B50A4876
:107D8000008840B9012008490880F3F775FA07A078
:107D9000FDF732FD07E0002003490880F7F742F8BD
:107DA00007A0FDF729FD10BD48050020B9D8B1D5C1
:107DB000BDBBC1F7BCCCB5E7C6F70D0A000000009B
:107DC000BFAAC6F4BDBBC1F7BCCCB5E7C6F70D0A68
:107DD000000000007047000010B50F48008868B927
:107DE00001200D49088000BF00200C49C8710C48D3
:107DF000F6F778FE0BA0FDF7FFFC0CE0002006492B
:107E0000088000BF01200549C8710548F6F795FEB6
:107E100007A0FDF7F1FC10BD4C050020EC2500206B
:107E2000C40A0020B9D8B1D543433143500D0A00EC
:107E3000BFAAC6F443433143500D0A0010B50F48A2
:107E4000008868B901200D49088000BF00200C4956
:107E500008720C48F6F746FE0BA0FDF7CDFC0CE0CF
:107E600000200649088000BF012005490872054826
:107E7000F6F763FE08A0FDF7BFFC10BD4E0500201D
:107E8000EC250020EC0A0020B9D8B1D54343325F7D
:107E900043430D0A00000000BFAAC6F44343325F0B
:107EA00043430D0A00000000F6F778FF10B51248B2
:107EB000008880B901201049088000BF00200F49C8
:107EC00088710FA0FDF798FC1148F6F70BFE11A082
:107ED000FDF792FC0FE000200749088000BF012059
:107EE0000649887110A0FDF787FC0948F6F725FEC2
:107EF00011A0FDF781FC10BD46050020EC250020F7
:107F0000434C4F53455F44435265616C790D0A0001
:107F10009C0A0020B9D8B1D5D6B1C1F7BCCCB5E721
:107F2000C6F70D0A000000004F50454E5F44435213
:107F300065616C790D0A0000BFAAC6F4D6B1C1F71D
:107F4000BCCCB5E7C6F70D0A0000000070477047CB
:107F50007047000010B50C48008850B901200A494C
:107F6000088000BF0948F6F7BDFD09A0FDF744FCF5
:107F700009E000200449088000BF0448F6F7DDFD51
:107F800007A0FDF739FC10BD4A050020D80A0020E3
:107F9000B9D8B1D5C9FDD1B9C4A3BFE90D0A000054
:107FA000BFAAC6F4C9FDD1B9C4A3BFE90D0A000038
:107FB000704770477047000010B51048008870B9CE
:107FC00001200E49088000BF0D48F6F78BFD00BF69
:107FD0000C48F6F787FD0CA0FDF70EFC0DE0002025
:107FE0000649088000BF0648F6F7A7FD00BF054810
:107FF000F6F7A3FD08A0FDF7FFFB10BD4405002028
:10800000D80A0020B00A0020B9D8B1D5B8DFD1B95C
:10801000C4A3BFE90D0A0000BFAAC6F4B8DFD1B9F6
:10802000C4A3BFE90D0A000070B502460B46FF214C
:108030002F25002012E0145C614000240AE001F0CA
:1080400080061EB185EA4106F1B201E04E06310E0E
:10805000661CF4B2082CF2DB441CE0B29842EAD36E
:1080600081F0FF0070BD2DE9F04705460E460D205A
:10807000FBF798F80A20FBF795F82C46002710E04C
:108080002078F5F7B8FD80462078F5F7A7FD814602
:108090004046FBF787F84846FBF784F8641C781CD9
:1080A00087B2B742ECDB0D20FBF77CF80A20FBF728
:1080B00079F8BDE8F08710B5FFF772F910BD2DE92A
:1080C000F04107460C461646F6F7A0F8A020F6F752
:1080D0006FF8F6F7C9F800B130E0A046E11704EBFD
:1080E0001161C1F30720F6F763F8F6F7BDF800B1A8
:1080F00024E0E0B2F6F75CF8F6F7B6F800B11DE060
:10810000F6F784F8A120F6F753F8F6F7ADF800B1CA
:1081100014E000250BE0711EA94201D0012100E00E
:1081200000210846F6F71AF87855681C85B2B54262
:10813000F1DBF6F785F80120BDE8F081F6F780F86D
:108140000020F9E72DE9F04706460F4690463C46E9
:10815000002534E035B1E11704EBD1614911A4EBFE
:10816000411109BB25B1F6F76BF80620F3F70BFFB9
:10817000F6F74CF8A020F6F71BF8F6F775F800B103
:1081800024E0A146E11704EB1161C1F30720F6F7E3
:108190000FF8F6F769F800B118E0E0B2F6F708F862
:1081A000F6F762F800B111E0705DF6F701F8F6F746
:1081B0005BF800B10AE0601C84B2681C85B24545DA
:1081C000C8DBF6F73DF80120BDE8F087F6F738F890
:1081D0000020F9E710B506E000F02CFA044620462E
:1081E00001F0CCF800BF00F0DDFD0028F4D010BD98
:1081F00070B504460D46E1B21948FCF732FA00BFEB
:108200001748008800F080000028F9D0154890F841
:10821000A800012822D11448807802281AD11348D6
:108220000078962808DA114802780078401C0F4B35
:1082300018700F48845411E00C4801780C48FDF781
:1082400045F90948007C401C07490874002007498B
:10825000087003E00020034981F8A800204670BDA3
:10826000004C0040101700207C2100203A0500201F
:108270004D24002038B50E4A106F126FD16B88471D
:10828000009069460B48F4F7B7FB0446012C09D16E
:1082900002210948F8F7E8FC20B10748F8F7F7FC95
:1082A000012038BD14B90448F8F7F1FC0020F8E7C4
:1082B000F0070020C02600205437002010B51848D1
:1082C00090F8380000F0010040B1164840790128CC
:1082D00004D115A0FDF790FA012010BD104890F8C8
:1082E000380000F0010038B102200E49487114A096
:1082F000FDF782FA0120F0E7174908698047022854
:1083000001D00220E9E70A211448F8F7ADFC20B1BA
:108310001248F8F7BCFC0320DFE70020DDE700008F
:10832000380E0020D4250020424D535F50524F5448
:108330004F43414C5F4742323031350A0D00000057
:10834000424D535F50524F544F43414C5F4742326E
:108350003031310A0D0000006C000020143700207D
:1083600010B51449086980470446022C11D1124AFD
:10837000106F126FD16A8847042819D1F4F7A6F953
:10838000B8210E48EFF73AFF0DA0FDF735FA0120AE
:1083900010BD012C0AD1F4F799F9B8210748EFF77D
:1083A0002DFF0CA0FDF728FA0220F1E70320EFE7EC
:1083B0000020EDE76C000020F00700200C370020C3
:1083C000BDF8C8EBD6B1C1F7B3E4B5E7C1F7B3CC9C
:1083D0000D0A0000BDF8C8EBBDBBC1F7B3E4B5E7BB
:1083E000C1F7B3CC0D0A000010B50D48008F00F4A2
:1083F000804028B90A4890F8380000F0010028B100
:108400003D210748EFF7FAFE012010BD0549086934
:108410008047022801D00220F7E70020F5E700009E
:10842000380E00206C00002010B50D48C078AA2836
:1084300004D10CA0FDF7E0F9012010BDF8F726F8F3
:1084400020B90FA0FDF7D8F90220F6E71A4908690C
:108450008047022801D00320EFE70020EDE700006D
:10846000380E002052455620445F43445A5F48412D
:108470004E44494E475F43524D2041410A0D000092
:1084800052656164792D537461746520526563652A
:108490006976656420546865204368617267696E17
:1084A000672050696C652041626F7274204D65735E
:1084B000736167650A0D00006C00002010B5F7F7C6
:1084C000E5FF20B909A0FDF797F9032010BDF9F7E2
:1084D00009F908B90120F9E713490869804702281A
:1084E00001D00320F2E70020F0E7000052756E6E25
:1084F000696E672D53746174652052656365697692
:10850000656420546865204368617267696E6720FE
:1085100050696C652041626F7274204D65737361A0
:1085200067650A0D000000006C00002010B52148AE
:10853000807EAA2804D120A0FDF75EF9012010BD9D
:10854000F7F7A4FF20B923A0FDF756F90320F6E7BB
:108550002820F4F7F1F8B8B90620F4F7EDF898B947
:108560001C20F4F7E9F878B92120F4F7E5F858B9B8
:108570000920F4F7E1F838B90A20F4F7DDF818B962
:108580002620F4F7D9F808B10320D8E71F49086975
:108590008047022801D00520D1E73C211C48F8F78C
:1085A00063FB20B11A48F8F772FB0420C7E70020EC
:1085B000C5E70000380E002043445A5F5F43524F26
:1085C00020414120746F204368617267696E670AB9
:1085D0000D00000053746172742D53746174652032
:1085E00052656365697665642054686520436861F7
:1085F0007267696E672050696C652041626F7274A2
:10860000204D6573736167650A0D00006C000020E2
:108610002C37002010B505210548F8F725FB20B1BF
:108620000348F8F734FB012010BD0020FCE70000F0
:108630004437002010B500F0B5FB08B1002010BD94
:10864000074808490968445C06480068401C052141
:1086500090FBF1F201FB1200024908602046EEE7B0
:108660003C0C0020340C002070B504460D4600265A
:1086700029462046F0F7A6FBF7F7D4FF064630461A
:1086800070BD0146072070477047014602207047C1
:1086900010B51248008F00F4804078B100200F49D7
:1086A000886301200E49487100BF0E4800880446C7
:1086B000FEF7EEF90CA0FDF79FF80EE040F6B8319A
:1086C00007480830FAF722FC38B10CA0FDF794F8FF
:1086D000002103480830FAF719FC10BD380E0020BD
:1086E000D4250020F0070020445F43445A5F4841EE
:1086F0004E44494E475F43484D0D0A004E4F2048B7
:10870000616E647368616B65205369676E616C0AA2
:108710000D0000000146002070477047014601200F
:1087200070477047014603207047000010B50B48A2
:10873000007920B1012807D002280DD108E00221DC
:108740000748F4F73BFA07E00548F4F769FA03E055
:108750000220F4F775FA00BF00BF10BDD425002039
:10876000D16A010801460520704710B5F2F792FE64
:1087700010BD01460420704770B500264048C07CFB
:10878000012813D1F2F772FE80B1FCF7BBFE68B985
:10879000F0F7B0FC50B1F8F781FA38B939480079F0
:1087A000012803D1F0F702FE064600E00026354618
:1087B0002C46354890F8380000F0040038B93048AD
:1087C000C07C012825D13048807EAA2821D02046AF
:1087D000FEF7B8FA2D4A106F126F516B88470128C7
:1087E0000DD12848007950B900BF01202549887172
:1087F00027A0FDF701F82A48F6F79FF900BF0120EE
:108800001F49C8742048806B20F004001E4988630B
:1088100018E01B48C07CA8B92248007920B1012883
:1088200007D002280DD108E006211F48F4F7C6F949
:1088300007E01D48F4F7F4F903E00620F4F700FA26
:1088400000BF00BF104890F8380000F0020030B1BF
:108850000D48806B20F002000B4988630EE00A4847
:1088600090F8380000F0080040B110A0FCF7C4FFF9
:108870000548806B20F008000349886370BD000044
:1088800030260020EC250020380E0020F0070020C4
:108890004F50454E5F44435265616C790D0A0000AC
:1088A0009C0A0020D42500203568010843445A5F03
:1088B00048414E44494E475F43524D2041410A0DC5
:1088C00000000000014606207047000038B51C4932
:1088D000096FB1F90200002801DB014600E04142C6
:1088E00089B2009169461748F4F786F808B101206B
:1088F00000E00020044614480079012803D1012C2F
:1089000001D1F2F7EBFC32211048FAF7FFFA012807
:1089100006D10020FEF78AFB00210C48FAF7F6FA90
:10892000FA210A481030FAF7F1FA012807D100209D
:10893000FEF724FA002105481030FAF7E7FA38BDAF
:10894000F0070020B4260020EC250020142600208B
:1089500070B505460E463046F4F7EEFD044604B900
:1089600070BD812D26D004DC042D07D0802D4DD183
:1089700016E0822D0AD0832D48D128E094F85400C7
:10898000032802DB2046F5F72FFA40E094F8540064
:10899000032804DBE06C10B18220E16C884736E0EC
:1089A00094F85400032804DBE06C10B18020E16CE3
:1089B00088472CE094F85400032807DB2046F5F79D
:1089C000B3FAE06C10B18120E16C88471FE094F8A5
:1089D0005400032819DB9120005D022806D10421F0
:1089E0009120015522780120FEF7DCFFE06C18B1E0
:1089F0008320E16C884708E0207800F05FFB207856
:108A000000231A46194600F0CBFB00E000BF00BF70
:108A100000BFA5E770B506460D463046F4F78CFD5D
:108A200004461CB394F85400022805DCE068E8B161
:108A30003046E168884719E094F85400812808D14D
:108A40003DB184F85400324681210120FEF7AAFF8F
:108A50000CE094F85400812808D03DB9802084F8B7
:108A60005400324680210120FEF79CFF70BD70B596
:108A700004460D4629462046FFF7CCFF70BD70B571
:108A800005462846F4F758FD04468CB194F8540086
:108A9000022805DCE06858B12846E168884707E00D
:108AA000832084F854002A4683210120FEF77AFFB0
:108AB00070BD00002DE9F04107460D4690461E4668
:108AC0003846F4F739FD0446002C39D094F85400A8
:108AD000032835DB94F85400802802D1032084F861
:108AE000540094F8400000F0010038B1A06C38B395
:108AF000324641462846A36C984721E0124805605B
:108B000006710079002809DD0F480079082805DC86
:108B10000D4802794146401DEFF757FB0A4904F121
:108B2000580002F046FE04F1580002F00EFE38B183
:108B3000822084F854003A4682210120FEF732FF59
:108B40000120BDE8F08100008C16002070B50646BB
:108B50000C463046F4F7F0FC05461DB1E1B228465C
:108B6000F5F7FBF970BD002001E0411C88B23C28FC
:108B7000FBDB704710B514206C4981F86C0041F2A2
:108B8000883008800120887001216848C170002168
:108B90000171032141714FF47A71C18041F2680182
:108BA0000181422181725921C172442101735421F2
:108BB000417300218173C173012101740221417449
:108BC000192181740B21C1740A210175002141759D
:108BD00081751021C175002101764176112254A1C1
:108BE0001A30EFF7F2FA51482B3056A10A680260AA
:108BF000496841604FF4D2704C49A1F833004FF4FA
:108C0000FA714A48A0F8351041F22431A0F8391021
:108C10006E2180F83B10C82181874FF47A61C187AB
:108C20000020424981F840004FF47A60A1F84100E9
:108C30004FF416713D48A0F84310022180F845100A
:108C400000203A49A1F8460000213848A0F8481011
:108C5000B0F84A006FF30B0000F5A2703349A1F899
:108C60004A00084690F84B0020F0F00110312F48E0
:108C700080F84B103C21A0F84D1001202B4981F8C1
:108C80004F006FF0310232490A20FCF75FFCC1B29D
:108C9000264880F85010032180F851106FF03102FF
:108CA0002B490520FCF752FCC1B2204880F8521035
:108CB000042180F85310002180F8541080F85510DA
:108CC00080F8561080F8571080F8581080F8591026
:108CD00080F85A100120154981F85D0000211348E1
:108CE000A0F85E1080F860106420104981F86500DB
:108CF00040F259110D48A0F8661040F26311A0F837
:108D000068106FF0310212491920FCF71FFCC1B244
:108D1000064880F86A106FF031020D491C20FCF7FC
:108D200015FCC1B2014880F86B1010BDF00700209F
:108D30004C56504335323739584E44303133383140
:108D4000380000005330303148303031000000002E
:108D5000CDCCCC3D2DE9F0410B3020F00706104D75
:108D600019E02068B04215D3B0420AD9871B201DF4
:108D7000D4F80480EFF729FAA019C0E90078286038
:108D800004E060682860201DEFF71FFA201D2660B0
:108D9000BDE8F081251D2C68002CE2D10020F7E70A
:108DA000780D00200448006804490968884201D110
:108DB000012070470020FCE7340C0020380C002014
:108DC00007480068401C052190FBF1F201FB1200EE
:108DD00004490968884201D1012070470020FCE75E
:108DE000380C0020340C002070B504460D4618489D
:108DF0000078B0B929462046FFF736FC15490968C6
:108E0000084414490860144801780078401C124A4C
:108E10001070092902DB01200D4908700F480088F5
:108E200070BD00200A4908700A4800680C490860B3
:108E300000200849086008490870094800680A21AC
:108E4000B0FBF1F00549088008460088E8E700001B
:108E5000E1000020D8000020E0000020D400002025
:108E6000DC00002086B0F8F7F1FC62B64FF4004158
:108E70000803F5F789FFF8F7A7FC01A8F7F70EFA42
:108E8000F5F72DFFF5F7C0FBF5F78EFAFFF713F9AD
:108E9000F0F79CFAF0F706F8EFF7B8FF4FF47A30E6
:108EA00002F0E2FC4FF4E13002F038FD40F2CF2155
:108EB00040F2F310F8F740FDF3F72CFEFFF75AFEEF
:108EC000FBF7DEFBF5F738FAFDF70CFA59495AA023
:108ED000FCF792FCF7F74CFBF2F73AF9F3F754FD85
:108EE00001205849887300BF5748F5F726FEF5F76B
:108EF00099FF00BF0020554908725548F5F7F2FD6B
:108F000000BF00205149C8715248F5F7EBFD00BF82
:108F100000204E4948725048F5F7E4FD88E0FAF722
:108F200033F8FDF77BF94D480078012828D100205F
:108F30004A4908704348807B48B10320F3F7FCFBA3
:108F400028B90420F3F7F8FB08B9F0F75BF8F0F75D
:108F5000E9FAFBF790FB4249086880474049C86836
:108F600080473F49486880473D4988688047F8F70F
:108F700027FAF2F769FFEFF727FEF5F7D1F957E087
:108F800036484078012807D1002034494870F3F76B
:108F90003DF8F7F729FE4BE03048807801280ED1E4
:108FA00000202E4988700220F4F7ECFA0446EFF70F
:108FB000C1FB00B22B498881FBF757FB38E02748FB
:108FC000C078012807D100202449C870F2F7CCFBF3
:108FD000F2F77AFD2CE02148007901280BD100201E
:108FE0001E490871F7F748FDF3F768FFF2F7F0F94B
:108FF000F5F7FEFD1CE019484079012807D1002053
:1090000016494871EFF796FDFFF7E4F810E01348B2
:10901000C07901280CD100201049C871F6F78EFDE7
:10902000F0F7E6FAF6F7F0FFFCF77CFBFBF7D0FB76
:1090300075E700003CC10108B0E6B1BEBAC5202505
:10904000730D0A00D42500202C0C0020EC250020F4
:10905000EC0A0020C40A0020000B002000170020AA
:1090600080000020A00D00202DE9F04704460F46A7
:10907000154699463DB161190E48814203D8A0F5C5
:109080000070844203D24FF0FF30BDE8F08737B163
:10909000002602E0B85DA055761CAE42FAD3064821
:1090A000A4EB0008AAB21FFA88F12046FBF704FBE4
:1090B0000020EAE75C4B00205C49002070B50546C3
:1090C0002846F4F739FA04461CB194F854000228F3
:1090D00001DC002070BD022084F85400E06810B16B
:1090E0002846E16888479120005D002834D0D4F8F4
:1090F000A800B0B19120005D052804D10021D4E979
:109100002902904728E09120005D042804D1012124
:10911000D4E9290290471FE00321D4E929029047AE
:109120001AE0206DC0B19120005D052805D1002115
:10913000226DD4F8A40090470EE09120005D042831
:1091400005D10121226DD4F8A400904704E0032149
:10915000226DD4F8A400904715E004F1940104F1C5
:10916000700002F009FB70B1D4F8A80020B103210F
:10917000D4E92902904706E0206D20B10321226D39
:10918000D4F8A400904704F1700002F0D5FA00284A
:10919000E3D0202104F19000EFF730F8012099E7A7
:1091A0002DE9F04105460E46174698462846F4F745
:1091B000C3F904461CB194F85400012802DC0020D5
:1091C000BDE8F081606848B343463A4631462846D8
:1091D000D4F804C0E04708B3D4F88C0040B194F848
:1091E0004530182204F17000D4F88C1002F0B6FA61
:1091F00094F8400000F0010058B9D4F8880040B15C
:1092000094F84530102204F15800D4F8881002F088
:10921000A5FA032084F854000120D1E70020CFE70D
:1092200070B5054600242846F4F786F9044614B1C3
:1092300094F8540070BD0020FCE72DE9FF41804602
:109240000E4615461F464046F4F776F904464CB1E3
:1092500094F85400022805DD25B194F8400000F090
:10926000010018B1002004B0BDE8F08104F15800FD
:1092700002F062FA08B10020F5E7694604F15800EF
:1092800002F07AFA08B90020EDE7009830609DF806
:10929000040038709DF8040000280ADD9DF80400E1
:1092A000082806DC9DF804200DF105012846EEF79C
:1092B0008CFF94F85400822802D1032084F85400D3
:1092C0000120D0E72DE9F04786B080460F461546CD
:1092D0001E46DDE90E9A00244046F4F72DF90446B7
:1092E00054B194F85400022806DD082E04DC04F181
:1092F000700002F02AFA18B1002006B0BDE8F0872D
:10930000F7F733FC94F85400832803D094F8540002
:10931000032803DAF7F72BFC0020EEE7CDF814A0C2
:1093200000978DF80560CDF8109015B900208DF8E4
:1093300005009DF8050000280ADD9DF805000828B5
:1093400006DC9DF8052029460DF10600EEF73DFFED
:10935000FF208DF80400694604F1700002F029FA3C
:109360009120005D10B92046F4F73EFDF7F7FFFBB2
:109370000120C2E7034600207047000010B50446F4
:10938000062C13D2DFE804F0120306090C0FF3F7E2
:1093900007F90FE0F3F748F90CE0F3F751F909E0AA
:1093A000F3F70AF906E0F3F757F903E002A0FCF738
:1093B00023FA00BF00BF10BD556E6B6E6F776E2035
:1093C0006576656E742069732069676E6F72656477
:1093D0000A000000F0B54FF480541B4A0023072711
:1093E00002EA070600256E406D402E4307D0D21DCD
:1093F0006FF0070602EA0602134D551B641B114667
:10940000124D29604FF00005104E75600A19083A98
:109410006FF0070602EA06020D4D2A604FF00005C4
:109420000B4E366875600A4E366835600846151A68
:109430004560074D2D680560064E45683560064E4F
:1094400045683560F0BD00000A270020440C00206C
:109450004C0C0020540C0020500C002010B501468C
:10946000184800E0006803688B42FBD3024643685B
:1094700013448B4205D143684C6823444360014642
:1094800000E000BF0A464B6813440468A34211D1B0
:109490000D4C03682468A34208D04B6804686468D4
:1094A00023444B6003681B680B6005E0064B1B6898
:1094B0000B6001E003680B60884201D0016000E0AE
:1094C00000BF10BD440C00204C0C00202DE9F047DB
:1094D00005464FF000093848006810B9FFF77AFFD9
:1094E00000E000BF7DB105F00700C0F11008C8F131
:1094F000FF30A84201D2012000E0002008B9454415
:1095000002E0002500E000BF012000EBE57000282C
:109510004CD0002D48D029480068854244D8284EB8
:109520003046046801E0264624686068A84202D2FA
:1095300020680028F7D120480068844232D0306883
:1095400000F10809206830606068401B10280AD9C3
:10955000671900BF00BF6068401B786065603846CF
:10956000FFF77CFF00E000BF144960680968081A33
:10957000124908600846006812490968884204D206
:109580000E4800680F49086000E000BF606840F0C6
:1095900000406060002020600B480068401C0A49C1
:1095A000086004E000BF02E000BF00E000BF00BFB1
:1095B00000BF4846BDE8F0874C0C0020500C00204E
:1095C000440C0020540C0020580C00202DE9F04FD2
:1095D00099B0834600201890402106A8EEF70EFEB1
:1095E000002005904FF6FF7004905C460020F14982
:1095F0000874B4F8050048F22001884204D0B4F899
:109600000500491C884243D1CDF80CB0B4F802A043
:10961000B4F8050002906088B0F5967F04DC62889B
:10962000E11DE548EEF7D1FD5146E348FEF71BFD8D
:10963000AAF1020003990A5C401C085C42EA00207F
:109640001690AAF1020081B20398EFF7E7FE179097
:10965000DAA0DDE91612FCF7CFF8DDE91601884241
:1096600005D0DCA0FCF7C8F819B0BDE8F08F0020E9
:10967000D04948740299E031C8B25246CE49FBF74E
:109680004DFC6420DB4908800420CA498870EBE760
:10969000B4F80500B0F5004F5FD034DCB0F5D06F02
:1096A00001F0C38714DCB0F5607F72D009DC80283C
:1096B00054D0B0F5C07F79D0B0F5207F41F0E68777
:1096C00083E0B0F5906F66D0B0F5B06FF6D1AAE048
:1096D000B0F5286F01F0D2870CDCB0F5F06F01F027
:1096E000B787B0F5086F01F0B887B0F5186FE5D10E
:1096F00001F0B8BFB0F5025F01F0C587B0F5065FB5
:10970000DCD101F0C2BF48F20702811A904201F099
:109710009E870DDC6FF400410844062881F0B6876F
:10972000DFE810F043005200610066008000820F05
:10973000062901F09C8709DC012901F08D870229A7
:1097400001F08F870329B9D101F090BF192901F0E9
:1097500099871A29B2D101F097BF00BFE07901289B
:109760001ED194498870A44981F8760008460021EA
:10977000C1660167A0F874100146A268CA66E06875
:10978000086701208B4988709C4908709A496C31A0
:1097900002E029E00AE02CE099A0FCF72DF802E0B5
:1097A0009FA0FCF729F801F072BF00BFE079012803
:1097B00006D102207F4988709EA0FCF71DF802E0C8
:1097C000A1A0FCF719F8EEE700BFE179A2A0FCF731
:1097D00013F8A649D4F809200A60B4F80D208A804D
:1097E000E07B8871DFE700BFA1A0FCF705F8DAE7AE
:1097F00000BFA5A0FCF700F8207A012801D1A8A09D
:1098000000E0A9A00146AAA0FBF7F6FF207A40B924
:109810000120AA490870AA48007810B90420A84974
:109820000870C0E700BF0120A6490870E07918B9A8
:10983000A5A0FBF7E1FF02E0A7A0FBF7DDFFE079C1
:10984000012841F07786267A3146A7A0FBF7D4FF9E
:10985000012E14D1607A40B90120984908709848C7
:10986000007810B9042096490870607A012801D167
:10987000A1A000E0A2A00146A3A0FBF7BDFF022E1D
:1098800009D1607A012803D1A3A0FBF7B5FF02E05C
:10989000A5A0FBF7B1FF042E1BD104F10900EEF7E0
:1098A000CAFC85B2102D0FD22A4604F10901524894
:1098B0001030EEF78AFC04F109019FA0FBF79CFF32
:1098C00001204E49087004E004F109019FA0FBF754
:1098D00093FF072E0AD1657A2946A3A0FBF78CFFD8
:1098E0004548A0F86950012044490870062E0ED161
:1098F000657A2946A3A0FBF77FFF3F48A0F84D50AB
:10990000A0F84F50A0F8515001203C490870082E93
:1099100003D1657A012039490870092E1DD104F15F
:109920000900EEF788FC85B2102D0ED22A4604F10C
:1099300009013148EEF749FC04F1090197A0FBF752
:109940005BFF01202D49087004E004F1090199A092
:10995000FBF752FF0120294908700A2E14D1657ABD
:10996000012D07D10120244981F8870098A0FBF739
:1099700043FF06E00020204981F8870094A0FBF710
:109980003BFF01201D4908700B2E00D1657A0C2E7B
:109990000FD1657A012D07D10120174981F889007F
:1099A00091A0FBF729FF32E10020134981F88900DB
:1099B0002AE12FE17C210020822200200A0D44634D
:1099C0007263202530782C56637263202530780A24
:1099D0000D0000000A0D20284463726320213D2001
:1099E00056637263292072657475726E212121217C
:1099F000210A0D003805002010170020FC0100206E
:109A000072656769737465726564207375636365F5
:109A1000737365642C436F64652025730A0D000021
:109A200072656769737465726564206661696C65E7
:109A3000640A0D004C6F67696E205375636365732C
:109A40007365640A0D0000004C6F67696E20466103
:109A5000696C65640A0D0000686561727420636F4B
:109A6000756E742025640A0D000000002D0E002084
:109A700072656365697665207374617465206461DD
:109A80007461200A0D0000007265636569766520C7
:109A90006368617267652064617461200A0D00006B
:109AA000456E61626C65000044697361626C6500BB
:109AB0006368617267652025730A0D003505002013
:109AC0000C02002036050020706172616D20726505
:109AD00061640A0D00000000706172616D20777290
:109AE0006974650A0D000000706172616D20616427
:109AF00064722025780A0D00656E61626C65000055
:109B000064697361626C65006368617267696E673E
:109B10002025730A0D000000636C6F736520726569
:109B20006C61790A0D0000006F70656E2072656CC3
:109B300061790A0D00000000626C7565746F6F74C6
:109B400068206E616D652025730A0D00626C756575
:109B5000746F6F7468206E616D65206D69737461D8
:109B60006B652025730A0D0048656172742042659B
:109B700061742054696D6520256420207365630A33
:109B80000D0000004F76657254656D7056616C75FE
:109B9000652025642020200A0D00000053797350B1
:109BA00061726150696C65442E736E3A25730A0DBB
:109BB000000000005379735061726150696C654414
:109BC0002E736E206661756C742025730A0D00007B
:109BD000517569636B2043686172676520456E61EA
:109BE000626C650A0D000000747269636B6C65201D
:109BF0004368617267696E6720536F6320456E61C9
